:100000005446495300010000089B0100C2558C155D
:10001000050901121511031848304130050901285E
:10002000151103184830413005090108151103174F
:1000300048304130030000000000000000000000D4
:100040005446435300200000048B010000000000D0
:10005000004001200121000025210000272100008F
:10006000292100002B2100002D2100003D2100004E
:100070003D2100003D2100003D2100002F21000016
:10008000312100003D210000332100000B5400000D
:100090000B550000372100003D2100001106001023
:1000A000372100008D360000E13600003D210000C0
:1000B0003D210000DF500000372100003721000003
:1000C000134E0000372100003D2100003D210000BB
:1000D0000000000000000000000000000000000020
:1000E0000000000000000000000000000000000010
:1000F0000000000000000000000000000000000000
:1001000000000000000000000000000000000000EF
:1001100000000000000000000000000000000000DF
:1001200000000000000000000000000000000000CF
:1001300000000000000000000000000000000000BF
:1001400000000000000000000000000000000000AF
:1001500000F003F800F020F8FEE70D48016821F0F8
:100160000301002001C101C101C101C170470000AC
:10017000E40B0010FEE7FEE7FEE7FEE7FEE7FEE722
:10018000FEE7FEE7FEE703480047FEE7FEE7000064
:10019000202100003D21000000F002F800F068F886
:1001A0000AA090E8000C82448344AAF10107DA45D2
:1001B00001D100F05DF8AFF2090EBAE80F0013F0BC
:1001C000010F18BFFB1A43F001031847F87C010028
:1001D000287D01000A444FF0000C10F8013B13F099
:1001E000070408BF10F8014B1D1108BF10F8015B90
:1001F000641E05D010F8016B641E01F8016BF9D183
:1002000013F0080F1EBF10F8014BAD1C0C1B09D1D9
:100210006D1E58BF01F801CBFAD505E014F8016B4B
:1002200001F8016B6D1EF9D59142D6D370470000DD
:10023000103A24BF78C878C1FAD8520724BF30C812
:1002400030C144BF04680C607047000000230024E4
:1002500000250026103A28BF78C1FBD8520728BFD6
:1002600030C148BF0B6070471FB51FBD10B510BD32
:10027000DFF80CD0FFF7F8FF04F048FA14F0EEFEB8
:100280000040012003B4FFF7F1FF03BC14F0EEFEC1
:100290007047002818BF0120FE49096808627047AE
:1002A000FC480068006A002818BF01207047F94A1E
:1002B000126802EBC00041637047F649096801EB20
:1002C000C000006B00F480707047F24A1021126881
:1002D00002EBC00041637047EE490A68D2F8402142
:1002E00060F30D220868C0F840217047E9480068B3
:1002F000D0F84001C0F305207047E64A00F00F0334
:10030000C0F303101268002902EBC31202EB401085
:10031000D0F8401114BF41F0010121F00101C0F8F3
:1003200040117047DB4A00F00F01C0F30310126860
:1003300002EBC11101EB4010D0F8400100F00100C8
:100340007047D44900230A6813620268D1F800C0DC
:10035000CCF800204268D1F800C0CCF804208268B4
:10036000D1F800C0CCF80820C268D1F800C0CCF8A1
:100370000C20426AD1F800C0CCF84020826AD1F843
:1003800000C0CCF844200269D1F800C0CCF8182095
:100390004269D1F800C0CCF81C20826BD1F800C0B3
:1003A000CCF86020C26BD1F800C0CCF87020026C91
:1003B000D1F800C0CCF87420426CD1F800C0CCF861
:1003C0007820826CD1F800C0CCF88020C26CD1F8C3
:1003D00000C0CCF88420026DD1F800C0CCF8882091
:1003E000426DD1F800C0CCF88C20426ED1F800C02C
:1003F000CCF89C20826ED1F800C0CCF8A020C26E50
:10040000D1F800C0CCF8A420026FD1F800C0CCF81D
:10041000A820826FD1F800C0CCF8C020C26FD1F8FC
:1004200000C0CCF8C420D0F88020D1F800C0CCF8AF
:10043000C820D0F88420D1F800C0CCF8CC20D0F867
:100440008820D1F800C0CCF8D020D0F88C20D1F88A
:1004500000C0CCF8D420D0F89420D1F800C0CCF85B
:10046000DC20D0F89C20D1F800C0CCF8F020D0F8E7
:10047000A020D1F800C0CCF8F420D0F8A420D1F806
:1004800000C0CCF8F820D0F8A820D1F800C0CCF8F3
:10049000FC20D0F8AC20D1F800C0CCF80021D0F876
:1004A000B020D1F800C0CCF80421D0F8B420D1F8A5
:1004B00000C0CCF80821D0F8B820D1F800C0CCF8A2
:1004C0000C21D0F8BC20D1F800C0CCF81021D0F815
:1004D000C020D1F800C0CCF81421D0F8C420D1F845
:1004E00000C0CCF81821D0F8C820D1F800C0CCF852
:1004F0001C21D0F8CC20D1F800C0CCF82021D0F8B5
:10050000D020D1F800C0CCF82421D0F8D420D1F8E4
:1005100000C0CCF83021D0F8D820D1F800C0CCF8F9
:100520004021D0F8DC20D1F800C0CCF84421D0F82C
:10053000E020D1F800C0CCF84821D0F8E420D1F870
:1005400000C0CCF84C21D0F8E820D1F800C0CCF89D
:100550005021D0F8EC20D1F800C0CCF85421D0F8CC
:10056000F020D1F800C0CCF85821D0F8F420D1F810
:1005700000C0CCF85C21D0F81821D1F800C0CCF82C
:100580008021D0F81C21D1F800C0CCF88421D0F80B
:100590002021D1F800C0CCF88821D0F82421D1F84E
:1005A00000C0CCF88C21D0F82821D1F800C0CCF8BC
:1005B0009021D0F82C21D1F800C0CCF89421D0F8AB
:1005C0003021D1F800C0CCF89821D0F83421D1F8EE
:1005D00000C0CCF89C21D0F83821D1F800C0CCF86C
:1005E000A021D0F83C21D1F800C0CCF8A421D0F84B
:1005F0004021D1F800C0CCF8B021D0F84421D1F886
:1006000000C0CCF8C021D0F84821D1F800C0CCF807
:10061000C421D0F84C21D1F800C0CCF8C821D0F8C2
:100620005021D1F800C0CCF8CC21D0F85421D1F819
:1006300000C0CCF8D021D0F85821D1F800C0CCF8B7
:10064000D421D0F85C21D1F800C0CCF8D821D0F862
:100650006021D1F800C0CCF8DC21D0F86421D1F8B9
:1006600000C0CCF8E021D0F86821D1F800C0CCF867
:10067000E421D0F86C21D1F800C0CCF8E821D0F802
:100680007021D1F800C0CCF8EC21D0F87421D1F859
:1006900000C001E088920100CCF8F021D0F8782168
:1006A000D1F800C0CCF8F421D0F87C21D1F800C0FA
:1006B000CCF8F821D0F88021D1F800C0CCF8FC218A
:1006C000D1F800C02122CCF83420D1F800C0CCF8F9
:1006D0003C20C269D1F800C0CCF82420C26AD1F80D
:1006E00000C0CCF84820026BD1F800C0CCF84C20F8
:1006F000426FD1F800C0CCF8AC20D0F89820D1F8E7
:1007000000C0CCF8E020D0F88421D1F800C0CCF8AB
:100710000022D0F88821D1F800C0CCF80422D0F80B
:100720008C21D1F800C0CCF80822D0F89021D1F863
:1007300000C0CCF80C22D0F89421D1F800C0CCF83D
:100740001022D0F89821D1F800C0CCF81422D0F8AB
:100750009C21D1F800C0CCF81822D0F8A021D1F803
:1007600000C0CCF81C22D0F8A421D1F800C0CCF8ED
:100770002022D0F8A821D1F800C0CCF82422D0F84B
:10078000AC21D1F800C0CCF83022D0F8B021D1F89B
:1007900000C0CCF84022D0F8B421D1F800C0CCF889
:1007A0004422D0F8B821D1F800C0CCF84822D0F8C3
:1007B000BC21D1F800C0CCF84C22D0F8C021D1F82F
:1007C00000C0CCF85022D0F8C421D1F800C0CCF839
:1007D0005422D0F8C821D1F800C0CCF85822D0F863
:1007E000CC21D1F800C0CCF85C22D0F8D021D1F8CF
:1007F00000C0CCF86022D0F8D421D1F800C0CCF8E9
:100800006422D0F8D821D1F800C0CCF86822D0F802
:10081000DC21D1F800C0CCF86C22D0F8E021D1F86E
:1008200000C0CCF87022D0F8E421D1F800C0CCF898
:100830007422D0F8E821D1F800C0CCF87822D0F8A2
:10084000EC21D1F800C0CCF87C22FA4A126832F0D0
:10085000FF0C08D1D1F800C0DCF890C062F3030CA3
:100860000A68C2F890C0F44A1370836F13F0010F46
:100870001CBF02231370D0F8880010F0010F03D0C2
:10088000107840F0010010700868D0F8C0000A68C5
:1008900020F00100C2F8C0000868D0F8D000096854
:1008A00020F00100C1F8D0007047E349087070479C
:1008B000E2480068D0F8C00000F001007047DF484F
:1008C0000068C068704770B5DC4D04462868D0F8F1
:1008D000400114F0020F20F00D0118BF41F001019A
:1008E00014F0080F18BF41F0040114F0040F18BFF2
:1008F00041F008012868C0F8401114F0010F70D0D1
:1009000001F031F8064601F031F801462868C06868
:1009100000280EBF30460846314600282868D0F827
:10092000C00114BF40F0010020F001002A68C2F8A5
:10093000C00128680029D0F8E00114BF40F0010090
:1009400020F001002968C1F8E001BB4890F800C020
:100950001CF0010F5DD0BA480168496C026841F48F
:10096000803151640168896CC1F3090240F2E731BA
:1009700003689B6CC3F30903934202D1491EF7D16C
:1009800017E0B1B11CF0010F07D02868D0F8D000F3
:10099000296840F00100C1F8D0001CF0020F38D0E7
:1009A0002868D0F8C000296840F00100C1F8C000F4
:1009B0002FE02968D1F8D0102A6821F00101C2F88F
:1009C000D0102968D1F8C0102A6821F00101C2F8BE
:1009D000C0100168496C006821F48031416418E05E
:1009E000FFE72868D0F8C001296820F00100C1F8AD
:1009F000C0012868D0F8E001296820F00100C1F8A2
:100A0000E0012868D0F8C000296820F00100C1F892
:100A1000C00014F0200F18BF002413D0204600F0AF
:100A2000ACFF0028286800EB4410D0F8401214BF37
:100A300041F0010121F00101C0F84012641C022CB8
:100A4000ECD370BD2868D0F84002296820F001007E
:100A5000C1F840022868D0F86002296820F001003F
:100A6000C1F8600270BD2DE9F0037449024602F03E
:100A70000F03D1F800C000200CEBC315C2F3031321
:100A800005EB4313D3F8403113F0010F0DD142F0C1
:100A90001003C3F3031305EB4313D3F8403113F0F2
:100AA000010F04BFBDE8F00370470CEBC214D4F88B
:100AB0001C31DCF81C10C3F3080901F00807D4F856
:100AC0000011C1F30A08002142EA0113C3F3031322
:100AD00005EB4313D3F8403113F0010F14D004EBAE
:100AE0004113D3F844C1CCF3080617F1000C1CBF26
:100AF000D3F844C1CCF3023CD3F8403106FA0CFCE5
:100B0000C3F3054360441844491C0229DCD300FBAD
:100B100008F0C9EB0911BDE8F00300EB4100704794
:100B200070B5464801680968006801F01F06406812
:100B3000C0F30C050120FFF796FF04460220FFF7E3
:100B400092FF044400F073FB211805FB06F0C0EB94
:100B5000001001EB40004FF47A71484347F23051E6
:100B6000B0FBF1F070BD2DE9F041344F0546386817
:100B7000006810F01F0408BF01240120FFF773FF75
:100B800006460220FFF76FFF064400F050FB2D4A97
:100B90003118B5B1B2FBF5F0884298BF00200AD9F0
:100BA000C4EB0413401A5B00B0FBF3F0B0F5005F38
:100BB00088BF41F6FF703B685B6860F30C033868E0
:100BC000436038684068C0F30C006043C0EB00101D
:100BD00001EB4000B2FBF0F0BDE8F08170B51748C2
:100BE00001680968006801F01F054068C0F30C0641
:100BF0000120FFF738FF04460220FFF734FF0444CA
:100C000000F015FB06FB05F1C1EB011104EB4101FE
:100C100008440C49B1FBF0F070BD08490A685268FD
:100C20000B68C2F30C025B6860F30C030868436056
:100C300010467047E0FE030000400020889201004B
:100C40008492010000389C1CF84800684068C0F39A
:100C50000C007047F549096801EBC010D0F800019D
:100C60004EF66021C0F30A00B1FBF0F0401C4008D2
:100C700070474EF66022B2FBF1F1491C4908B2FB05
:100C8000F1F2F0B4E94D521C56082A684FEA510CB3
:100C900002EBC01238B1D2F804318C1F24F00104E9
:100CA000012806D019E0ACF10603981F20F00104DA
:100CB00013E02868D0F8D00010F0010F0DD04800E4
:100CC000B0F5006F88BF40F2FF702F68D7F8E07072
:100CD00060F30A072868C0F8E07041EA0C40C2F8E7
:100CE0000001C2F80431C2F810413046F0BC704730
:100CF000CE4A00F00F01C0F30310126802EBC111DD
:100D000001EB4010D0F84401C0F308007047C74A17
:100D100000F00F03126802EBC312D2F81431C0F3D3
:100D2000031002EB4010CB1AD0F844219B1E61F354
:100D30000802C0F84421D0F8441163F31841C0F808
:100D400044117047B9490A68D269096812F0100F56
:100D500000F00F0201EBC211D1F82021C0F3031003
:100D600001EB4010D2B2D0F84401C0F3080008BF34
:100D70000022801A0004000C08BF012070474FEACF
:100D8000101C0007C00EAA4B02FA00F01B6803EB10
:100D9000CC1303EB810101F5C0410B6818430860D7
:100DA0007047A34B020900071B68C00E03EBC21279
:100DB00002EB810101F5C041096821FA00F000F061
:100DC0000300704799480068006D704797491020EC
:100DD0000968C8657047954B00F00F02C0F3031017
:100DE0001B6803EBC21202EB4010C0F84C117047B5
:100DF0008E4A00F00F01C0F30310126802EBC1111C
:100E000001EB4010D0F84C017047884B00211A6864
:100E1000D26912F0080F0CD000F00F011A68C0F36D
:100E2000031002EBC11101EB4010D0F84401C0F3F4
:100E30000231084670477D4A1368DB69D2F800C06A
:100E400043F00803CCF81C3000F00F031268C0F325
:100E5000031002EBC31202EB4010D0F8442161F3FF
:100E60000E32C0F844217047704B00211A68D269D5
:100E700012F0080F0CD000F00F011A68C0F3031035
:100E800002EBC11101EB4010D0F84801C0F3024160
:100E900008467047654A00F00F03C0F3031012685C
:100EA00002EBC31202EB4010D0F8482161F312426A
:100EB000C0F848217047042988BF704730B4002328
:100EC0005A4C2268D269254612F0080F00F00F0232
:100ED0002D68C0F3031005EBC21202EB40121CBFD9
:100EE000D2F84401C0F302330020D4F800C0DCF88B
:100EF0001CC01CF0080F1CBFD2F84801C0F3024010
:100F0000C91A0844042803DD081A011D042003E05F
:100F10000028BCBF0144002019442368DB69D4F8D1
:100F200000C043F00803CCF81C30D2F8443161F320
:100F30000E33C2F84431D2F8481160F31241C2F8BE
:100F4000481130BC7047394900280868806904D0CE
:100F5000096840F0080088617047096820F00800BF
:100F600088617047314A00F00F01C0F30310126826
:100F700002EBC11101EB4010D0F8480180B270477C
:100F80002A4B00211A68D26912F0080F0CD000F029
:100F90000F011A68C0F3031002EBC11101EB4010FE
:100FA000D0F84801C0F30051084670471F490200BD
:100FB000086880690A6800F00100926904D0096835
:100FC00042F001028A617047096822F001028A61D9
:100FD000704730B4022ADDF808C026BF921E5208BE
:100FE0000022022B26BF9B1E5B080023114C00F041
:100FF0000F05A4FB0C4C4FEA1C14DFF830C0C0F303
:101000000310DCF800C00CEBC51C0CEB4010D0F852
:1010100054C161F3196C62F3134C63F30B2C64F34A
:10102000070CC0F854C130BC704700008892010022
:10103000A0920100CDCCCCCC70B49B4D00F00F043D
:10104000C0F303102D68DDF80CC005EBC41404EBED
:101050004010D0F854010029C0F30166C0F30345E5
:10106000C0F30324C0B218BF0E6012B16900891C1E
:10107000116013B16100891C1960BCF1000F04BF3D
:1010800070BC704700EB80008000CCF8000070BCA2
:10109000704770B491B000224FF480456C10EC465C
:1010A00001E0082A05D2531C03EB8303B5FBF3F3DD
:1010B00004E0D31F03EB8303B4FBF3F35B1A002BB1
:1010C000B8BF5B424CF82230521C102AE9D30026EC
:1010D000009B01215CF821209A42BCBF13460E46BA
:1010E000491C1029F6D3704900F00F02C0F3031019
:1010F000096801EBC21101EB4011D1F85801C1F8A8
:101100005861082807D2401C00EB8000B5FBF0F0C6
:1011100011B070BC7047C01F00EB8000B4FBF0F052
:1011200011B070BC7047604A00F00F01C0F30310AB
:10113000126802EBC11101EB4010D0F858010828E9
:1011400034BF401CC01F00EB800034BF4FF480410F
:101150004FF40051B1FBF0F0704710F00F0F08BFD3
:101160007047514A00F00F000029126802EBC010CE
:10117000D0F824110CBF21F4803141F48031C0F843
:1011800024117047002110F00F0F0BD0464A00F0D9
:101190000F00126802EBC010D0F8240110F4803F59
:1011A00018BF0121084670473F4902460868D0F839
:1011B000AC0012F0010F0A68C0F3C000D2F8AC20F6
:1011C00005D0096842F00802C1F8AC2070470968F0
:1011D00022F00802C1F8AC207047334A1368586700
:1011E000106881677047304900280868D0F8AC0063
:1011F00005D0096840F00200C1F8AC0070470968EA
:1012000020F00200C1F8AC007047274900280868A8
:10121000D0F8AC0005D0096840F00100C1F8AC007E
:101220007047096820F00100C1F8AC00704770B445
:101230001D4E00203168D1F8401111F0010F04BF9C
:1012400070BC704711F0040F336801F00805D3F843
:101250001C31D6F800C0C3F30803DCF800C1CCF39E
:101260000804D6F800C0DCF844C1CCF3080C18BF61
:10127000C1F307403268D269C1F3052112F00802B8
:1012800004D03268D2F84421C2F30232002D18BFD4
:10129000491C0CFA02F201FB0200604370BCC3EB74
:1012A000031100EB4100704788920100FEF7F8BF80
:1012B00010B5FEF7F5FF012818BF10BD0020FEF79E
:1012C000E8FF21210020FEF7F2FF2121BDE81040B8
:1012D0000120FEF7ECBF10B5FEF7DAFFFEF7E0FFE6
:1012E00001280AD10020FEF7D4FF21210020FEF7BB
:1012F000DEFF21210120FEF7DAFF0121052001F0A8
:1013000068FC0121052001F064FCFF4900204870C1
:1013100010BD10B5602001F0B2FCBDE810406020A7
:1013200001F0A0BCF84A0146507A002818BF0120FD
:10133000002918BF012151727047F34A91699061E9
:1013400008467047F04800210172C1717047EE48AD
:1013500000210172C17170472DE9F34F00F00F05B4
:101360006800861E9DB0002445EA0410FEF7DAFFEF
:1013700000284DD01E9AC4EBC400002102EB0017D8
:10138000EC46C1EBC10307EBC30200200CEBC30327
:1013900052F8208043F82080401C0E28F8D3491CC6
:1013A0000229EED3D9490022301909684FF002080A
:1013B000C0EBC000434601EB001723FA02F101F035
:1013C0000101C1EBC101C2EBC2000CEBC10107EB93
:1013D000C00091E8004E00F58840521CC0E9CE9A4A
:1013E000C0E9D0BE01F11009424599E8004EC0E9BC
:1013F000D29AC0E9D4BE01F1200999E8004EC0E9B3
:10140000D69AC0E9D8BED1E90C91C0E9DA91D4D31B
:10141000641C022CA8D31FB0BDE8F08F70B5054640
:10142000FEF764FF29460446B84DC0EBC400C20075
:10143000286800F5804013F01FFE2968C4EBC40043
:1014400001EBC00000F58040002101604160816037
:10145000C160016141618161C1610162416281627A
:10146000C1620163416370BDA7494861FFF72BBAB0
:10147000A74801688968A74A11430268916001681A
:101480000968A54A00681143016000F077BE2DE9A4
:10149000F0479F4A06460D46106880689D49014303
:1014A00010688160106800689B49084311680860F3
:1014B00000F064FE0024944F002D63D00020FEF75E
:1014C000E8FE286820B1FEF73CFF0020FEF7E1FEB1
:1014D00030467E61FFF7F7F90020FEF723FF002872
:1014E00034D0DFF828826E6816B3FEF7FFFE81461F
:1014F000C0EBC900C200D8F80000314600F58040BA
:1015000013F0BAFDD8F80010C9EBC90001EBC00018
:1015100000F58040046044608460C46004614461FC
:101520008461C461046244628462C462046344638B
:10153000E96841B1D8F800004FF4807200F5C0406E
:1015400013F09AFD02E0754800F038FD0120FEF727
:10155000E9FE18B91120FEF7E5FE28B1A9680029B7
:101560001CBF0120FFF7F8FE0220FEF7DBFE18B9D2
:101570001220FEF7D7FE28B1296900291CBF0220DE
:10158000FFF7EAFE3C72FC71BC61787A0020787249
:10159000602001F074FBBDE8F047602001F062BB01
:1015A00010B50020FEF775FE00F0CAFD584801682E
:1015B0000968026821F0030141F00D7141F080518A
:1015C000116001688968006821F0020141F00D7125
:1015D00041F08051816010BD602001F047BB10B523
:1015E000602001F043FBFEF75BFE01280AD10020DA
:1015F000FEF74FFE21210020FEF759FE2121012098
:10160000FEF755FE46480168496C006821F48031B8
:1016100041640020FEF73DFE00F092FD3C48016869
:101620000968026821F0030141F00D7141F0805119
:10163000116001688968006821F0020141F00D71B4
:1016400041F08051816010BD2F48406970472E489D
:101650000078002818BF0120704770B5FEF720FE03
:10166000002818BF70BD0025274C2572E571212187
:101670002846FEF71CFE21210120FEF718FE2570EA
:10168000BDE870400120FEF704BE10B5FEF708FE6D
:10169000002818BF10BD00201B4C2072E0712121D2
:1016A000FEF705FE21210120FEF701FE0120FEF7D5
:1016B0000CFE01202070BDE81040FEF7EABD0020BE
:1016C000FEF7E7BD10490020C8710120FEF7E1BD1B
:1016D0000D49C86170470C48C069704770B50A4C25
:1016E0000025E069411CE161207800281CBF002032
:1016F000FEF7CFFD20212846FEF7D9FDA16900297C
:101700001CBF284688470DE004400020A09201003D
:10171000909201000200341203003412384200207B
:1017200084920100FB48016841F02001016070BD16
:1017300070B5F94C0125E069411CE1612078002871
:101740001CBF0020FEF7A5FD20212846FEF7AFFDB7
:10175000A16900291CBF28468847EE48016841F06E
:101760002001016070BDED487047ED487047EA48C0
:10177000006A7047E848406A70472DE9F007DFF8D3
:101780009C834FF0000C87B008F1380665464FF097
:10179000FF3408F80C4006F80C500CF1010CBCF1B9
:1017A0001C0FF6DB4FF0000C002807D912F80C7064
:1017B00008F80C700CF1010C6045F7D80027B94609
:1017C0004FF0010C002810D918F90720002A09DB76
:1017D000082AB4BF1432083A1C2A3CBF0CFA02F2A1
:1017E00042EA09097F1C8742EED3002002466F4679
:1017F0000CFA02FA1AEA090F1ABFB854401CBC547A
:10180000521C1C2AF4DB0022002816D918F9029079
:10181000B9F1000F0EDBB9F1080FB4BF09F11409DB
:10182000A9F10809B9F11C0F3ABF17F8099006F899
:101830000290B454521C8242E8D3DFF8DC820022CA
:101840000028C8F8205009D916F90290914502D015
:10185000C8F8206002E0521C8242F5D3B04E00204E
:1018600006F1380234541554401C1C28FADB0020C1
:10187000002906D913F8009006F80090401C814218
:10188000F8D80023994600290BD9F056002805DB2B
:101890001C283CBF0CFA00F040EA09095B1C8B4293
:1018A000F3D3002001460CFA01F313EA090F1ABF23
:1018B0007854401C7C54491C1C29F4DB002100286E
:1018C00009D97356002B03DB1C2B3CBFFB5C535424
:1018D000491C8142F5D30021C8F8245000289EBF3E
:1018E00007B0BDE8F007704753568B4205D0C8F8E3
:1018F000242007B0BDE8F0077047491C8142F3D3AC
:1019000007B0BDE8F0077047C0EB0010854900EB59
:10191000C00001EBC0007047C0EBC00101EB00103C
:10192000814901EB80007047DFF8ECC1012B8CF896
:1019300002008CF8031003D9401C20F0010011466E
:1019400000FB01F24FF6FF718CF8040001EA42023D
:10195000ACF80C2001EA4000ACF80E0070476E4A6B
:101960005071917170476C48807970476A4840792E
:1019700070476E4A1070517070476C49085C704730
:1019800070B5654D0446687A002804BFE87913F005
:101990000CFC287A002808BF70BD4FF0000C686965
:1019A00063466246614610F0020F09D0DFF874C149
:1019B00010F0040F04D0AB89664623F001033344D2
:1019C00010F0010F04D010F0100F0CBF564A56490A
:1019D000ED692560C4E90321C4E901C310F0200FBB
:1019E00014BF534800206061012070BD4A490020A7
:1019F0000872704710B50446FEF778FCC0EBC000D3
:101A0000C2004C48006800F580412046BDE8104007
:101A100013F032BB2DE9F041FEF768FC04460020CC
:101A2000FFF7E6F90022002C84BF0125414E21D9A1
:101A3000D6F800C0C2EBC20300210CEBC30C05FAC0
:101A400001F3034210D04B080CEB830303F58043F2
:101A5000CF071B68FF0EFB40C3F30B03B3F57F6F8B
:101A600002D90020BDE8F081491C1C29E7D3521C93
:101A7000A242DDD30120BDE8F0812DE9F35F00F043
:101A80000F070024DFF8AC807E0044F2387547EA87
:101A90000410FEF747FC002835D00222019BC4EB5E
:101AA000C4009246002103EB001B4FF0000C002AFB
:101AB00009D92AFA0CF000F0010088421CBF0CF191
:101AC000010C9445F5D394451AD2A6F10209A1441C
:101AD000D8F800E0C1EBC100C9EBC9090BEBC003AA
:101AE0000EEB0919CCEBCC0C002009EBCC0909EB6F
:101AF000800C5CF805C043F820C0401C0E28F6D3CB
:101B0000491C0229D1D3641C022CC0D302B0BDE809
:101B1000F09F0000304000200440002038420020A8
:101B200054420020A8420020E04600200E40002041
:101B30003C470020A09201002DE9F05F00F00F0665
:101B400070000024A0F1020B012744F2387846EA25
:101B500004194846FEF7E6FBA0B34846FFF755F9DF
:101B600007FA00F54846FFF743F90022002D29D96E
:101B70000BEB0401C1EBC101FE4B1B6803EB011A27
:101B8000C2EBC20300210AEBC30907FA01F30342C7
:101B900012D04B0809EB83034FEAC17C53F808309D
:101BA0004FEADC6C23FA0CF3C3F30B03B3F57F6F3E
:101BB00002D90020BDE8F09F491C1C29E5D3521C26
:101BC000AA42DDD3641C022CC1D30120BDE8F09FE2
:101BD000C1EBC103E7494FF6FF7C096801EBC30184
:101BE000430801EB830101F58041C007C00E0CFAE8
:101BF00000FC0B6802FA00F023EA0C0318430860AB
:101C00007047DC4AC1EBC101126802EBC101420816
:101C100001EB820101F58041C0070968C00E21FA7D
:101C200000F080B270472DE9FF4FD24883B01D46C7
:101C30000068109C00F5804017460E460190FEF7A4
:101C40002FFB5FEA00081CBF0020FEF722FB0020EC
:101C5000FFF7CEF8824670190090B04284BF4FF073
:101C6000010B4FF6FF7E28D90198C6EBC6014FF055
:101C7000000C00EBC101039B17E00BFA03F010EA24
:101C80000A0F11D05808DD0751F82020ED0E0EFA8A
:101C900005F922EA090234F8029B0CF1010C09FA59
:101CA00005F52A4341F820205B1CBC4538BF1C2B9E
:101CB000E3D30098761C8642D6D3B8F1000F04BF58
:101CC00007B0BDE8F08F0020AB49C87107B0012014
:101CD000BDE8F04FFEF7DDBA2DE9F0470746A5480D
:101CE0009A46144600680E46089D00F58049FEF7A6
:101CF000D7FA5FEA00081CBF0020FEF7CAFA06EB1D
:101D00000A03B34284BF9D4907EB040C1CD9C6EB00
:101D1000C6003C4609EBC0000FE00A571C2A0BD254
:101D200002EBD27A4FEA6A0AD20750F82AA0D20E02
:101D30002AFA02F225F8022B641C644538BF1C2CD9
:101D4000EBD3761C9E42E2D3B8F1000F08BFBDE88A
:101D5000F08700208849C871BDE8F0470120FEF7F0
:101D600098BA2DE9F05F0027DFF80C82814A4FF620
:101D7000FF7600280C4646D0116801F5804900F036
:101D80000F01C0F3031001290EBF00210229BDE895
:101D9000F09F022828BFBDE8F09F01EB000AFEF784
:101DA0007FFA05001CBF0020FEF773FA0020CAEB83
:101DB000CA0109EB0119C0EBC001002209EBC10CFB
:101DC00051080CEB810303F5E761D3F838A7D3077B
:101DD000DB0E06FA03FB04FA03F32AEA0B0A4AEACB
:101DE0000303521C0B601C2AEAD3401C0228E2D3D6
:101DF000002D08BFBDE8F09F88F80770BDE8F05FD0
:101E00000120FEF746BA106800F58049FEF748FA4F
:101E100005001CBF0020FEF73CFA4FF0000CCCEB95
:101E2000CC00002209EBC0015308D007C00E06FA0F
:101E300000FB51F823A004FA00F02AEA0B0A4AEA50
:101E40000000521C41F823001C2AEDD30CF1010CB8
:101E5000BCF1210FE3D3002DCED1BDE8F09F10B52A
:101E6000FEF770FF4449088210BD434AC1B200F436
:101E70007063128A914288BF11464FF0640C01FBD7
:101E80000CF1B1FBF2F11A0A02FB0C1189B210F449
:101E9000805F12BF08B2484200B270470028B8BF46
:101EA000404280B2B4BF00214FF4805100F4706210
:101EB0001143314AC0B2128A504341EA10207047A0
:101EC0002F4800F07BB8FFF73EB870B52C4800F003
:101ED00075F8284840F6F801006800F5804013F0D6
:101EE000D0F80020FEF799FE00210846FEF7A3FF78
:101EF00000210120FEF79FFF00211120FEF79BFF2C
:101F000000210846FEF7C6FF00210120FEF7C2FFB0
:101F100000211120FEF7BEFF0120FEF79BFE0446C4
:101F20000120FEF7E5FE06461120FEF7E1FE05461C
:101F3000A64288BF2646A54288BF254631460120D5
:101F4000FEF7E5FE29461120FEF7E1FE0020FEF730
:101F5000ACFC00210220FEF76EFF00211220FEF7EC
:101F60006AFF00210220FEF795FFBDE870400021C6
:101F7000122007E0A09201000440002054420020FB
:101F800038420020FEF786BF214910B50220486183
:101F9000FEF799FC1F4C4FF48071206800F5C0409B
:101FA00013F06FF820684FF4E76100F5804013F0FC
:101FB00068F8BDE810400020FEF72FBE70B5154D43
:101FC00004464FF48071286800F5C04013F059F8BA
:101FD000002101206256002A15DBD31702EB137C87
:101FE0004FEA2C132E682CF00F0C06EBC31303EBF7
:101FF000810303F5C043A2EB0C0252001E6800FAF5
:1020000002F232431A60491C1C29E3D370BD000060
:1020100004400020A092010070B400246E4982B0F8
:102020004FF0010C002814BF0C7081F800C06B4DFC
:10203000286800686A4A10432A6810600978694A6B
:1020400031B113686848D86013686848986006E042
:1020500013686748D86013684FF0BB709860654894
:10206000006830F0FF0305D11368DB6860F30303F9
:102070001068C36040F2E243D1B11068806816680E
:1020800040F01800B0600120009005E00198461E65
:1020900001960028FAD10098461E0096002818BF25
:1020A0000193F3D110688068166840F48050B060E6
:1020B0000120009005E00198461E01960028FAD103
:1020C0000098461E0096002818BF0193F3D11068AF
:1020D000C068166840F03000F0601068D0F8B000BA
:1020E000166840F00100C6F8B0000120009005E03D
:1020F0000198461E01960028FAD10098461E0096C7
:10210000002818BF0193F3D11068C0F87CC0136891
:102110004FF4E06018611068C0F8884000291CBFC7
:102120001068C0F894C028680068296820F004008E
:1021300040F00D7040F08050086002B070BC7047F5
:1021400028480168C968026821F03001D16022493D
:10215000097839B101688968006821F0180121F413
:10216000805181601D4801680968006821F0040100
:1021700041F00D7141F080510160704717480168CE
:102180000968174A0068114301601348017815482F
:1021900031B10168896841F2180211430268916007
:1021A0000168C968026841F03001D1600168D1F866
:1021B000B010006841F00101C0F8B01070470E493E
:1021C000C0B241EA00200749096808647047054920
:1021D0000A480968086470472C400020909201006A
:1021E000040034128C920100057601002000760173
:1021F00005F40100D0FE030013005FA000005FA003
:1022000059485849026891610268891CD161026885
:10221000491E516302681268036822F0030242F00B
:102220000D7242F080521A6002685269036822F00F
:10223000010242F00D7242F080525A610268126946
:102240001143026811610268484991600068484979
:10225000C160484900200860704770B501F06DF911
:10226000444D2C682CB10020286001F06BF9204609
:1022700070BD30BF00F0BFFD0028F2D000F0CEFDF1
:102280006860EEE72DE9F04101F057F9354E364C24
:10229000DFF8E080771CD8F800503DB10020C8F886
:1022A000000001F04FF92846BDE8F08172B62068C1
:1022B00046632068876120BF206886612068476385
:1022C00062B6BFF36F8FBFF34F8F00F094FD00280D
:1022D000E1D000F0A3FDC8F80400DCE72248016863
:1022E0000968026821F0030141F00D7141F080514D
:1022F0001160026820499160016809691F4A0068FD
:102300001143016130BF704772B616491648026822
:1023100051630268C91CD1610068891E816162B67F
:102320007047114801680968154A00681143016047
:1023300070470D4801680968006821F0030141F009
:102340000D7141F080510160704772B60549064831
:10235000026891610268891CD1610068491E41636D
:1023600062B6704700003412909201003C003412B3
:1023700028003412304000200800341201003412CA
:10238000030034127047002818BF0120B6490968BD
:10239000486070470022002908D950F8043B5B1CB4
:1023A00001D000207047521C8A42F6D301207047AA
:1023B00030B44FF0000C6346002A13D950F8044B98
:1023C00051F82350AC421CBF0CF1010C1FFA8CFCDD
:1023D0005B1C9BB29342F1D3BCF1000F1EBF0020E7
:1023E00030BC7047012030BC70472DE9F0410546F4
:1023F00001F0ADF800249C4B21274FF4825826466B
:10240000186807602E6018680068196840F00400BA
:1024100008601868006810F0040FFAD11868C0F856
:10242000008040202946002251F804CB1CF1010C09
:1024300008D018680660601CC4B2082CE0D30220E3
:10244000BDE8F081521C8242EED31868066001207C
:10245000BDE8F0812DE9F041044601F078F8002054
:10246000814B0925844619680D60C4F800C01968BD
:1024700009681A6841F0040111601968096811F0CF
:10248000040FFAD121464FF48066002251F8047BF4
:102490007F1C09D01968C1F800C0401CC0B20328D5
:1024A000E1D30220BDE8F081521CB242EED318689D
:1024B000C0F800C00120BDE8F0812DE9F05F0F46B3
:1024C000804604264FF0020A4FF0000BDFF8989187
:1024D00001F03DF8D9F80000C0F800A044463846A5
:1024E0000F2190E82C10A4E82C101030491EF8D2CF
:1024F000D9F800000068D9F8001040F00400086026
:10250000D9F80000006810F0040F07D000BF00BF2A
:10251000D9F80000006810F0040FF7D1D9F80000D6
:10252000C0F800B0454638460F21D5E90023D5E96B
:1025300002C4D0F800E0964504BF42689A4205D133
:102540008268624504BFC268A24208D0761E03D3E7
:102550004046FFF74AFFBBE70220BDE8F09F103579
:102560001030491EE1D20120BDE8F09F70B50D4644
:10257000044600F0ECFF4FF480722146284612F02A
:102580007BFD012070BD2DE9F041C0B014460E4620
:10259000054610F0FF0F23D025F0FF086F4600F02E
:1025A000D6FF4FF480724146384612F065FDE8B21E
:1025B000C0F58077A74288BF274668443A4631462F
:1025C00012F064FD4046FFF710FF022843D0694631
:1025D0004046FFF772FF022841D03D443E44E41BD1
:1025E000B4F5807F19D34FF480723146684612F0FB
:1025F0004DFD2846FFF7F9FE02282CD069462846F3
:10260000FFF75BFF02282AD0A4F5807405F58075DA
:1026100006F58076B4F5807FE5D2C4B16F4600F050
:1026200096FF4FF480722946384612F025FD224667
:102630003146684612F02AFD2846FFF7D6FE0228EA
:1026400009D069462846FFF738FF022807D040B076
:102650000120BDE8F08140B00A20BDE8F08140B023
:102660000B20BDE8F08100007492010028490A683F
:1026700010600968086100F016B825490A68106002
:102680000968486100F00FB8214909684867704738
:102690001F490968886770471D4801210268116653
:1026A0000068016570471B4A1168096B10F0010F43
:1026B00018BF21F4404110F0020F1CBF21F440511B
:1026C00041F4805110F0040F18BF41F4406110F044
:1026D000080F18BF41F4407110F0100F18BF41F0FF
:1026E000C00110F0200F18BF41F0300110F0400F72
:1026F00018BF41F00C0110F0800F18BF41F003012A
:1027000041F4BE00116840F02040086370470000AB
:102710007C92010084920100FE4801688A68FE49AB
:1027200003680A439A600268D26811430268D16064
:1027300001684969F94A0068114341617047F548E9
:1027400001684969026821F0010141F00D7141F011
:10275000805151610168C968026821F0400141F06F
:102760000D7141F08051D16001688968006821F0E5
:10277000400141F00D7141F080518160704710B50A
:10278000E44C20688168E448226801439160216834
:10279000C96808432168C86020684069DF49084368
:1027A00021684861DE483F210268D160026800214B
:1027B0009163026891640068C0F8B01003210A2098
:1027C00000F007FA0A2000F028FA20684069216822
:1027D00020F0010040F00D7040F08050486120680A
:1027E000C068216820F0400040F00D7040F080503B
:1027F000C86020688068216820F0400040F00D70BB
:1028000040F08050886010BDC54A13681860136896
:1028100059604843116888607047C14A136818605E
:1028200013685960484310F0010F18BF401C11682D
:1028300088607047BA490968C1F8B0007047B84964
:1028400018B109680120886470470968002088640D
:102850007047B3490A6890630868C068096840F027
:102860000200C8607047DFF8B8C210B4DCF800405E
:102870002062DCF800004162DCF800008262DCF8D3
:102880000000C362DCF8001001200863DCF80000DF
:10289000406B10F0010F09D000BF00BF00BF00BFA8
:1028A000DCF80000406B10F0010FF5D110F00200D1
:1028B00018BF4FF0FF3010BC704799480168C968D5
:1028C000006821F00201C160704795480168C9683D
:1028D000006841F00101C1607047914BD3F800C01E
:1028E000CCF82000186841621868826219680120DB
:1028F00008641868406C10F0010F08D000BF00BFDA
:1029000000BF00BF1868406C10F0010FF6D110F046
:10291000060018BF4FF0FF30704781480168C96852
:10292000006821F00101C16070477D480168C968F5
:10293000006841F00401C1607047027C017B02F035
:102940003F0241EA0241764A1368996513680168BB
:10295000596213684168996213688168D962136883
:10296000012119651168496D11F0010F08D000BFF0
:1029700000BF00BF00BF1168496D11F0010FF6D113
:102980001368DB6D83821368DB6D1B0CC3821368D5
:102990001B6E038313681B6E1B0C438313685B6EF3
:1029A00083831268526EC2F30E42C28311F002009A
:1029B00018BF4FF0FF30704759480168C968006878
:1029C00021F00401C160704755480168C96800687A
:1029D00041F00801C1607047DFF844C110B4DCF871
:1029E0000040A267DCF800201062DCF800004362BF
:1029F000DCF800008162DCF8001001200867DCF8D8
:102A00000000406F10F0010F09D000BF00BF00BFF1
:102A100000BFDCF80000406F10F0010FF5D110F09E
:102A2000060018BF4FF0FF3010BC70473C480168EB
:102A3000C968006821F00801C160704701684FEA69
:102A4000314237490B68C3F898200A684068C2F8D9
:102A50009C000868C068096840F02000C8607047A2
:102A60002F4A136818621068416211680120C1F88A
:102A700090001068D0F8940010F0010F09D000BF4A
:102A800000BF00BF00BF1068D0F8940010F0010F25
:102A9000F5D110F0060018BF4FF0FF307047204806
:102AA0000168C968006821F02001C16070471C48B6
:102AB0000168C968006841F01001C1607047A3F166
:102AC000050C174B10B41C68C4F888C0D3F800C0BC
:102AD000CCF82000186842621868816219680120E9
:102AE000C1F880001868D0F8840010F0010F09D0F8
:102AF00000BF00BF00BF00BF1868D0F8840010F00E
:102B0000010FF5D110F0060018BF4FF0FF3010BCD8
:102B1000704700009092010040003412010034120E
:102B20009492010003480168C968006821F010010F
:102B3000C160704794920100234810B502680221D9
:102B40001165026801211166036810225A67036843
:102B500041F206025A66036800229A660268C2F8C9
:102B6000881002689021C2F884100168D1F884109E
:102B7000026841F00101C2F8841002684FF48171CB
:102B8000116600680166032000F047F80021032069
:102B900000F01FF8002010BD10B5032000F048F829
:102BA00009484FF4807102681166026800211166BD
:102BB000026810219167006802214165002010BD64
:102BC00002490020087070478092010038400020C0
:102BD000704700F00303DA004FF0FF0C0CFA02F22A
:102BE0004FF0050C0CEBC303994000F00C030028D8
:102BF00008DA304800681844436911409343194388
:102C0000416170472C4800681844D0F800331140E7
:102C100093431943C0F80013704700F01F010122CD
:102C200002FA01F1244A4009126842F82010704764
:102C300000F01F01012202FA01F11F4A4009126847
:102C400002EB8000C0F88010704700F01F010122E5
:102C500002FA01F1184A4009126802EB8000C0F83C
:102C60008011704714490968086070471249096863
:102C7000C1F88000704710480068006870470E492E
:102C80000968C1F8800170470A4800688068704789
:102C900008490A6892680968886010467047054AC2
:102CA0001268926800F1100352F8230042F82310D2
:102CB00070470000709201006C92010002210C200C
:102CC000FFF787BFC64801688A68C64903680A4398
:102CD0009A600268D26800681143C1607047C048BA
:102CE00001688968026821F4805141F00D7141F05A
:102CF000805191600168C968006821F4805141F0F9
:102D00000D7141F08051C1607047B74982B00868C9
:102D1000006F10F4007F1CBF4FF47A70009014D045
:102D2000421E009230B10868006F10F4007F18BF97
:102D30001046F5D16420009003E00868006F019010
:102D40001046421E00920028F7D10868006F10F468
:102D5000007F03D10A684CF271001066096842F2E4
:102D60004130886602B070479F494FF40D520B689E
:102D70009A660A68126F0B68DA66002808BF01209D
:102D800080B24FF05C5242EA00200A68506609683F
:102D90004FF01140C1F88000B7E7934982B008684E
:102DA000006F10F4007F1CBF4FF47A7301931CD0A6
:102DB0000198421E019220B10868006F10F4007F54
:102DC000F6D10868806E10F0010F0ED00868D0F8B8
:102DD0008400CDE900030198421E019228B10868E1
:102DE000D0F88400009A9042F5D009684FF40D5055
:102DF000886602B070477A480068806810F4805096
:102E000008BF704778480068806E00F00100704786
:102E100075480068406EC0F30F2070477248006824
:102E2000D0F88400704710B50C20FFF70EFF0C207F
:102E3000FFF7F3FE6C4902200968486710BD6A4934
:102E400010B50968032088670C20FFF7F1FEBDE884
:102E500010400C20FFF7F9BE644A11681060084664
:102E60007047614810B50168096F0068C1665F4826
:102E70000068002818BF80475D48016841F4805110
:102E8000016010BD594840687047554810B5016849
:102E90008A68544903680A439A600268D2680068E5
:102EA0001143C160504C0320216888670C20FFF754
:102EB000BFFE0C20FFF7C9FE00F092F94D4B042035
:102EC0001968C1F8880019684FF6FF70C1F88C00C6
:102ED00072B621684FF40D5088662068006F216833
:102EE000C86621684448486621684FF01140C1F81F
:102EF0008000FFF70AFF19684FF40070086662B699
:102F000010BD10B572B6FFF748FF3A484FF40031D4
:102F10000268116662B60068D0F80402304C0028DE
:102F200041D0324B4FF6FF71081A986021688969C9
:102F3000226801F00F01D26902F00F021144091D4D
:102F4000884047F2305181422DD227490968D1F893
:102F50008410C1F101110A04B2FBF0F040F2C91271
:102F60005043C3E90310B0F57A7F38BF4FF47A704D
:102F7000DFF888C0DCF80810002908BFCCF808008A
:102F8000DCF80410CCF80010DCF80820CCE90120B3
:102F900091421FD9814205D9824201D95A6002E08B
:102FA000586000E0596000F02CF9206880682168C2
:102FB00020F4805040F00D7040F080508860206810
:102FC000C068216820F4805040F00D7040F08050BF
:102FD000C86010BD8142E5D88242E1D8DEE700003A
:102FE00090920100001034129C9201003C4000209D
:102FF000304000209892010000FFFF376847002012
:10300000134801688968134A0068114381601248B7
:1030100001684969026841F40071516101680969F8
:10302000026841F00401116101680969006841F01A
:103030001001016170470849096888607047BFF353
:103040004F8F054905480968C860BFF34F8FFEE7F9
:103050009092010004003412709201000400FA05FD
:10306000254801688968254A006811438160244821
:1030700001684969026841F0010151610168096B09
:10308000204A21F440511143026811630168096A22
:10309000036821F00F021C490A431A621B4B8A1E67
:1030A0001B68C3F8C42000680165704714480068B5
:1030B000006900F0700070471148154902681163FB
:1030C0000268144951630168496C026821F40031B7
:1030D00051640168496C40F2FF3211430268516447
:1030E0000168496C006821F48031416470470448EC
:1030F000006840687047000090920100040034129C
:103100008492010000205FA003005FA08C92010068
:10311000C08C5FA095995FA0022824BF0020704753
:10312000B84B53F8202043F820101046704770B574
:10313000B54C2068006FB34D10F0010F06D0216828
:103140000120C8662868002818BF80472068006FE3
:1031500010F0020F08BF70BD02202168C8666868C1
:10316000002808BF70BDBDE870400047A74810B5F3
:1031700001688A68A64903680A439A600268D268AF
:1031800011430268D160A04902220B681A65D1F888
:1031900000C00123CCF86030D1F800C00323CCF884
:1031A0006C3009684A6501688968026821F080010D
:1031B00041F00D7141F0805191600168C96800686B
:1031C00021F0800141F00D7141F08051C160092072
:1031D000FFF723FD0221BDE810400920FFF7F9BCED
:1031E0008A4801688A688A4903680A439A600268C3
:1031F000D26800681143C1608349022009680865EC
:1032000070478149022009684865804801688968DB
:10321000026821F0800141F00D7141F08051916010
:103220000168C968006821F0800141F00D7141F02A
:103230008051C1607047754800688068C0F3C01055
:10324000704771480168096F11F4007F04D000686D
:103250004FF440710166704700684FF48071016659
:10326000704710B5684C2068C06F10F0020F4FF027
:10327000010018BF03202168486700F0F3F8634994
:103280000A689269096802F00F02D040C969226891
:1032900001F00F01C8400521B0FBF1F04FF40571BA
:1032A0000009C2F8801013F0F6FE5A4A5A4B13F088
:1032B00005FF13F0C3FE2168C1F884002068006F89
:1032C00010F4007F04D021684FF44070086610BDF0
:1032D00021684FF48070086610BD4B480168096F83
:1032E00011F4807F04D000684FF44071016670478C
:1032F00000684FF4007101667047434B30B41A68A0
:10330000D26F12F0010F1DBF4FF0030C1A68C2F804
:1033100074C0022204BFD3F800C0CCF874204FF070
:10332000020C00EB4005C5EBC0104FF49674C1EBE6
:10333000C0004C4300EB8000384904EB4010A1FB77
:10334000001032490022C0080C68A469096804F022
:103350000F04C96901F00F012144C8400521B0FBE9
:10336000F1F0B0F5803F05D3511C4008CAB2B0F56A
:10337000803FF9D242EA0C211A6841F01001C2F8EC
:1033800088101968C1F88C001868006F10F4807FED
:1033900005D019684FF44070086630BC7047196852
:1033A0004FF40070086630BC704717480168096F19
:1033B00011F4003F04D000684FF4403101667047BB
:1033C00000684FF48031016670470F480168096F4B
:1033D00011F4803F04D000684FF44031016670471B
:1033E00000684FF400310166704707480068006FBD
:1033F000C0F30020704704480068006FC0F340200D
:103400007047000050400020989201009092010007
:10341000800034127B14AE47E17A843FCDCCCCCC13
:10342000244900200A6890600968086022494860C1
:10343000704710B51F4C21684860216800208860E3
:103440000221401EFFF7C5FB21680720086010BD60
:103450001849002009680860704717480188491C0E
:10346000018070471448806870472DE9F041124C84
:10347000002705462780A0684FF47A71B0FBF1F071
:103480000C4E401E31684860306887600221C81EBB
:10349000FFF79FFB3168072008602188A942FCD311
:1034A00030680760BDE8F0810449484302498860FC
:1034B00070470000689201005840002040420F0011
:1034C000704770B52C4C05464FF40D502168886646
:1034D00021680320C86621682848486621684CF2A4
:1034E0007100086621682648C1F88000216842F210
:1034F0004630886602210020FFF76BFB0020FFF7B3
:103500008CFB002D08BF70BD2068806E42F24131F7
:1035100008432168886670BD174810B5026801210C
:10352000916700684FF40D5181660020FFF780FB22
:10353000BDE810400020FFF788BB0F490120096853
:10354000486770470C4901200968886770470A4935
:103550004CF27100096808667047074881B04CF268
:103560007101026811660168096F0268D16600681E
:10357000006F009001B0704778920100073839372A
:10358000009C1C9170B5FE4E00244FF48061347095
:103590007470FC4811F075FD4FF48061FA4811F029
:1035A00070FDFA4DB460B4702C606C60AC60EC607F
:1035B0002C616C61AC61EC612C626C62AC62EC629F
:1035C0002C636C63AC63EC632C646C64AC64EC647F
:1035D0002C656C65AC65EC652C666C66AC66EC665F
:1035E000F470582105F1700011F04BFD582105F1E0
:1035F000C80011F046FDF4603471C5F87841C5F893
:103600007C41C5F88041C5F88441C5F88841C5F8BA
:103610008C41C5F89041C5F89441C5F89841C5F86A
:103620009C41C5F8A041C5F8A441C5F8A841C5F81A
:10363000AC41C5F8B041C5F8B441C5F8B841C5F8CA
:10364000BC41C5F8C041C5F8C441346170BDCC4827
:103650008078002818BF01207047C94800790028E9
:1036600018BF01207047C648C078002818BF012045
:103670007047C3484078002818BF01207047C048F1
:1036800000697047BE48C06870472DE9F041BC4FE3
:1036900080463878002814BFBD48BE48057814BF5E
:1036A000BD48BE48047805FB04F6FFF735F821460F
:1036B0002846FFF7A9F8B44A4346A2F580610846B8
:1036C000FFF7D1F8FFF73BF872004146AE4811F022
:1036D000DDFC01207870BDE8F081A9488068704762
:1036E0002DE9F04FA64CADF2344D94F801A094F8BA
:1036F000029094F803802779FDF7D8FDCDF82C04CB
:10370000FDF7A5FFCDF82804FDF7D2FD0020FDF759
:1037100084FACDF82404FDF7B8FF0026CDF818642C
:1037200004F03FF9012811D00DF58060FEF728F96B
:10373000002800F06F810DF5806004F0B4FEDDF824
:10374000080410B3B9F1000F05D01EE00120CDF838
:10375000180400F062B90546FEF7DEFF904C012127
:103760002078FFF751F88F4A2B46A2F1380108461E
:10377000FFF779F8FEF7E3FF2078294642008948F1
:1037800011F084FC7E4901208870DDF804040028D3
:1037900070D0BAF1000F6DD1DFF8E4B104469BF8A8
:1037A000000000283DD1DBF8085025B378480078A8
:1037B000CDF8200478480078CDF81C04FEF7ACFF63
:1037C000DDF81C14DDF82004FFF727F821462A460F
:1037D0000846FFF782F8FEF7B2FF73480078022828
:1037E00004BF284604F048FB6F480078092804BF4E
:1037F000204604F041FB6D480078012811D96A4D3C
:103800002878042804BF204604F036FB2146684689
:1038100012F0CAF904462878052804BF684604F067
:103820002BFBCDF81C449BF80000002814BF58481F
:103830005848047814BF58485848057804FB05FBDD
:10384000FEF76AFF29462046FEF7DEFF4E4ADDF806
:103850001C34A2F580610846FFF705F8FEF76FFFFC
:103860004FEA4B024848DDF81C1411F00FFC4449A4
:1038700001204870DDF8100400284ED0B8F1000F88
:103880004BD1DFF8FCB004469BF8000038BBDBF8F6
:103890000C5025B346480178464800780844401C3F
:1038A0004008019002200090FEF736FFDDE900108D
:1038B000FEF7B3FF21462A460846FFF70EF8FEF74B
:1038C0003EFF3D480078022804BF284604F0EAFB8A
:1038D00039480078092804BF204604F0E3FB254658
:1038E00033480178334800780C18FEF715FF601C48
:1038F00040080221FEF788FF304A2B46A2F158010A
:103900000846FEF7B0FFFEF71AFF620029462B4873
:1039100011F0BCFB01208BF80300DDF81404002833
:1039200070D0002F6ED1DFF858B004469BF800002D
:1039300028BBDBF8105015B32148017840780844C3
:10394000401C4008019002200090FEF7E5FEDDE9F2
:103950000010FEF762FF21462A460846FEF7BDFF2B
:10396000FEF7EDFE10480078022804BF284604F058
:103970009BFC0D480078092808BF204622E024E07F
:103980006440002074470020744B002074530020D2
:10399000814000207E400020824000207F400020A7
:1039A00085400020AC530020F940002080400020DA
:1039B0008340002084400020FE4000203C54002032
:1039C0008640002008BF04F06FFC2546F4480178CB
:1039D00040780C18FEF7A0FE601C40080221FEF79C
:1039E00013FFF04A2B46A2F128010846FEF73BFFE1
:1039F000FEF7A5FE62002946EA4811F047FB0120C8
:103A00008BF80400FDF7F2FF761C032E05D2FDF7BC
:103A10003CFE85E600F0B0FE82E6FDF749FCDDF8ED
:103A20002404FDF7FAF8DDF82C0438B1DDF8280499
:103A300010B1FDF72AFE01E0FDF70FFEDDF81804D6
:103A400038B1D94880F801A080F8029080F803804E
:103A50000771DDF818040DF2344DBDE8F08F10B594
:103A60000024FDF7F1FDD04910F0020F0AD04A788A
:103A7000002A08BF012410F0040F03D08A78002A1E
:103A800008BF012410F0010F18BF10F0100F03D071
:103A9000CA78002A08BF012410F0200F03D008794B
:103AA000002808BF01240020002C08BF10BD002002
:103AB0000870BDE8104013E608B50F2100F0FEFEC7
:103AC000012804D1FFF7CBFF009001F068F8B64859
:103AD000417800291CBFC178002906D0017900294E
:103AE0001FBF80780028012008BD002008BD08B550
:103AF0000F2100F0E3FE012804D1FFF7B0FF009092
:103B000001F04DF8A848417800291CBFC178002970
:103B100006D0017900291FBF80780028012008BD48
:103B2000002008BD7047A048002141708170C1701D
:103B3000017170479C480078002814BF9B489C483E
:103B4000017814BF9B489C48007801FB00F09B491A
:103B50004FEA400201F5806011F08EBA2DE9F0477E
:103B6000914F814608983978002914BF8F499049B0
:103B70000D78A0EB030805FB08F603FB05F4FEF740
:103B8000CBFD41462846FEF73FFE8D4809EB440534
:103B900000EB4408A0F5806C0CEB44012B46424638
:103BA0000846FEF760FEFEF7CAFD72002946404651
:103BB00011F06CFA01207870BDE8F0877F487047FB
:103BC0002DE9F047784F044601463878DFF8ECC11C
:103BD000DFF8D881DFF8D891764D774E002815BFF1
:103BE00098F8002099F800202B78337802FB03F036
:103BF0004FEA4002604611F049FA3878DFF8C0C158
:103C00002146002815BF98F8002099F800202B784D
:103C1000337802FB03F0BDE8F0474FEA400260460C
:103C200011F034BA002818BF01205F49487070476E
:103C300010B55D4C002804BFA06010BDDFF884C142
:103C40005A490B785B490A7801465A43520060464C
:103C500011F01CFA5B48A06010BD5B485B4900781E
:103C6000420001F1380011F007BA5848704770B5AA
:103C7000554C0546014622785448520011F006FA88
:103C800022782946BDE870405200514811F0FEB933
:103C9000002818BF01204449887070474D480178BA
:103CA0004D48007808444D49420001F1580011F098
:103CB000E3B94A48704770B5464E474D0446014641
:103CC00032782878454B10444200184611F0DEF94E
:103CD000327828782146BDE87040414B10444200BC
:103CE000184611F0D3B9002818BF01202E49C8701A
:103CF000704710B52C4C002804BFE06010BDDFF801
:103D0000E4C034490B7834490A7801461A44520019
:103D1000604611F0BBF93348E06010BD20480178DF
:103D2000407808443049420001F1280011F0A4B95C
:103D30002D48704770B51A4A0546107851784218D8
:103D4000520014462946284811F0A0F92246294677
:103D5000BDE87040134811F099B9002818BF012040
:103D600011490871704710B50F4C002804BF20613D
:103D700010BD0B490A78497811444A0001461B4896
:103D800011F084F91948206110BD0749002200286C
:103D90004A708A70CA700A7118BF012008709FE4C7
:103DA00086400020145500206440002081400020FF
:103DB0007E400020824000207F4000207447002089
:103DC000744B0020744F0020854000207453002065
:103DD000AC5300208340002084400020E4530020A6
:103DE0003C54002094540020EC5400203C5500200A
:103DF0002DE9F00F0023B0F90050B0F902C01E46C3
:103E0000A5EB0C02984699461C461F46002AB8BFEF
:103E1000ACEB05021FFA82FA00EB410232F902CC48
:103E200032F9045CACEB0502002AB8BFA5EB0C022A
:103E300092B2BAF1080F2DBF082A4FF0000A4A1EAD
:103E40004FF0010A28BF8A1E0FFA82FC5246E24553
:103E500027DC30F912504545C4BFA846D7B25245B9
:103E60001BDD00EB420B3BF902BCABEB0505ED1D86
:103E70000E2D03D85B1CDBB262450ED19E420BD2E5
:103E80001E46624503D10E2D98BF54B201D9541E6F
:103E900064B2A31B4FFA83F90023521C92B29445DB
:103EA000D7DA081F864206DDB945DFBFA7420020EA
:103EB000BDE8F00F70470120BDE8F00F704770B506
:103EC000FF4AFE4906461478097800EB4402104682
:103ED000FFF78EFF054621463046FFF789FF002297
:103EE000F849002D1CBF00280A7008D10878401C32
:103EF000C0B208700A2882BF0A70002070BD01207D
:103F000070BD2DE9F34F93B00DA8139A099002A844
:103F10000790EA48CDF820D04FF0000800780390D1
:103F20000690E7480DF1040E474603780493B2F972
:103F3000006032F9134001203546A446ADF8343014
:103F4000ADF80080ADF80430ADF80880012B2ADD13
:103F500032F91090B145C8BF4E46A94504DA4D4626
:103F6000DDF81C90A9F8000002EB400932F910A01E
:103F700039F902BCABEB0A09B9F1000FB8BFAAEBE3
:103F80000B090FFA89F9C14509DDC846D345D4BFED
:103F90008146A0F10109DDF820A0AAF80090401C9C
:103FA00000B28342D4DCDDF81890581C00B209EB53
:103FB000030B834525DD32F91030A342C8BF1C46F0
:103FC0006345BCBF9C46AEF8000002EB400332F9EB
:103FD000109033F902ACAAEB0903002BB8BFA9EB90
:103FE0000A031BB2BB4208DD1F46CA45D4BF0346C5
:103FF000431EDDF82490A9F80030401C00B2834530
:10400000D9DCB148A4EB0C0C0268012092F81F31F6
:104010009C45C4BFA6EB050C9C4505DD92F81E31FE
:10402000BB42B8BF43451FDB099BB2F91C21B3F962
:1040300000C031F91C309A4216DBBEF900C0534271
:1040400031F91CC09C450FDBDDF820C0BCF90040F5
:1040500031F914C0624507DB079AB2F900C031F9A3
:104060001C209A42A8BF00200B90012840F0EB8052
:10407000BDF93400139C0990BDF900000C90BDF906
:1040800004001190BDF908001090DDE9030B5844BD
:104090000A90401E00B2CDE907B00E46ABF1010018
:1040A000002100B2CDE9051009988A46D14634F9BD
:1040B00010000F900C98D046574634F91000049128
:1040C00003910E90FFF7F5FD05460C9800280BDBD9
:1040D00034F910200E99B2EBA10F01DA059003E03C
:1040E000401E00B20028F3DA0C9858450BDA34F978
:1040F00010200E99B2EBA10F01DA069003E0401CEC
:1041000000B25845F3DB099883450BDC34F91020E5
:104110000F99B2EBA10F01DA079003E0401E00B245
:104120008345F3DDDDE9090181420CDD34F910201E
:104130000F99B2EBA10F01DA089004E0401C0A9934
:1041400000B28842F2DBDDE9071081422DDA06EB8E
:10415000410036F91120B0F90230D01A0028B8BF5A
:10416000981A049A104400B2049005EB410035F906
:104170001120B0F90230D01A0028B8BF981A039A5B
:10418000104400B2039004EB410034F91120B0F95F
:104190000230D01A0028B8BF981A50440FFA80FA9B
:1041A000481C01B208988142D1DBDDE90501884253
:1041B0002ADA06EB400136F91020B1F90230D11AA3
:1041C0000029B8BF991A41440FFA81F805EB400164
:1041D00035F91030B1F90220991A0029B8BFD11A67
:1041E00049440FFA81F904EB400134F91020B1F988
:1041F0000230D11A0029B8BF991A39440FB2401CB5
:10420000069900B28842D4DBDDE90301401AB0EB25
:104210006A0FDCBFA9EB0800B0EB670F10DC07F0FA
:1042200007FD80B9119835F9101027480068B0F9DA
:104230001C01814204DC109935F91110884202DA20
:104240004FF0FF300B901398FFF739FE002806BFA0
:104250004FF0FF300B900B9815B0BDE8F08F2DE9B3
:10426000F04FDFF86490064685B0D9F8000090F86A
:10427000241100291CBFB0F8380100280AD0FDF72E
:104280002AFAD9F8001091F82411B0FBF1F201FBE1
:10429000120018B105B00120BDE8F08F01F0B2FDA9
:1042A0000546FFF7EFF90446D9F80000002DB0F9F4
:1042B00038110491B0F93A7174D007E083400020BE
:1042C000844000207840002078410020FE4800789B
:1042D000102804BF284603F0E5FEFC484FF0000814
:1042E0000378FB480278A4B1002103EB020CBCF177
:1042F000000F84BFD9F80000B0F8289109D934F92B
:10430000020B0028B8BF404248454DDC491C8C4593
:10431000F5D8CDE90082C6460020CDE902235DF83C
:1043200020A002AA06EB4A0352F820B033F9024B50
:104330004FF000080121C146A446BBF1010F0CD982
:1043400033F9022B9442BCBF144689469445C4BF3E
:1043500094468846491C8B45F2D8A4EB0C010AB25E
:1043600004998A421BDB0AEB09010AEB080335F8C2
:10437000111035F81330C91A511A09B20029B4BF07
:104380004B420B46002AB8BF5242934207DA00293B
:10439000B8BF4942B94202DAF04605E002E0401CEB
:1043A0000228BCD34FF00108B8F1000F08BF01F09C
:1043B000BCFD404605B0BDE8F08F2DE9F74F04463F
:1043C000C4484FF0000882B00578C3484FF0060992
:1043D00047460078C2464646C3460090FFF7EEFBCC
:1043E00086460098002200282ED90021002D26D9CB
:1043F00002FB051080B234F910000028B4BF43421C
:104400000346B3EB490F16DD0028DCBF08F10103BA
:104410000FFA83F8B8BF4342C4BF7B1C1FB200DB56
:1044200003469A4507DA0028ACBF034643420FFA19
:1044300083FA16468B46481C81B2A942D8D3501C39
:1044400082B200988242D0D306FB05B0009034F9C6
:104450001020A5F101094FF0000C1FFA89F35FEA63
:104460000B0020D006FB050189B2002A0CDD34F9CF
:1044700011A004EB410131F9021CBAEB01010ED588
:10448000401E1FFA80FC0EE009DA34F911A004EB9B
:10449000410131F9021CAAEB01010029F0DC401EA8
:1044A0000004000CDED1CB4520DA06FB05B080B25B
:1044B000002A0BDD34F9101004EB4000B0F90200C3
:1044C000081A0DD50BF1010083B20FE008DA34F9B8
:1044D000101004EB4000B0F90200081A0028F1DCCB
:1044E0000BF101001FFA80FBCB45DEDB57EA080029
:1044F00004BF05B0BDE8F08F17B9B8F1000F5EDC5E
:10450000009806FB053281B206FB05C080B2039D10
:10451000039B3EF8104035F8100092B23EF911C0EE
:10452000039F33F811103EF8125037F812200CEBAD
:1045300001032618081A891A1BB20844AF18991BE0
:10454000DA1B11440AB2ACEB0401ACEB050400B277
:10455000214409B20028B4BF44420446002AB4BF33
:1045600055421546641B2FD5002AB8BF5242002879
:10457000B4BF44420446121B0028B4BF4442044660
:104580000029B4BF4D420D46641B26D50029B8BF93
:1045900049420028B8BF4042081A82420FDC03F1AA
:1045A0001E000028B8BF4042BCF1000FB8BFCCF1DC
:1045B000000C6045A2BF012005B0BDE8F08F4FF0B0
:1045C000FF3005B0BDE8F08F0028B4BF4442044678
:1045D000002AB8BF5242A21ACEE70028B8BF404214
:1045E0000029B8BF4942401AD7E72DE9F05FDFF84C
:1045F000ECA080460026DAF80000374690F8241137
:1046000000291CBFB0F8300100287CD0FDF763F80A
:10461000DAF8001091F82411B0FBF1F201FB12005E
:10462000002870D101F076FB5FEA00096BD02C48BE
:104630000078102804BF484603F01EFC25484FF0C0
:10464000000C444690F800B02348634690F800E020
:10465000BEF1000F19DD34F9020B0125BBF1010F8A
:1046600010DD34F9022B101A01B20029B8BF4942FB
:1046700008B2604502DD84461E462F466D1C10467A
:104680005D45EEDB5B1C7345E5DBDAF80020B2F834
:104690003001844537DB06FB0B7008EB400338F82C
:1046A000101033F8023CC91A39F8103009EB4000F9
:1046B00009B230F8020C181A081A00B20028B4BF68
:1046C0004342034600290EE0FE40002083400020C4
:1046D000844000207E4000207F4000207841002060
:1046E000F94000200FE0B8BF49428B420BDA0028A6
:1046F000B8BF4042B2F83211884204DA01F015FC2A
:104700000020BDE8F09F0120BDE8F09F10B505F046
:10471000ADF805F024F9002010BD0000FE48007837
:104720007047FD480078022805D005281CBF0020EE
:10473000704704F03FB807F095B9F7490870704723
:1047400010B50446062828BF10BDDFE800F01203AC
:10475000070F120B084600F02FFA0AE0084607F090
:1047600075F906E0084604F019F802E0084606F07C
:1047700015FFE948047010BDE84900200968B1F848
:10478000641011F4807F08BF7047FDF766BDE349F0
:1047900000200968B1F8641011F4807F08BF7047E9
:1047A000FDF770BDDD4900200968B1F8641011F40F
:1047B000007F08BF704710F071BDD849002009681C
:1047C000B1F8641011F4806F08BF704710F0A6BDF7
:1047D000D149487800281CBF401E4870704770B50A
:1047E000CF490868D0F8CC00CB4C10F0030F0BD0A9
:1047F000096840F4BE0040F02040C1F8C80060786D
:10480000002804BF01206070C64800688068C34D5E
:1048100010F0020F296807D1C3480068406910F002
:10482000010F01D0607840B1B1F86410002011F49C
:10483000807F18BFFDF726FD07E0B1F86410002067
:1048400011F4806F18BF10F069FDB849084208BF25
:1048500070BD2968496E090C617070BD10B572B6E3
:10486000FEF75AFEBDE81040FEF7E9BB10B54FF465
:104870002F30FDF7BAFD72B6FEF74EFEBDE81040D0
:10488000FEF7DDBBA44800697047A348C0687047C5
:10489000A14948617047A048406970479E498861B6
:1048A00070479D48806970479C48026802F5B07364
:1048B000118A508A02F5A072FCF75FBF2DE9F04F14
:1048C000DFF8549295B08A46C9F8100004F02BFF27
:1048D000C9F80C0000287CD090F800C089F802C00C
:1048E000417889F80310837804460CF1010089F8B7
:1048F000043000F0FE0089F80500E27889F806200F
:10490000207989F80700607989F8080009F10A051B
:10491000A0792870E0796870207889F809006046ED
:10492000FDF702F899F8081099F80700FDF717F855
:1049300069782878FDF71DF86946204604F010FFD5
:10494000608AD9F8145000281CBF6843050BB4F8DE
:104950001A80D9F81860B8F1000F08BF4FF48058DA
:10496000678C002F08BF4FF4805700201AF0020F09
:1049700018BF11201AF0040F18BF40F00A001AF0F7
:10498000080F18BF40F004001AF0010F18BF40F0E4
:104990002000616A01EA000A0098109004981190C2
:1049A000089812900C9814900198139010A95046F2
:1049B000FCF76DFD1AF0020F66D004F0CEFB5FEA43
:1049C000000B2AD004F0E0FB6843050B5946002099
:1049D00000E015E0FCF74DF9218A00291CBF0020FA
:1049E000FCF795F904F0F0FB7043000B00F5006054
:1049F000010A0820012202FA00F30B4215D112E04D
:104A000046480068B0F8640010F4807F18BFFDF7D6
:104A100039FC002015B0BDE8F08FB4F80CB0BBF144
:104A2000000FD3D1D8E7401EE5D5061FA07B002894
:104A300018BFA0F1010B02D1FCF7E7F98346E07B38
:104A4000002814BF401EFCF70FFA0BEB06010429E7
:104A500003DD711A0E1D042103E00029BCBF761A84
:104A600000210644042E03DD301FC540042604E067
:104A7000002E02DA7042854000260020FCF7DBF9A8
:104A800031460020FCF706FA1AF0010F23D0A18A64
:104A900000291CBF0120FCF7ECF8268B3EB1314603
:104AA0000120FCF734F931461120FCF730F9A67DDE
:104AB0003EB1711E0120FCF7BEF9711E1120FCF7FA
:104AC000BAF9E67D3EB1711E0120FCF7E3F9711ED3
:104AD0001120FCF7DFF91AF0200F30D0A18B00294C
:104AE0001CBF0220FCF7C5F8268C3EB131460220DF
:104AF000FCF70DF931461220FCF709F9A67F3EB10B
:104B0000711E0220FCF797F9711E1220FCF793F931
:104B1000E67FA6B1711E0BE07C40002078410020AA
:104B20008C92010090920100849201000800030021
:104B30000220FCF7AFF9711E1220FCF7ABF9E07A06
:104B400000281CBF0001FCF70EF8029803F03DFF9F
:104B5000039830B12B4699F8032099F8021003F01E
:104B60003FFF3A464146284603F0A4FF0598FFF769
:104B70005FF8069801F04AF81AF0100F05D009986E
:104B8000FFF7B7F80A9801F0D0F80D98FFF7EBF8A7
:104B90000E9801F042F915B00120BDE8F08F10B574
:104BA000FCF71DFD03F019FF02490020C860012039
:104BB00010BD00007C400020FE4948707047FD4851
:104BC00040787047FC4810B4FC4A0168914218D103
:104BD0004168B1F5887F14D80022D0F808C0034698
:104BE0001146B2EB9C0F24BF10BC704753F8214014
:104BF000491C2244B1EB9C0FF8D3002A04BF10BC1F
:104C00007047002010BC7047EB48FDF7EEBBE94948
:104C1000012048707047E7490020087070472DE96F
:104C2000F34FDDB000208A4646904D904C9072B60E
:104C3000FCF70AFD8046FEF7FEFA48B1FEF7D5FB09
:104C40004D90FEF7B2FBFEF7D6FB4C90FEF7BDFB96
:104C5000FCF70EFCFCF72AFB5690FCF7F8FC55908D
:104C6000FCF726FBFEF7C7F85490FEF796F84FF4D2
:104C70009350FEF704F862B60020814630AF47F843
:104C80002090401C0628FAD3CD4E18F0020F4FF0AA
:104C9000010407D0309430684FF4E76100F580409C
:104CA00010F0EFF9C64A44F2387018F0010F12689C
:104CB00002EB000510D04FF4E071284610F0E1F946
:104CC0000120FBF72FFB002818BF32941120FBF7BF
:104CD00029FB002818BF339418F0200F10D04FF490
:104CE000E071284610F0CDF90220FBF71BFB0028ED
:104CF00018BF34941220FBF715FB002818BF359419
:104D0000DFF8C0B2DFF8AC82309868B30020FCF75F
:104D10006FF800909BF800008DF80400AA48007816
:104D2000012894BFA948AA4800788DF80500002002
:104D3000FCF726F9002818BF4FF0FF3003908DF8DC
:104D400006A0B8F80400ADF808000020FBF7FAFF51
:104D5000ADF80A00306800F5804005903068069094
:104D6000306800F50050079031984FF0FF0A48B3C3
:104D70000020FCF73DF808909BF800008DF8240017
:104D80008DF82540CDF82C908DF826A0B8F80400B9
:104D9000ADF828000020FBF7D5FFADF82A009DF8FC
:104DA00005003268C0EBC00102EBC10101F5804192
:104DB0000D919DF80410484302EB40000E9000F561
:104DC00000500F90DFF80C92DFF80CB2329870B3FD
:104DD0000120FCF70DF81090FBF771FD00280CBFC7
:104DE0009BF8000099F800008DF844000120FCF7C2
:104DF0000CF804FA00F08DF845000120FCF7B2F839
:104E0000C04313908DF846A0B8F80600ADF84800EE
:104E10000120FBF797FFADF84A001595306842F284
:104E2000204100F58460169030680844179033984C
:104E300090B31120FBF7DCFF1890FBF740FD002832
:104E40000CBF99F800009BF800008DF86400112059
:104E5000FBF7DBFF04FA00F08DF865001120FCF78A
:104E600081F8C0431B908DF866A0B8F80600ADF835
:104E700068001120FBF766FFADF86A00306844F265
:104E8000A87108441D90306842F2206100F5C460AA
:104E90001E90306808441F90504D349858B302203B
:104EA000FBF7A6FF209028788DF884000220FBF7FE
:104EB000ACFF04FA00F08DF885000220FCF752F8F0
:104EC000C04323908DF886A0B8F80600ADF888009E
:104ED0000220FBF737FFADF88A00306844F618016E
:104EE00008442590306842F6A01100F51A6026901B
:104EF000306808442790359858B31220FBF778FFA4
:104F0000289068788DF8A4001220FBF77EFF04FA41
:104F100000F08DF8A5001220FCF724F8C0432B9078
:104F20008DF8A6A0B8F80600ADF8A8001220FBF78F
:104F300009FFADF8AA00306844F6880108442D90B6
:104F4000306842F6E02100F52E602E90306808446B
:104F50002F900120FCF7B7FF0120FCF727F85990AC
:104F60000020FCF7EAF958900020FCF7DBF9579095
:104F70000020FBF752FE5A90FCF787FB0020489078
:104F8000499037903E904698002840F0C98302F03F
:104F900008FD012800F0C4834998802800F2C083EE
:104FA00040A8FCF7EDFC002800F0B48340A803F013
:104FB0007AFA15E09840002000AF020054435246B0
:104FC000A092010081400020804000207F4000200E
:104FD0008240002083400020844000208640002042
:104FE0004898401C489000F09083002048904998D1
:104FF000401C4990002038AA012142F82010401C92
:105000000628F8D33798002808BF369013D0012817
:1050100004BF0020369000F0E580022804BF002085
:10502000369000F01482032804BF0120469000F05F
:10503000468300F075BB369930A850F8210000284F
:1050400000F0C880369A684600EB42100022479272
:1050500007794279D0F800803F92B0F90860426940
:105060004B923E998269C068C1F104054A90F9B13A
:10507000002D7CDB3F984FF00009002860D905F136
:105080000800012101FA00FBE81D01FA00F0509030
:1050900001234A9803FA09F1084018BF01200021B2
:1050A00051904B98C9EBC9038C4600EBC30A80E0D2
:1050B0003F984FF00009002842D901214A9801FA8F
:1050C00009F3034214BF4FF0010E4FF0000E002011
:1050D0004B99C9EBC903844601EBC30A29E00121BE
:1050E000814011EA080F21D041084E915AF821B0B1
:1050F000C107CC0E2BFA04F132F9023B0CF1010C82
:105100009B1B89B2BEF1000F18BF5B42002BC8BFCA
:1051100041F4805141F400614FF6FF73A3402BEA44
:105120000303A1400B434E994AF82130401C1C2830
:1051300001D2BC45D3D33F9809F101098145BCD3C5
:105140003FE00120884010EA080F2FD048084F9018
:105150005AF82000CB07DC0E4E90E04032F9023BBB
:105160000CF1010C80B29B1BDDF844E100E02CE067
:10517000BEF1000F18BF5B4210F4805F02D0002B1D
:1051800004DA01E0002B01DD20EA0B00002DC4BF92
:10519000509B18434FF6FF7E0EFA04FE4E9BA04034
:1051A00023EA0E0303434F984AF82030491C1C2978
:1051B00001D2BC45C5D33F9809F101098145FFF4EF
:1051C00067AF002D04BF0120479038A9369A479851
:1051D00041F822003698401C36900628FFF42BAF89
:1051E00000F06DBA369930A850F82100002800F080
:1051F0002681369A684600EB421000224E920479CE
:105200004679837905684793B0F9088042694A92E4
:10521000C368826950934089479B3E991840C1F109
:1052200008074F90E9B1002F77DB4FF0000A002EFE
:1052300072D90120B8404B90781E012101FA00F08C
:1052400053900123509803FA0AF1084018BF012037
:1052500000213F904A98CAEBCA038C4600EBC30B6F
:1052600095E04FF0000A002E56D90123509803FA1A
:105270000AF1084018BF012000213F904A98CAEB6C
:10528000CA038C4600EBC30B40E001208840284253
:1052900039D0480851905BF82000CB074FEAD3691A
:1052A0004B9020FA09F032F9023BDDF8FCE00CF1FA
:1052B000010C80B2A3EB0803BEF1000F18BF5B42E4
:1052C00010F4805F09D0002B0EDA10F4706018BF64
:1052D000A0F5807040F4805006E0002B04DD10F44F
:1052E000706018BFA0F5807040F080004FF6FF7E20
:1052F0004B9B0EFA09FE23EA0E0300FA09F0034362
:1053000051984BF82030491C1C2901D2A445BCD32C
:105310000AF1010AB245A8D340E043E001208840E9
:10532000284231D0480852905BF82000CB074FEA62
:10533000D369519020FA09F032F9023BDDF8FCE024
:105340000CF1010C80B2A3EB0803BEF1000F18BFF3
:105350005B4210F4805F02D0002B04DA01E0002BE6
:1053600001DD4B9B9843002FC4BF539B18434FF65E
:10537000FF7E519B0EFA09FE23EA0E0300FA09F0A4
:10538000034352984BF82030491C1C2901D2A445F4
:10539000C4D30AF1010AB245FFF453AF002FC8BFCE
:1053A0004E9848DC4FF0000A002E42D94798C0F5CD
:1053B00080703F90479840F4807B4A990020CAEB68
:1053C000CA03024601EBC3092DE0012181402942B5
:1053D00026D04FEA5008521C59F82870C107CB0E4E
:1053E00027FA03F11FFA81FCDDF8FCE00CF0FF0165
:1053F00001EB5E01DDF83CE101EA0B01714588BF7C
:1054000071462CF0FF0C4CEA01014FF6FF7C0CFAC0
:1054100003FC27EA0C0C99404CEA010149F82810DA
:10542000401C1C2801D2A242CFD30AF1010AB24586
:10543000C3D301204E90369A38A941F822003698FD
:10544000401C36900628FFF4CDAE00F038B93699EE
:1054500030A850F82100002800F02B813E9852908F
:10546000684600EB411000214E910168509101798E
:10547000479141793F918179B0F908904269519201
:10548000D0E906844289C0684F905298C1F5807671
:1054900002EA010710F0010F15D03F984FF0000B02
:1054A00000287DD901214F9801FA0BF2104018BF56
:1054B00001204A905199CBEBCB02002001EBC201B5
:1054C00082464B91E2E00020FBF770FD05464799CC
:1054D0003F984143032000EB410020F00302414686
:1054E00020460FF0D3FD2846FBF760FD3F984FF0B4
:1054F000000B002854D901224F9802FA0BF1084002
:1055000018BF012000214A905198CBEBCB020D46E9
:1055100000EBC20E50E0012000FA01F25098024266
:1055200047D038F9020B6D1CA0EB09034A980028FC
:1055300018BF5B42480853905EF82000CA074FEA44
:10554000D26A4B9020FA0AF082B2C2F3032002F032
:10555000FF0C12F4805F02D0002B05DA01E0002B73
:1055600002DDACEB060401E00CEB0604BC4205DDF9
:105570000F28AEBF3C46401C002406E0002C04DA95
:105580000028C6BF401E3C46002402F4805242EA76
:1055900000204FF6FF72204302FA0AF24B9B00E014
:1055A0007DE023EA020200FA0AF0024353984EF823
:1055B0002020491C1C2902D247988542ABD33F9832
:1055C0000BF1010B834596D369E0012101FA00F24A
:1055D00050990A4257D034F9021B4A9A0AF1010A3B
:1055E000A1EB0901002A18BF494238F9022BA2EBAE
:1055F000090218BF52420029B4BF4B420B46002A91
:10560000B8BF52429A423ED94B9B4208539253F83C
:105610002220C3074FEAD36E5B9222FA0EF293B2B6
:10562000C3F3032203F0FF0C13F4805F02D00029C0
:1056300005DA01E0002902DD0CEB060501E0ACEB28
:105640000605BD4205DD0F2AAEBF3D46521C0025B2
:1056500006E0002D04DA002AC6BF521E3D46002592
:1056600003F4805141EA022129434FF6FF735B9A0C
:1056700003FA0EF39A4301FA0EF142EA01034B9A40
:10568000539942F82130401C1C2802D247998A4580
:105690009BD33F980BF1010B8345FFF403AF529866
:1056A000032826BF01204E904E9838A9369A41F81B
:1056B00022003698401C36900628FFF4C8AE01231D
:1056C000002038A951F8202022B1401C0628F9D327
:1056D000012B02D03E98401C16E037981F2812D2AA
:1056E000401C01463790012000FA01F25D990A4200
:1056F00009D13799491C3791032904D800FA01F2DE
:105700005D990A42F5D000203E90469840B9FBF7DB
:10571000BCFF3CE4FFF73BF8469800283FF437AC69
:10572000FBF7C6FD0020FCF7CEFB5998FBF73EFCCB
:105730005898FBF702FE5798FBF7F4FD5A98FBF7D1
:105740006CFA569830B1559810B1FBF79EFF01E006
:10575000FBF783FFFDF76FFD48B14D98002818BF98
:10576000FDF76FFD4C98002818BFFDF7B6FD549863
:10577000002818BFFDF7C9FA469800280CBF012081
:1057800000205FB0BDE8F08F2DE9F04FADF2047D51
:105790004FF0000807464646CDF8008700F04FB9A5
:1057A000304603F0C0FF002800F04881008900EA7D
:1057B000070424F0CC0030F47C4000F03F810F213E
:1057C0003046FFF77BF8002800F03881FBF73CFFFC
:1057D0000546DDF80007002840F02E8105F00E0098
:1057E000FBF742FE03210020FBF765FBDDF8000715
:1057F000002840F0218114F0010F20D0FF210F205C
:10580000FFF70DFACDF80007FBF752FDDDF80007B2
:10581000002840F01181FFF738F88146EA464FF042
:10582000040B5046FCF7E6F899F92C1052465846FE
:1058300003F0B8FFDDF80007002840F0FD8014F009
:10584000060F35D00120FEF7A0FACDF80007FBF7D0
:105850002FFDDDF80007002840F0EE8014F0020F65
:1058600011D0FEF7ABF98146FFF70FF805235FEA89
:10587000090204D090F92D10184603F093FFDDF8CB
:10588000000700287DD114F0040F11D0FEF796F91F
:105890008146FEF7FAFF06235FEA090204D090F979
:1058A0002E10184603F07EFFDDF80007002868D1AF
:1058B00005F01100FBF7D8FDDDF80007002860D1E6
:1058C00014F0100F1FD0FF210F20FFF7A8F9CDF81B
:1058D0000007FBF7EDFCDDF80007002851D1FEF7CB
:1058E000D4FF8346E9464FF0080A49460120FCF7F9
:1058F000C4F89BF930104A46504603F053FFDDF8D8
:10590000000700283DD114F0600F39D00120FEF7C8
:105910003CFACDF80007FBF7CBFCDDF800070028C8
:105920002FD114F0200F14D015F0100018BFFEF77F
:10593000C0F98146FEF7A9FF09235FEA090204D0F6
:1059400090F93110184603F02DFFDDF8000700280C
:1059500072D114F0400F13D015F0100018BFFEF7ED
:10596000A8F98146FEF791FF0A235FEA090204D0F5
:1059700090F93210184603F015FFDDF8000700B962
:1059800000E045E005F02000FBF76EFDDDF80007C4
:10599000F0BB14F4807F1DD0FF210F20FFF73FF9EB
:1059A000CDF80007FBF784FCDDF8000780BBFEF7AD
:1059B0006CFF81466D464FF00C0A29460220FCF729
:1059C0005CF899F934102A46504603F0EBFEDDF8F6
:1059D0000007E8B914F4107F2ED00120FEF7D5F9A6
:1059E000CDF80007FBF764FCDDF8000780B914F47C
:1059F000007F11D0FEF79CF90546FEF746FF0D2308
:105A00002A0004D090F93510184603F0CBFE00E0D0
:105A100012E0DDF8000778B914F0400F0CD0FEF763
:105A200087F90446FEF731FF0E23220004D090F9D7
:105A30003610184603F0B6FEFFF7B1F8761C03F0F7
:105A40006EFEB04204D9DDF8000700283FF4A8AE8E
:105A5000FE4880F80080DDF8000700280CBF012018
:105A600000200DF2047DBDE8F08F2DE9F04FF748DE
:105A7000CDB04578FEF752FE01287DD1F44800688C
:105A8000B0F93610B0F9340003F0E4F915F0020F64
:105A900073D040ACFFF796F80026DFF8B8833027C4
:105AA0004FF488794FF0FF3A90B190E80E10A4E8D7
:105AB0000E1000F1100191E80E1084E80E10D0E9EC
:105AC0000812D0E90A30CDE94A30CDE9481215E094
:105AD000FF22302120460FF0DEFA5020CDF8008161
:105AE000CDE943604596CDF82CA1CDF828A1CDF89D
:105AF00024A14696CDE9476ACDE94197DFF858B32E
:105B00005846FCF772FC4598401C459040F277706F
:105B1000FFF73AFE012814D047980022401C479016
:105B20001F21022005F079FC40AC03F0DFFD90B1AD
:105B300081694891C169499141694A91C0684B9016
:105B400011E015F0080F14BFA220A1204490469840
:105B5000401C4690E8E7CDF82CA1CDF828A1CDF85F
:105B600024A1CDF820A1CDE942760021CDE94089DC
:105B700022460846A36801E034E01FE052F820C046
:105B8000401C6144B0EB930FF5D34E42FF22511CF1
:105B90006846E6600FF07FFAD4E90001A2688DE85C
:105BA000470004F1100004AE0FC80FC620340FCC1C
:105BB0000FC658466946FCF780FC0CE015F0010F53
:105BC00009D040F22220FFF7DFFD20B901221F217A
:105BD000022005F022FCFDF7A6FF01212A46084617
:105BE00005F01BFC4DB0BDE8F04F01F0D6BE974963
:105BF000888070479549C880704700B5FEF7E2FF7E
:105C0000002000BD00207047002070472DE9F04FB4
:105C10008E4EADF20C4D0028B06004BF0DF20C4D5D
:105C2000BDE8F08F317811F0020F6BD18B49DFF8AE
:105C300034820C788A490D78C6F80C800090FDF704
:105C40004CFDCDF80404884890F800908748077808
:105C5000874890F800A0BAF1010F8CBF0DF1040B3A
:105C6000C346DDF804040099002809FB07F04FEA59
:105C700040024BD001A80FF009FA4B4601AA009749
:105C80005846DDF8041411F0A7F9BAF1010F0FD945
:105C9000594640460FF088FF404509D06F4A0146FB
:105CA000404613786E4A12785A4352000FF0EEF9CC
:105CB0000027F068B846002D18D930F9021B0122E0
:105CC000012C0FD930F902CBACEB010109B200294C
:105CD000B8BF49420BB2BB42C8BF1F466146521C07
:105CE000A242EFD308F10108A845E6D3584800685E
:105CF000B0F82C01B842C4BF0020F060307840F00A
:105D0000020030700DF20C4DBDE8F08F58460FF0D8
:105D1000BDF9BAE74D48816829B1017811F0020F49
:105D20001CBFC0687047002070472DE9F84F474EF0
:105D30000028306108BFBDE8F88F317811F0100FEE
:105D400018BFBDE8F88F4B4D82464B484FF0000915
:105D500004784A480778FBF777FC10F0100F02D060
:105D6000FDF790FC814604EB07084FEA48025146D4
:105D700028460FF08BF9B9F1000F09D002200090EE
:105D800008F1010043082A464946104611F024F95B
:105D90000020B5F90030A91C0122012F0FD931F9DB
:105DA00002CBACEB03031BB2002BB8BF5B421BB2B0
:105DB0008342C8BF18466346521CBA42EFD331F93A
:105DC000023B0122012C0FD931F902CBACEB0303CA
:105DD0001BB2002BB8BF5B421BB28342C8BF184640
:105DE0006346521CA242EFD319490968B1F82E113B
:105DF0008142C8BF00257561307840F010003070D6
:105E0000BDE8F88F1148016929B1017811F0100F30
:105E10001CBF40697047002070472DE9F0410B4ED0
:105E200084B00028B06104BF04B0BDE8F0813178CF
:105E300011F0200F1CBF04B0BDE8F081104D80466A
:105E4000104800270178029140781DE0984000201A
:105E5000784100205443524600AF02007E400020AB
:105E60007F400020645500208140002082400020B7
:105E7000804000206459002083400020844000209E
:105E8000BC590020864000200390FBF7DDFB10F09A
:105E9000200F02D0FDF7F3FB0746DDE902014418AD
:105EA0006200414628460FF0F1F847B10220009009
:105EB000601C43082A463946104611F08DF800222E
:105EC0002C4617460DF10808039B34F9021B0120EC
:105ED000012B11D934F902CBACEB010109B2002935
:105EE000B8BF49420BB29342C8BF1A466146401C34
:105EF00058F820308342EDD87F1C022FE4D3082AC3
:105F0000B8BF0025F561307840F02000307004B053
:105F1000BDE8F0810E48816929B1017811F0200FA8
:105F20001CBFC0697047002070470A4808490068D4
:105F300090F825218878401CC0B28870824228BF22
:105F400070470020887001210846FEF7F9BB000069
:105F5000984000207841002070470020704708B525
:105F600003F00700012806D18DF8000002466946BB
:105F70000A2001F0F2FC002008BD08B503F007007C
:105F8000012807D100208DF80000012269460A206F
:105F900001F0E3FC002008BD10B503F00700012864
:105FA00008BFFEF75BFC002010BD08B503F007003A
:105FB000012807D103208DF8000001226946002046
:105FC00001F0CBFC002008BD08B503F00700012854
:105FD00007D10B208DF8000001226946002001F056
:105FE000BCFC002008BD08B503F00700012806D15D
:105FF0008DF8000002466946002001F0AEFC00204A
:1060000008BD1FB513F0070F08D19DF80800F02850
:1060100007D0012202A9062001F09FFC04B0002055
:1060200010BDFEF7F1FDF9E71FB513F0070F04D11E
:10603000012202A9104601F090FC04B0002010BD1E
:106040002DE9F843804603F007000026FE4D089C2A
:106050000F46012802D0022806D002E00520A870D1
:106060002E810020BDE8F883A87805281BD1288957
:10607000A04210D2FDF73BF8AC218DF80010010AC8
:106080008DF801108DF8020028891DF8001088F89D
:106090000010401C288180B2A04204D12E81012032
:1060A00038700320A8700120BDE8F88370B503F0B4
:1060B00007020026E54CE44DDDF810C0012A02D0AD
:1060C000022A46D043E0FDF712F80521A9702268A4
:1060D000AC2111702268010A517021688870DC4877
:1060E00022680168897CD17000682268017C117186
:1060F000017E11F0040F0ED0C18A2268090A517185
:106100002268817D9171818A2268090AD171226891
:10611000017D11720DE0818A2268090A517122689D
:10612000017D9171C18A2268090AD1712268817D3D
:106130001172226820215172226802219172216815
:10614000CE7221680E732168007E48732E81002074
:1061500070BDAA78052A0FD12A89624504D2236826
:106160009B5C0370501C28812889604504D12E81D6
:10617000012008700320A870012070BD30B403F026
:106180000704B24BB04D029A4FF0000C012C02D024
:10619000022C3AD036E00220A8704FF42F30A5F838
:1061A00008C00168880A444211EB842418BF401CCF
:1061B000404201EB8000C01C20F0030041F6E87172
:1061C0000144B0F5283F14D8CC78086864F31F6008
:1061D000A04CA0420DD10020002A13D901EB000CE5
:1061E0001C689CF804C004F800C0401C8242F5D82A
:1061F00008E00020002A05D9196801F800C0401CF9
:106200008242F9D830BC00207047AC78022C10D103
:106210002C89944204D21B681B5D0370601C28818A
:106220002889904205D1A5F808C0012008700320F4
:10623000A87030BC0120704730B403F00704834BD2
:10624000814D029A4FF0000C012C02D0022C51D04B
:106250004DE00220A8704FF42F30A5F808C0016867
:10626000880A444211EB842418BF401C404201EBD1
:106270008000C01C20F0030141F6E8700844B1F52D
:10628000283F2BD8C478016864F31F61714CA14288
:1062900024D11A68017C11701A68417C51701A6807
:1062A000817C91701A68C17CD1701A68017A117171
:1062B0001968427A4A711A68817A91711A68C17AAA
:1062C000D1711A68017D11721A68417D51721A6884
:1062D000817D91721968C07DC87208E00020002A93
:1062E00005D9196801F800C0401C8242F9D830BCB9
:1062F00000207047AC78022C10D12C89944204D233
:106300001B681B5D0370601C28812889904205D1A1
:10631000A5F808C0012008700320A87030BC012037
:1063200070472DE9F04103F007020026474D464F24
:10633000069C012A02D0022A3AD036E003F0D6F9B0
:1063400040B3D0E906212B68C0681A70D5F800C0A8
:10635000130A8CF80130D5F800C0130C120E8CF81B
:1063600002302B68DA702A6811712B680A0A5A7198
:106370002B680A0C090E9A712A68D1712968087273
:106380002A68010A51722A68010C9172010E28686C
:10639000C17207E00020002C04D929680E54401C6B
:1063A0008442FAD80220B8703E810020BDE8F08116
:1063B000BA78022A0FD13A89A24204D22B689B5C98
:1063C0000370501C38813889A04204D13E810120DD
:1063D00008700320B8700120BDE8F08170B403F0AC
:1063E00007031A4C184D039A4FF0000C012B02D0F2
:1063F000022B5BD057E00220A8704FF42F30A5F895
:1064000008C001680026880A434211EB832318BFA5
:10641000401C404201EB8000C01C20F0030101F54C
:106420000050B1F5283F98BF10F0030F32D10A4B4E
:106430000168994204BF002319462BD150F821501E
:10644000491C2B44072909E0C0400020A492010008
:106450007841002034CD12AB54464953EED303B1FA
:10646000C6B12268017C11702268417C517021689C
:10647000827C8A702268C17CD1702268017D117192
:106480002268417D51712268817D91712168C07DB2
:10649000C87108E00020002A05D9216801F800C071
:1064A000401C8242F9D870BC00207047AB78022BA8
:1064B00010D12B89934204D22468E45C0470581CE8
:1064C00028812889904205D1A5F808C001200870CC
:1064D0000320A87070BC012070472DE9F04103F043
:1064E00007040027F74EDDF818C0012C05D013F083
:1064F000070F06D0022C43D03FE00220B070378156
:106500003BE00125002412F0010F1FD04FF42F3083
:106510000168880A434211EB832318BF401C4042A4
:1065200001EB8000C01C20F00303B3F5283F23D803
:1065300000204FF40051B0EB930F07D251F804CB79
:10654000401C6444B0EB930FF8D3ADB112F0020FCE
:106550000ED003F0CBF878B182680021B1EB920F36
:1065600006D250F8043B491C1C44B1EB920FF8D3FF
:10657000002D18BF346200D137620020BDE8F081E1
:10658000B278022A13D13289624508D2C2F10303DC
:10659000346ADB0024FA03F30370501C3081308925
:1065A000604504D13781012008700320B0700120BC
:1065B000BDE8F08130B403F007030024DFF804C322
:1065C000029A012B02D0022B0BD007E005208CF899
:1065D0000200ACF8084020208CF8030030BC0020FA
:1065E00070479CF80230052B14D1BCF80830934258
:1065F00005D29CF803500570581CACF80800BCF894
:106600000800904206D1ACF8084001200870032031
:106610008CF8020030BC012070472DE9F04383B0B4
:1066200003F00705A84EA74FDDF828C04FF000087B
:10663000012D0AD013F0070F3B461B8903F101041B
:10664000A4B211D0022D22D01DE001A9684601F0AC
:1066500042FB0520B87031680198087031680098D5
:106660004870A7F808800EE0634502D23068C25433
:106670003C813889604506D1A7F8088030680178E8
:10668000407801F01FFB03B00020BDE8F083BA782A
:10669000052A0ED1634503D23268D25C02703C8178
:1066A0003889604505D1A7F80880012008700320CB
:1066B000B87003B00120BDE8F08370B503F00700A7
:1066C0000026804C804DDDF810C0012803D013F067
:1066D000070F06D024E026812868067028684670D7
:1066E0001EE02089604503D22B681A54401C20818B
:1066F00080B2604514D175A00122006826810A701D
:106700002968C2B2097891420AD12968C0F30720EA
:106710004978814204D100221146032001F01DF97D
:10672000002070BD10B503F00700012808BF01F07C
:1067300097FF002010BD70B503F00704614D012CD8
:1067400009D013F0070F2B46D3F820C01B8908D0BF
:10675000022C17D014E00020288104F058FE286293
:106760000EE0002B04BF1002286206D0012B04D1DA
:106770004CEA0200286204F043FE2889401C28816C
:10678000002070BD002B04BF4FEA1C21017005D012
:10679000012B03D180F800C001200870581C28810B
:1067A000012070BD70B5064603F00700454C0D464C
:1067B000012808BF00200DD013F0070F02D00228D7
:1067C0000BD008E02089002804BF10460CF0D7FC4D
:1067D0002089401C2081002070BD0CF0CDFC307061
:1067E0000120287070BD2DE9F00103F00704354E3B
:1067F000012C0CD013F0070F364BB446344F9CF8E5
:106800000350D3F800C006D0022C30D02BE000207B
:106810003081708127E03189002908BFF27020D0D3
:10682000012904BF100230621BD0022919D1306A3D
:106830001043306280B2062D13D2DFE805F0030565
:10684000070A0D10F8810CE0B8810AE0ACF83400BA
:1068500007E0ACF80C0104E0ACF8500001E0ACF843
:106860005200481C3081BDE8F00100207047748957
:10687000022C20D20022062D13D2DFE805F00305FA
:10688000070A0D10FA890CE0BA890AE0BCF8342036
:1068900007E0BCF80C2104E0BCF8502001E0BCF893
:1068A0005220002C04BF110A017004D0012C02D127
:1068B000027001200870601C7081BDE8F0010120A9
:1068C00070470000C0400020A492010055AC0000B9
:1068D000747F002078410020DFF820C410B59CF8B8
:1068E0006CC013F0070F4FEADC0C04D003F0070272
:1068F000022A08D005E0002A14BF6046002006F0F6
:106900003EFC002010BD80F800C00120087010BDC2
:106910000020704770B503F007020026F84CF94DCF
:10692000DDF810C0012A02D0022A15D012E005F0CD
:10693000C6F821680870FDF7F1FE2168487002F082
:1069400009FC21688870FDF7ECFE2168C8700520FD
:10695000A8702E81002070BDAA78052A0FD12A893F
:10696000624504D223689B5C0370501C28812889EF
:10697000604504D12E81012008700320A8700120F9
:1069800070BD70B5064603F007000D4602281CBF17
:10699000002070BD00F0FBFF002814BF012400247C
:1069A00000F0F8FF002814BF0222002222433270B8
:1069B0000120287070BD70B503F00702D04C00258F
:1069C000D04EDDF810C0012A02D0022A42D03FE0AA
:1069D000FEF7F8F8002828D04169FF292CBFFF21D5
:1069E000C9B2226811708169FF2934BFC9B2FF2181
:1069F00022685170C169FF2934BFC9B2FF212268E2
:106A000091702268017CD170226890F82010117179
:106A1000018C0A0A21684A71016A2268090C917185
:106A2000006A2168000EC87111E0206805702068B6
:106A300045702068857021685020C8702168FF204B
:106A4000087121684871216888712168C871358191
:106A5000002070BD3289624504D223689B5C0370BC
:106A6000501C30813089604502D135810120087089
:106A7000012070BD70B503F007020025A04BA14CAA
:106A8000DDF810C0012A02D0022A08D005E01868FB
:106A90000EF0ACFD0520A0702581002070BDA2780D
:106AA000052A0FD12289624504D21B689B5C0370C2
:106AB000501C20812089604504D125810120087067
:106AC0000320A070012070BD70B503F007020025FF
:106AD0008C4C012A02D0022A11D00EE00520A070B1
:106AE00000212581084601F0F6F84FF6FF7101EA12
:106AF0004000A08101F0FBF86061002070BDA27829
:106B0000052A16D12289B4F80CC0624507D212F0CA
:106B1000010F1CBFE37803700DD0501C2081208929
:106B2000604506D12581012008700320A07001F086
:106B3000ECF8012070BD666922F00103F35A1E0AC9
:106B40000670E370E9E770B503F0070200256D4CAD
:106B5000012A02D0022A0AD007E00520A070258170
:106B6000D020A08101F054FA6061002070BDA278AD
:106B7000052A16D12289B4F80CC0624507D212F05A
:106B8000010F1CBFE37803700DD0501C20812089B9
:106B9000604506D12581012008700320A07001F016
:106BA00045FA012070BD666922F00103F35A1E0AFE
:106BB0000670E370E9E77FB50D46044613F0070F52
:106BC00004D003F00700022808D004E0012202A943
:106BD000092000F0C2FE04B0002070BD04F06FFF79
:106BE00020700120287004B070BD10B503F00702BA
:106BF000444C012A02D0022A0DD00AE002F0FBFE2A
:106C00000021606200281ABF4FF40660E081E18134
:106C10002181002010BD2289E3899A4207D2D4F84D
:106C200024C01CF802C080F800C0501C20812089BC
:106C3000984204BF01200870012010BD10B4DFF895
:106C4000C8C013F0070F04D003F00702022A2ED0A9
:106C50002AE0012A01D09AB126E0DCF80000406960
:106C6000DCF8001040F001004861DCF80000006B27
:106C7000264920F440500843DCF80010086313E074
:106C8000DCF80000006BDCF8001020F4405040F409
:106C9000BE0040F020400863DCF800004069DCF8EA
:106CA000001020F00100486110BC00207047DCF8A3
:106CB0000020526902F0010202700120087010BC2D
:106CC000704770B50D46044613F0070F04D003F06B
:106CD0000700022808D005E0002A14BF0120002088
:106CE00001F0B0FC002070BD01F0B3FC002814BF1F
:106CF0000122002222700120287070BD747F0020C4
:106D0000A4920100C04000208492010000205FA0F6
:106D100070B503F00700FA4D1446012808BF0020A3
:106D200017D013F0070F15D12889002808BFEA7083
:106D30000DD001280BD1E878FBF798FCF149E878F1
:106D40000B6800EA04021A630968A04348632889B3
:106D5000401C2881002070BD10B503F00702E84CEC
:106D6000012A02D0022A27D024E002F044FE0023A8
:106D7000002804BF6362E3811BD000F1500161620F
:106D80004168B1F5887F90F820100CD390F821204D
:106D900001EB020C01FB02C190F8222090F82300C5
:106DA0001044084404E090F822000A1801FB002077
:106DB000E0812381002010BD2289E3899A4207D215
:106DC000D4F824C01CF802C080F800C0501C2081F8
:106DD0002089984204BF01200870012010BD10B521
:106DE00013F0070F04D003F00702022A05D002E0D7
:106DF000104600F097FF002010BDC34A12780270C1
:106E00000120087010BD10B513F0070F04D003F077
:106E10000702022A05D002E0104601F029F90020FD
:106E200010BDBA4A127802700120087010BD1FB55B
:106E300013F0070F04D1012202A9082000F08DFDF4
:106E400004B0002010BD70B503F00700AC49012864
:106E500004BF0020088125D013F0070F22D1088934
:106E6000AB4E03283CBF33681A54401C80B20881E3
:106E7000032817D1FAF7FCFA3068B0F8010045BAD8
:106E8000FAF714FA040018BFFAF719FC3068007812
:106E9000002818BF01202946F9F7EBFE002C18BF87
:106EA000FAF710FC002070BD70B503F0070094499C
:106EB000012804BF0020088129D013F0070F26D134
:106EC0000889934D02283CBF2B681A54401C80B29D
:106ED000088102281BD1FAF7CBFAFAF7E7F9040088
:106EE00018BFFAF7ECFB286800780028286841787A
:106EF00008BF002005D00120F9F709FF2868417874
:106F00001120F9F704FF002C18BFFAF7DBFB002073
:106F100070BD7FB50D46044613F0070F04D003F093
:106F20000700022808D004E0012202A90D2000F089
:106F300014FD04B0002070BD04F083FD002814BFD0
:106F40000122002222700120287004B070BD7FB59C
:106F50000D46044613F0070F04D003F00700022883
:106F600008D004E0012202A90E2000F0F6FC04B0D3
:106F7000002070BD04F056FD20700120287004B080
:106F800070BD10B503F00700DFF874C10299012845
:106F900004BF0020ACF8080019D013F0070F16D179
:106FA000BCF808005A4B03283CBF1C682254401C04
:106FB00080B2ACF80800884209D118681968B0F8A6
:106FC0000100097840BA00B219B1FEF713FE0020A3
:106FD00010BDFEF70CFEFAE710B503F00700DFF86E
:106FE00020C10299012804BF0020ACF8080017D086
:106FF00013F0070F14D1BCF80800454B03283CBF21
:107000001C682254401C80B2ACF80800884207D1AA
:107010001868B0F8010041BA18680078FAF7A1FEC4
:10702000002010BD70B503F00702354CDDF810C02C
:10703000012A02D0022A07D004E000202081FBF7B9
:1070400021FF2062002070BD2289624506D2C2F174
:107050000303256ADB0025FA03F30370501C80B29A
:107060002081604504BF01200870012070BD7FB5FC
:107070000D46044613F0070F04D003F00700022862
:107080000DD009E09DF8080010F0010F04D0012296
:1070900002A90F2000F061FC04B0002070BD04F0D4
:1070A00067FD20700120287004B070BD7FB50C46CC
:1070B000054613F0070F04D003F00700022808D09C
:1070C00004E0012202A9052000F047FC04B00020E2
:1070D00070BDFDF723FB022808BF00200BD003285A
:1070E00008BF022007D0042808BF032003D00528CA
:1070F00014BFFF20012028700120207004B070BD53
:10710000C04000207C920100F9400020FE40002099
:10711000A492010010B5104613F0070F08BF04F049
:10712000B0FC002010BD10B5104613F0070F08BFCB
:1071300004F0B3FC002010BD70B5044603F0070056
:107140000D4602281CBF002070BD04F0B3FC207067
:107150000120287070BD70B403F007020024FC4BBE
:10716000DDF80CC0012A05D0022A04BF9A78022A51
:107170000AD01BE002209870F6481C816FF07F4116
:107180000068081A186211E01A89624506D21E6A60
:10719000D50026FA05F50570501C18811889604540
:1071A00004D11C81012008700320987070BC01205C
:1071B000704713F0070F04BFE748027000207047C4
:1071C00010B5944603F00700E149029A012804BF74
:1071D0000020088112D013F0070F0FD10889DF4B70
:1071E00090423CBF1C6804F800C0401C80B208817B
:1071F000904203D10C20196800F0AFFB002010BDB5
:107200002DE9F04103F007050026D14C9446012DED
:1072100004BF2681668122D013F0070FCC4B9A89D8
:107220005B6A02D0022D26D019E02089002808BF11
:10723000C4F824C010D0012814D0801EC749904241
:107240003CBF0D6805F800C0401C904204D109689D
:1072500003F52A30FBF797F92089401C2081002094
:10726000BDE8F0810CF10100A0811844B0F5807FE9
:1072700088BFA681F0E74FF0FF0C80F800C08AB10C
:10728000658903EB050C6B1CBCF5807F09D20CF5FE
:107290002A3C9CF800C080F800C0934204BF012043
:1072A000087063810120BDE8F08110B5944603F0B9
:1072B0000700A749029A012804BF0020088112D0C4
:1072C00013F0070F0FD10889A44B90423CBF1C68F4
:1072D00004F800C0401C80B20881904203D1022013
:1072E000196800F03AFB002010BD70B50D46044649
:1072F00013F0070F04D003F00700022805D002E0C6
:10730000104604F063FB002070BD04F062FB2070A7
:107310000120287070BD1FB513F0070F04D10122A2
:1073200002A9102000F019FB04B0002010BD03F0EA
:107330000701DFF81CC20098012907D013F0070FDE
:1073400004BF9CF80210012909D01FE001208CF82D
:1073500002000020ACF80800CCF81C0014E0BCF8D7
:107360000810814208D2DCF81C30491C42EA032292
:10737000CCF81C20ACF8081089B2814206D1032059
:107380008CF80200DCF81C00CCF8240000207047C8
:1073900003F00701DFF8B8C10098012907D013F006
:1073A000070F04BF9CF80210022909D01FE0022039
:1073B0008CF802000020ACF80800CCF8200016E0A1
:1073C000BCF80810814208D2DCF82030491C42EA9F
:1073D0000322CCF82020ACF8081089B2814206D1F3
:1073E000BCF82000ACF80E0003208CF8020000204E
:1073F000704770B403F007020025554C012A02D0F3
:10740000022A06D002E00220A070258170BC002074
:107410007047A278022A1CD12289B4F80EC06245B6
:107420000FD212F0030F04D1636A53F8046BC4E95E
:10743000086394F820300370206A000A2062501C10
:1074400020812089604504D1258101200870032016
:10745000A07070BC0120704770B503F007000025D4
:107460003B4C0E46012806D013F0070F04BFA0784E
:10747000022805D02BE00220A0702581256226E09D
:107480002089E189884219D2216A090A41EA026207
:10749000401C2262208110F0030F0FD1606AB0F50A
:1074A000303F28BF026006D2B0F5005F03D304224C
:1074B0002B49FBF768F8606A001D60622089E1894A
:1074C000884204D12581012030700320A070002063
:1074D00070BD30B403F007040025DFF874C0012C40
:1074E00008BFACF8085045D013F0070F02D0022CAB
:1074F00043D03FE0042A08BF4FF42C3038D013DCCF
:10750000002A08BF4FF4005032D0012A08BF4FF4C0
:107510002F302DD0022A08BF4FF4103028D0032A74
:1075200008BF104824D010E0052A08BF4FF42A30C5
:107530001ED00D48102A00681AD0112A08BF0B4827
:1075400016D0202A08BFB43012D0CCF81C5011E05D
:10755000C04000205C40002005400020A4920100B3
:10756000E040002000AF020078410020747F00203E
:10757000CCF81C0030BC00207047BCF80820042A5E
:1075800007D2C2F10303DCF81C40DB0024FA03F34A
:107590000370501C80B2ACF80800042824BF0120FE
:1075A0000870012030BC704710B503F007000128B7
:1075B00004D1002211460B2000F0CFF9002010BDAD
:1075C0002DE9F04103F0070CD94E069D0F46044605
:1075D000BCF1010F04BF0020308117D0D44913F053
:1075E000070F0B8903D0BCF1020F12D00EE0D14976
:1075F000022B3CBF0868C254581C80B23081A8429C
:1076000004D102220968042000F0A7F90020BDE897
:10761000F08113B1012B04D008E0FDF77FF8207052
:1076200004E0FDF77EF82070012038703089401C9E
:1076300030810120BDE8F08170B503F00700BC4D3A
:10764000012803D013F0070F05D024E00020E861E3
:107650002862E8701EE0B6492C8991F803C0C86919
:107660000CEB0201CBB2022C03D242EA0020E8610B
:1076700006E0AF49042C096A04D242EA01202862DC
:10768000EB7005E0052C03D2624508BF01F034F829
:107690002889401C2881002070BD10B503F0070127
:1076A0001046012905D013F0070F08BF00F01CF9A0
:1076B00004E09F490020C861C8700881002010BD07
:1076C00010B5104613F0070F08BF00F00DF90020A9
:1076D00010BD70B5072600244FF4103505EB0430BB
:1076E000FAF7B8FE022808BF70BD601CC4B2B442ED
:1076F000F4D3012070BD30B403F007030024DFF899
:1077000030C2029A012B02D0022B0CD008E00520D7
:107710008CF80200ACF808409CF805008CF80300D7
:1077200030BC002070479CF80230052B14D1BCF807
:107730000830934205D29CF803500570581CACF8F1
:107740000800BCF80800904206D1ACF808400120BF
:10775000087003208CF8020030BC012070472DE92E
:10776000F047AFF69860DDF820C0006803F0070529
:1077700000276F4E6F4C012D03D013F0070F06D07A
:1077800034E0378120680770206847702EE0338925
:10779000634503D22568EA545A1C32813289624516
:1077A00024D137814FF0010881F800802168C2B2EE
:1077B000097891421AD12168C0F3072049788142A3
:1077C00014D1072500244FF4103909EB0430FAF7DF
:1077D00041FE022804D0601CC4B2AC42F5D340463E
:1077E000012806BF86F80580377177710020BDE853
:1077F000F0872DE9F0414FF0000C03F007004E4EEA
:107800004B4C6546012803D013F0070F0CD068E0FD
:107810002570E580A5616570002046F82050401C69
:10782000C0B24028F9D35CE0207805283CBF401C5A
:107830002070C0B2012808BF100222D03C490228A3
:107840000B8A08BF98181CD024BFE1888B4248D906
:107850003A4F01F0030001F101083A54A7F1280062
:107860004FF410328069984502EB002008BF0021D8
:1078700009D1491CC9B20429FBD32F49FAF71DFECF
:1078800026E020822DE0032232EA010120D17A5C39
:10789000CB009A40491CC9B242EA0C0C0429F6D329
:1078A000617801F03F02491CC9B246F822C06170FC
:1078B00040290DD12049FAF700FE6570A069401CEF
:1078C000A061002046F82050401CC0B24028F9D3E7
:1078D000E088401C80B2E080218A884204BF0120F9
:1078E00020710020BDE8F08110B5114C214623899C
:1078F000CA78D1F81CC01118C9B2022B03D240EAD1
:107900000C20E06107E0B3F5817F06D2094A1268D6
:107910001A4402F8020CE17006E008BF904203D15D
:107920000549604600F00AFF2089401C208110BDF7
:10793000C0400020A4920100E4590020E84000204B
:10794000BE48002101704170C1700171BC4A0846F7
:107950001154401C0428FBD3704710B4B74C637813
:10796000002B1EBF002010BC7047E0702271002069
:10797000002A88BFB24B06D911F800C003F800C036
:10798000401C8242F8D80120607010BC7047AB48A0
:1079900040787047A94880787047A84900208870CF
:1079A000704770B50024FBF7D2FDA44D687801281C
:1079B00006D100F012F804461120E870002068702B
:1079C000FCF7ACFE022802D101F019FE18B9002C18
:1079D00004BF002070BD012070BD2DE9F04797481D
:1079E0000024C078112880F02681DFE800F00C1711
:1079F000250936FB3A81696F74AEFA8290959A0038
:107A0000FCF734FF26E08E4801780120FCF798FE51
:107A10008A4901208870044600F00DB98848007832
:107A200001F0E6FF01210320FCF78AFE83490120D3
:107A30008870044600F0FFB881484178007841EA38
:107A4000002003F0C9FF02210320FCF779FE7B49E7
:107A500001208870012400F0EEB879484178007860
:107A600070E0764E0120B07000277770317829BB26
:107A7000711D0D78307015F0040F18BFFEF7C2F8B5
:107A800015F0020F05D0FF210F20FDF7C8F845F0D3
:107A9000010515F0010F10D0FCF740FE022802D1BD
:107AA00003F0E0FF48B1FCF739FE052802D100F0F1
:107AB00081FE10B10020FCF768F93770B770BAE0AA
:107AC0005F480078401E01F0D9FBC3E75C480078AE
:107AD00003F0FAFFBEE75A480078002804BF0021EF
:107AE000032003D003F0C7FF01460220FCF728FE65
:107AF000A1E0534D2878002818BF012003F097FF1C
:107B00002878002818BF012000F03EFE93E04C4882
:107B1000007803F07DFF9DE74948007803F0EDFF12
:107B200098E74748007820B1012860D0022805D0A6
:107B300081E04FF42F30FAF758FC7CE001F0D2FDE1
:107B400000210420FCF7FCFD84E73C484FF00008CE
:107B500080F801804646454672B6FBF76CFB48B19B
:107B6000FBF743FC0646FBF720FCFBF744FC05460D
:107B7000FBF72BFCF9F77CFCF9F798FB8146F9F74A
:107B80000FFDFBF738F9070018BFFBF706F94FF4B4
:107B90009350FBF774F862B62A48C0F800802A4870
:107BA0000168D1F8CC10006841F4BE0141F02041D9
:107BB000C0F8C8100DF0B2FB72B6B9F1000F03D0D7
:107BC000F9F756FCF9F749FDFBF735FB38B1002E04
:107BD00018BFFBF736FB002D18BFFBF77EFB002F0D
:107BE00001E018E004E018BFFBF78FF862B622E06E
:107BF00013480078012804BF04210520A2D00228E0
:107C000004BF002103209DD0032819BF022108468C
:107C10000021042096E70A480178427841EA0221CF
:107C20008278C078120442EA006041EA00021E2114
:107C3000012003F0F2FB2046BDE8F087EC40002075
:107C4000F1400020304000208C92010002460020CC
:107C5000022928BF704752B1012A18BF704701EBB3
:107C6000810000EBC100F84901EB00107047C1EB47
:107C7000C100F64900EB800001EB4010704770B581
:107C8000FAF7F9FF00F008060820FAF7EFFFF04CCA
:107C900000256078302806D24FF40C61EB480DF0D7
:107CA000F0F9A570E570A079302806D24FF4D071B4
:107CB000E5480DF0E6F9E57125723046BDE8704003
:107CC000FAF7D0BF00FB01F2B2F50C7F9CBFE04A8F
:107CD000C2E9030170470028DD4AD26818BF02607C
:107CE000DB480029006918BF086050437047D84836
:107CF000012101710078D54980F00100C0EBC0007E
:107D000000EB800001EB40107047D14882780021E1
:107D100032B1C27822B9027882F001020270817019
:107D200001717047CA491E284A78487008BF002070
:107D300003D01F2808BF012000D1087010467047EB
:107D4000C3480078C14980F00100C0EBC00000EBDF
:107D5000800001EB40107047F0B4BD4E96F800C0B3
:107D6000BA4CCCEBCC0CF5680CEB8C0C04EB4C1C3B
:107D700003FB05F40CEB440C8D4234BF2C460C463F
:107D80003669F31A934238BF1A460026002A9CBF70
:107D9000F0BC70470023002C06D930F813702CF883
:107DA00013705B1C9C42F8D8761C0CEB450C00EB66
:107DB00041009642EED3F0BC70472DE9F041A44F4C
:107DC00014468C4601467A7806981D468A4218BFAA
:107DD000BDE8F0810121F970012802D0022825D0E8
:107DE0002AE038789949C0EBC000FE6800EB8000BB
:107DF00001EB4011A64234BF324622463869A84200
:107E000038BF05460023002D16D90020002A06D9C8
:107E10001CF8007021F81070401C8242F8D85B1CDE
:107E200001EB4601A444AB42EFD305E000232A4610
:107E300021466046FFF790FFBDE8F04100F096BB99
:107E4000002808BF70478249824B4A7882491B78D4
:107E5000002A097818BF022A05D0042A18BF092A67
:107E600001D0012278E77D4A1278012A84BF7C4A3A
:107E70001378012200F094BB2DE9F04F744983B0D0
:107E80000122CA70774A49781778724A23291678EE
:107E900024BF03B0BDE8F08FDFE801F01222122208
:107EA00012222222221222222222B7B7222A2A2A90
:107EB000B7B7B7B7B7B7B7B7B722B7B7B7ACAC00B4
:107EC00066490978012903D967490F7864490E7812
:107ED000002875D000233246394600F061FB8FE060
:107EE00000286DD0002332463946FFF735FF87E082
:107EF000F9F7BEFAF9F7DAF90090002818BFF9F798
:107F0000DEFB56480078012884BF55480678F9F70B
:107F10009BFB10F0040F18BF761C5448DFF830A10B
:107F2000006800F5804001909AF80100A0F1110866
:107F30009AF800004549C0EBC00000EB800001EB5F
:107F40004014DAF80C00B84238BF0746DAF81000DF
:107F5000B04238BF0646F9F708FC81460020F9F721
:107F60007EFF0025002E3FDD4FF0000A002F34DD9C
:107F70000199C5EBC50001EBC00B19F90A001C28DB
:107F800024BF002024F81A0023D200EBD07149103E
:107F9000C0075BF82110C00E21FA00F081B24FF04B
:107FA000FF30B8F1000F0CD0B8F1010F08BFC8B214
:107FB0000DD0B8F1020F04BF0846F9F756FF06E0EE
:107FC0001EE011F4805FC1F3032018BF404224F883
:107FD0001A000AF1010ABA45CFDB1D486D1CB542F3
:107FE000C06804EB4004BFDB0098002818BFF9F715
:107FF00069FB05E020B10023B21C3946FFF7ACFE57
:1080000003B0BDE8F04F00F0B1BA03B0BDE8F08FA7
:108010000F4801214172407980F0010000EB80019E
:1080200001EBC000084901EB001070470848C27915
:10803000002132B1027A22B9427982F00102427102
:10804000C171417270470000A4630020E45A00200F
:10805000F84000207F400020854000208040002024
:10806000824000207E40002081400020A09201003C
:10807000FE491E288A79887108BF002003D01F2876
:1080800008BF012000D1487110467047F748407979
:1080900080F0010000EB800101EBC000F44901EB2E
:1080A000001070472DE9F04FF24985B0012291F898
:1080B0000080F14991F80090EC490A728979EC4C02
:1080C00011291CBF1229132939D008B3E74949796E
:1080D00001EB810202EBC10104EB01120021B9F1B5
:1080E000000F06D930F8113022F81130491C8945AB
:1080F000F8D80021B8F1000F0AD909EB010302EB0F
:10810000410C30F81330491CACF868308845F4D87D
:10811000FAF7B1FD00F008050820FAF7A7FDD34CE7
:10812000607A002818BF012100F0B880E17128466C
:10813000FAF798FD0020207205B0BDE8F08FF9F73E
:1081400097F9F9F7B3F80190002818BFF9F7B7FAD3
:10815000C6488179A1F11106817A0091407900EB3E
:10816000800101EBC00004EB0015F8F7A8FBC34940
:108170004FF0110B0028096801F5804101F5F56702
:1081800001F5E76104BF8A46012004D0BA4658468B
:108190000F464FF0010BF9F762FEF9F7E4FA0024FD
:1081A0000390B9F1000F35D90098C0EBC000C000B2
:1081B0000290039800570828B4BF143008381C28D0
:1081C00024BF002025F8140021D200EBD0720299C0
:1081D000521001EB8201C00751F80A10C00E21FABB
:1081E00000F081B24FF0FF304EB1012E08BFC8B28F
:1081F0000BD0022E04BF0846F9F737FE05E011F454
:10820000805FC1F3032018BF404225F81400641CAE
:108210004C45CED35846F9F722FEF9F7A6FA0024CA
:108220008246B8F1000F33D90098A346C0EBC000D6
:108230004FEAC0091AF904001C2824BF05EB4400CA
:10824000A0F868B021D200EBD071491009EB810190
:10825000C007C959C00E21FA00F081B24FF0FF30BB
:108260004EB1012E08BFC8B20BD0022E04BF084683
:10827000F9F7FBFD05E011F4805FC1F3032018BF9F
:10828000404205EB4401A1F86800641C4445D1D389
:108290000198002818BFF9F715FA39E7607980F0DE
:1082A00001006071002141E72DE9F04F774D6F4CDF
:1082B000DFF8D4812978627895F801C0704E714F4B
:1082C00098F8003085B06144092A7BD00FDC002A81
:1082D0001CBF022A042A75D0002804BF05B0BDE8DF
:1082E000F08F5B1C05B00122BDE8F04F34E5112A88
:1082F0001CBF122A132AEFD1F9F7BAF8F8F7D6FF04
:108300000290002818BFF9F7DAF9307801288CBFFD
:10831000397898F800105948491C006800F58040E9
:10832000039028786A782369104462789942A2F110
:108330001109A27A62D22378D4F80C80C3EBC3036C
:10834000DFF84CC103EB83030CEB431301FB08F193
:1083500003EB410A804528BF80460220009012208E
:1083600001900025C2EBC2002E4604906C465DF8D9
:108370002600F9F774FD54F82600F8F739FD834616
:108380000399C6EBC60001EB00100499002400EB32
:10839000C1072CE00120A04010EA0B0F26D004EB0F
:1083A000D470401007EB8000E107D0F81808C90E20
:1083B000C84081B24FF0FF30B9F1000F0DD0B9F1D4
:1083C000010F00E025E008BFC8B20CD0B9F1020FE0
:1083D00004BF0846F9F749FD05E011F4805FC1F3D9
:1083E000032018BF40422AF815006D1C641C454547
:1083F000B8BF1C2CCEDB761C022EB7DB02980028FF
:1084000004BF05B0BDE8F08F05B0BDE8F04FF9F747
:1084100059B93278012A88BF3B7800287FF461AFD0
:1084200005B0BDE8F08F70B50D4610490122CA7045
:10843000184A49781678144A212914781EBF22292F
:10844000232970BD002818BF002D28D00023224604
:108450003146FFF781FC631C012221462846FFF7C5
:108460007BFCA31C05EB4400012215E0F840002032
:10847000A46300208340002084400020A0920100DB
:1084800080400020824000207F4000208640002065
:10849000E45A00207E4000203146FFF75DFCBDE835
:1084A000704000F063B870B5604D0446687868B9F4
:1084B000A06858B15E490978012994BF5D495E49B9
:1084C0000B785E490122097800F06AF8606920B1F2
:1084D0006978002908BFFFF7E7FE6878112804BF14
:1084E0000020FFF7E1FE6878122804BF0020FFF7A4
:1084F000DBFE6878132804BF0020FFF7D5FE6878FC
:10850000002804BF6068FFF7B7FC6878112804BF33
:108510000020FFF7B1FC6878122804BF0020FFF7A5
:10852000ABFC6878132804BF0020FFF7A5FCE068C7
:1085300010B1A97921B105E0206918B1A97909B96B
:10854000FFF7B0FDA879112804BF0020FFF7AAFDAE
:10855000A879122804BF0020FFF7A4FDA8791328EA
:1085600018BF70BD0020BDE870409BE570B5FAF7FC
:1085700082FB00F008060820FAF778FB2B4C2079E4
:108580000025002801BF207880F001002070A57030
:108590001CBF0120A0703046FAF764FBE57070BD87
:1085A0002DE9F047994616460D460446F9F7E2F8DC
:1085B0005FEA000C1DD01D490878214AC0EBC000BD
:1085C000D1F80C8000EB800002EB401009FB08F2B0
:1085D00000EB4200A8452CBF2F4647460969A1EB96
:1085E0000901B14238BF0E460021002E09D8BDE86E
:1085F000F0874B46324629462046BDE8F047FFF754
:10860000ABBB0023002F08D91CF9032034F812203B
:1086100020F813205B1C9F42F6D8491C00EB480051
:1086200004EB4504B142ECD3BDE8F087F8400020EC
:10863000804000207F4000208240002085400020B4
:10864000E45A00202949002814BF002001200870A6
:1086500070472648007800280CBF01200020704792
:108660002248017871B122490A6852690B6842F0C8
:1086700001025A610A68126B1E4B096822F44052CB
:108680001A430A63002141608160C1600161416158
:108690007047E5E700B50178C27983B0114341F036
:1086A00040018DF8001041788DF801104188C1F328
:1086B00007118DF802108188C1F307118DF803109E
:1086C000817801F00F02017962F31F118DF8041017
:1086D00081798DF80510017A8DF80610407A8DF8B1
:1086E000070068460DF014F803B000BD0C410020EF
:1086F0008492010000205FA070B50E460446FCF78E
:108700000DF8042811D1A4F5107080280DD2A019FD
:10871000A0F24120802808D225020024002E04D98E
:108720002846F9F762FE012801D0002070BD641CC4
:1087300005F58075B442F3D3012070BD70B50D46C8
:108740000446FBF7EBFF04280AD1A4F5107080283B
:1087500006D220022946F9F7B0FE012808BF70BDF5
:10876000002070BD10B5074CFFF71BF9012808BFAA
:1087700010BD206801F05AF8002818BFFCF707F870
:10878000F2E7000078410020884A0028916814BF71
:1087900041F0010021F0010090607047834B99681F
:1087A000C1F30362120721F07F4142EA00600843EF
:1087B000986070477D488068C0F3036070477B48CD
:1087C0008068000F70472DE9F04F794F87B0386807
:1087D000B0F90E11B0F90C0100F03CFB0AF0B9FC45
:1087E0003868D0F8F800C0F30340FBF780F9FBF7D6
:1087F00095FF052836D1DFF8BC91DFF8BCB16B4D91
:108800004FF000084FF47A7AA868C0F30364386820
:10881000A100D0F8F800C5F80C80C84000F00F06A1
:1088200021460520C5F8108002F078FE002C7CD08F
:10883000022C1ED0042C79D0A8680A2CC0F3036146
:1088400020F07F404FEA017118BF41F0007141EA0A
:108850000000A860FFF7A5F8012803D0FBF75EFF32
:108860000528D1D0FBF75EF907B0BDE8F04F0AF05C
:1088700077BC0F213046FCF721F80028EAD000F041
:1088800038FC00F02CFCFBF7EAF806460020F8F76D
:10889000C4F94A48F8F751FD0120F8F743FDFAF70B
:1088A00011FA4748FAF7D8FAFAF7BDFAFAF7EAFAEE
:1088B0003968B1F80621504300F5FA70B0FBFAF0C0
:1088C00082B2AA8091F80801287050B1FAF7DAFA5A
:1088D0003968B1F80411484300F5FA70B0FBFAF0BA
:1088E00082B21046FAF740FAD9F80010354888618C
:1088F000F8F7BEFDF8F7C9FE287838B1401E10F031
:10890000FF00287004BFA888FAF72EFAA868C0F301
:108910000364FFF746F8012806D0A868C0F3036097
:10892000A04208BF002E1DD001E036E039E0D9F8A2
:108930000000C0F818B0FAF730FAFAF780FA002011
:10894000FAF78AFAFAF7CBF9F8F792FDF8F7B0FCE4
:108950000020F8F7F2FC00F0C2FB00F0CBFBFCF7C4
:108960001EF977E76846F9F70BF858B16846FFF744
:108970009AFD68460DF07AF80646F9F737F8FBF7E6
:1089800027FFC6E73868406E10F0704F02D0FBF743
:10899000FEFEBEE7FBF723FFBBE730460EF065F8AF
:1089A00058E7304603F04AF954E70000244100201C
:1089B000784100208492010000005FA0B58801008A
:1089C000197B010007005FA07047002808BF7047AF
:1089D0008022014601480CF04FBB7047E46500203F
:1089E0002DE9F047904601FB08F50F4601461E466B
:1089F0002A46F6480CF04AFBF44C03F0E9F880B341
:108A000000210D46B8F1000FC6BFF14A0023BDE8B2
:108A1000F0870020002F1FDDD2F800C09CF83E91A7
:108A2000A945DCBF9CF83F914D4510DC9CF83C917A
:108A30008145DCBF9CF83DC1604508DC14F901C0EC
:108A40000CFB06FC4CF3073C04F801C000E0635447
:108A5000401C491CB842DFDB6D1C4545D9DBBDE835
:108A6000F087FFE7B6F5805F1CBF0020002DD8BF60
:108A7000BDE8F0872156714341F307312154401C72
:108A80008542F7DCBDE8F0872DE9F0411C4615462C
:108A90000E460746F9F740FE21462846F9F7BDFE87
:108AA0000623CA4A31463846FAF709F8BDE8F041CC
:108AB000F9F745BEC74B1A61C3E902017047C449C3
:108AC0000020096891F8301011F0020F1CBFC14856
:108AD000406970470020BE49096891F8301011F0D4
:108AE000020F18BFBC4870472DE9F00700248FB073
:108AF000002B9EBF0FB0BDE8F0077047561E4FF029
:108B000000086F464FF0000C002E16D904FB02C57A
:108B100031F8159001EB45056D88A9EB05052DB2DF
:108B200027F81C500E351C2D98BF27F81C800CF11F
:108B3000010C1FFA8CFCB445E8D304FB02FC012AAB
:108B400020F81C804FF0010C13D904FB02C507EB81
:108B50004C0A00EB45093AF802AC39F8029C0CF1DA
:108B6000010CA9EB0A091FFA8CFC20F8159062454C
:108B7000EBD804F1010C1FFA8CF49C42C2D30FB065
:108B8000BDE8F00770472DE9F04FADF2246D03FB0F
:108B900002FA4FF0000CE946BAF1000F84BF00263C
:108BA0008E4D13D931F91C4004F10F071E2F98BFC9
:108BB00029F81C6004D935F81C70E41B29F81C4006
:108BC0000CF1010C0FFA8CFCE245EBD84FF0000CD5
:108BD000002B59D90CFB02F44FF0000B39F914802B
:108BE00008F11904322C3CD901252C46012A38D928
:108BF0000CFB024639F9167007F10A0EBEF1140F8C
:108C000014D907FB08FEBEF1000F0FDD09EB460E7D
:108C10003EF902ECA7EB0E071837302F06D831F9D2
:108C200016600F361E2E84BF6D1CEDB2641C24B27C
:108C3000A242DDD8142D11D900244FF0010B002AD7
:108C40001CD90CFB0245641C31F8156039F815700D
:108C500024B2F61B20F81560A242F2D8BBF1000F37
:108C60000CD10024002A09D90CFB0245641C31F800
:108C7000156024B220F81560A242F5D80CF1010C61
:108C80000FFA8CFC6345A5D80021BAF1000F8EBF06
:108C9000524A0DF2246DBDE8F08F30F8113022F801
:108CA0001130491C09B28A45F7D80DF2246DBDE890
:108CB000F08F2DE9F04FDFF828C19DB00DF11008BD
:108CC0009CE8F0008DE8F0000CF11004F0CCA8E86E
:108CD000F0000CF12004F0CC88E8F000DCE90C4C4A
:108CE000CDE90C4C0026002B9CBF1DB0BDE8F08FD9
:108CF0000DF1380BA2F1010AEE464FF0000C65466B
:108D000067466446BAF1000F31D906FB024831F8D4
:108D1000189001EB4808B8F80280A9EB08080FFA90
:108D200088F82BF8148008F10F08B8F11E0F9CBFCB
:108D30000CF1010C1FFA8CFC0BD9AC4507D9BCF126
:108D4000000F04D06546A4F1010C0CF0FF074FF0B2
:108D5000000C641CA4B25445D7D3AC4507D9BCF170
:108D6000000F04D06546A4EB550C0CF0FF07052D51
:108D700023D906FB027C31F91CC00CF10F041E2C18
:108D80001BD93EF81740002AA4EB0C0C0FFA8CF507
:108D90004FF0000C11D906FB02C43EF81C8031F8DC
:108DA0001470A8EB05080CF1010CA7EB08071FFADB
:108DB0008CFC20F814706245EDD806F1010C1FFA06
:108DC0008CF69E4299D31DB0BDE8F08F9C660020C2
:108DD0007841002038410020646600205C68002053
:108DE000A89201002DE9F0410746C348C44EDFF8C0
:108DF00018830578C148B2690478C248A0FB0230E4
:108E00004308A3EB8300831805FB04F04200C3EB87
:108E1000C30008EBC0100CF039F9B069421CB26114
:108E2000002F08BFBDE8F081032A38BFBDE8F081FC
:108E3000F9F772FC21462846F9F7E6FC08F5E063ED
:108E400008F56072B0493846F9F70DFDBDE8F0410C
:108E5000F9F775BCAA49C88070472DE9F041AB4EBF
:108E60008AB00546A648CDE90056A6F170080C4622
:108E7000CDF80880B0F9061003913F29C8BF3F2004
:108E800005DC11F1400FB8BF6FF03F0000DA03902E
:108E900000200490F9F740FC9848974F0178387803
:108EA000F9F7B2FC6846F9F748FD0890F9F747FC76
:108EB000C4E90068BDF814002081BDF81600608187
:108EC000BDF81800A081BDF81A00E081BDF81C00B3
:108ED0002082BDF81E006082BDF81C00BDF81E1087
:108EE0003A7801FB020035F910000AB0BDE8F081C4
:108EF0008348C06970478648704786487047B0F914
:108F000000300122012908DD30F912C09C45B8BFAC
:108F10006346521C12B28A42F6DB00220029D8BFF7
:108F2000704730F812C0ACEB030C20F812C0521C92
:108F300012B29142F5DC704770B4D4B2B0F900C0FF
:108F400001230646012C08DD30F913506545B8BFF2
:108F5000AC465B1C1BB2A342F6DB0023002C09DDF0
:108F600030F81350A5EB0C0520F813505B1C1BB216
:108F70009C42F5DC00EB4202CBB2B2F900100120BA
:108F8000012B08DD32F910C08C45B8BF6146401C8A
:108F900000B29842F6DB0020002BDCBF70BC7047AB
:108FA00032F810C0ACEB010C22F810C0401C00B22B
:108FB0008342F5DC70BC70475148406A70475648A0
:108FC00070472DE9F84F814654480F461646017800
:108FD0004078514D0C18FAF752FBDFF844815FEAF4
:108FE000000A4FF0020B16D0601C43084A46514657
:108FF0001046CDF800B00DF0EFFF98F80000022801
:1090000004BF5046FFF750F998F80000092804BF44
:109010004846FFF749F9FAF78BFE8246601C430881
:109020004A4651462846CDF800B00DF0D5FF98F8D5
:109030000000032804BF5046FFF736F998F80000F7
:10904000062804BF2846FFF72FF92D480169B1F51E
:10905000805F1CBF0020002C08D935F910204A433E
:10906000121325F81020401C8442F6D898F800000E
:10907000082804BF2846FFF717F998F800000128D0
:1090800004BF2846FFF710F937B34FF0FF32002036
:109090000146002C06D935F81130491C184400B29D
:1090A0008C42F8D81F490B68B3F8501031B1814297
:1090B000CABFB3F852100122814200DD00223A609B
:1090C000002E18BF30802A80688098F8000007289A
:1090D00004BF2846FFF7E8F84846BDE8F88F08487F
:1090E00000210162816170470548002101628161B0
:1090F00070477047704700007E4000207F4000208E
:1091000038410020ABAAAAAA7C6E00206C7900200E
:109110009C7E00205C7D0020F47E002086400020A4
:10912000F940002078410020704708283CBFFE49E4
:10913000087070470020FC4988604860FB48006860
:1091400090F88100082838BF087070470020F64961
:1091500048607047F4480078704770B5F34D0024BC
:10916000286890F86C0010F0020F0BD0FBF7D6FACD
:10917000022807D1EC482968007801EB8000B0F89C
:10918000840084B2204670BD70B5E84D4FF4805421
:10919000286890F86C0010F0020F0DD0FBF7BEFAB3
:1091A000022809D1E0482968007801EB8000D0F856
:1091B0008400000CC0F31304204670BDDA488078A8
:1091C000002818BF012070472DE9F041FBF7A6FAEF
:1091D000022803D102F046FC022803D04FF480504D
:1091E000BDE8F0814FF480552E4602F068FCDFF8B0
:1091F0003C830446CC4FD8F8000090F86C1011F076
:10920000010F0CD0B0F87600B9684042884206DB06
:109210002CB10020641EB860204602F055FCD8F83E
:10922000001091F86C0010F0040F18BF002C0AD049
:10923000B1F87C00621E9040B1F87E20824238BFB7
:109240001046C0F31306D1F8A40010F0020F1CBFA3
:10925000B978002902D0000CC0F31305B54298BFBD
:10926000354602F0B5FC00281CBF4FF40050B5F5A0
:10927000005F38BF05462846BDE8F0812DE9F04F74
:10928000DFF8A8A287B0DAF8001091F86C2012F08D
:10929000020F0DD0A44A91F88090DFF894B21778AD
:1092A000002809DB484503D2B84218BF06463DD125
:1092B00007B00020BDE8F08F3E464FF0FF38F7F7CB
:1092C000F7FFF8F761FE0025B9F1000F2ED9DAF8A3
:1092D0000000002400EB8500B0F8840081B2204635
:1092E000F7F7C7FCF8F7D1F96846F8F749FB00280B
:1092F0005FD0019878B101468E489BF80020007835
:109300005043421E38B131F9020B0028B8BF404229
:109310000444521EF7D2F8F769FBF7F7C9FFA045DE
:1093200084BF2E46A0466D1C4D45D0D3B74243D0D6
:10933000082E3CBF7C490E70DAF80000B0F88210AD
:1093400039B300EB870200EB8600B2F88420B0F856
:10935000840092B280B2801A484340F30F34FAF787
:109360002DFC754B9BF80020002193F800C002FBF8
:109370000CF2002A0DD930F81120224420F81120D7
:109380009BF8002093F800C0491C02FB0CF28A42B3
:10939000F1D84FF0806002F043FCDAF800000221BF
:1093A00000EB8600B0F8840082B2032002F035F8AA
:1093B00009E0FBF7ECF997E702F081FB03283CBFDB
:1093C000401C02F081FB012007B0BDE8F08F574838
:1093D00055490068B0F87600424288688242BCBFB6
:1093E000401E886070472DE9F04F8FB093460E46BF
:1093F00004464FF0000A02F062FBDFF830814A4F6A
:109400000500D14610D1FFF75AFBD8F80010B1F88B
:109410007810884208D30120C7F8089002F054FB66
:109420000FB00120BDE8F08F002E1FDDB8680028C6
:10943000B8BFC7F8089007DBD8F80010B1F874106F
:109440008842BCBF401CB860D8F80000B968B0F8CA
:109450007400884215DC032D13D2681CC7F80890ED
:1094600002F032FB0FB00120BDE8F08F09D1D8F82F
:109470000000B0F876004142B8688842C4BF401E80
:10948000B860B87850B1D8F8000090F8A40010F097
:10949000040F1EBF00200FB0BDE8F08FD8F8000009
:1094A000B0F972108C420EDD796821447960B0F811
:1094B0006E00884210DC4FF0FF30C7F80490FFF7D1
:1094C000DDFE824608E07868002805DD002CD4BF68
:1094D00001212146401A7860DFF8609099F8000079
:1094E00007283AD1164859460078420068460BF0E2
:1094F000CDFDADF80040ADF80260ADF804503889FC
:10950000ADF80600B888ADF80800D8F80000B0F84B
:109510007210ADF80A10B0F87410ADF80C10B0F875
:109520006E10ADF80E100DE068410020784100206B
:109530007E400020824000207F400020F940002033
:1095400085400020B0F87600ADF8100099F80000D2
:10955000072804BF6846FEF773FC50460FB0BDE80D
:10956000F08F3E4810B50068D0F8A40010F4807F5A
:1095700006D0C0F30330012101FA00F0F9F77DF8BD
:10958000374900204870887010BD70B5344D0024F4
:10959000A878002814BF01260026687828B902F0B0
:1095A000A7FA002808BF002100D001218E4224D054
:1095B0000A1C18BF0122AA7028480068D0F8A430FD
:1095C00013F0040F0ED021B1C3F30310082808D202
:1095D00006E00021A960696090F88100082800D2A7
:1095E0002870012413F0020F18BF0124002A18BFAD
:1095F00001220421032001F010FF204670BD17490D
:1096000000200968D1F8A41011F4807F08BF7047CA
:10961000DFF84CC09CF80120131C18BF012330B4A4
:10962000104CC1F303322468E46B012505FA02F201
:10963000224011F4007F01D00AB102E00AB10021FA
:1096400000E001218B4204BF30BC7047081C18BFEA
:1096500001208CF8010030BC97E700007841002021
:10966000684100207C9201005948006800F5407074
:1096700070475748006800F58070704770B5544CCB
:109680004FF41032534922601068884204BF50687A
:10969000B0F5087F24D1D2F808C0BCF5D04F1FD850
:1096A0004D49D06888420DD0002311461846B3EBCF
:1096B0009C0F07D251F8045B401C6B40B0EB9C0F31
:1096C000F8D36BB902F5807000F0B0F840B12068B3
:1096D00000F5407000F0B9F800281CBF012070BDF3
:1096E000002070BD4FF41030F8F77FBE3848394A7B
:1096F00000680168914206BF4168B1F5087F00200B
:109700007047334B1B6803F580731844F8F73BBF71
:109710002F4B1B6803F540731844F8F734BF2C48EF
:109720000068006970472A4909680A6982429CBF3B
:1097300000207047C0EBC00001EBC00000F5806066
:109740007047234A126802EB80035B6A1A44234B7A
:1097500053F82000FF3020F0FF0000FB012070478D
:10976000F0B41B4B00221D4E1C681746831893F95A
:1097700028C0BCF1000FB8BF41F822700DDBD3B296
:1097800004EB830556F823306D6AFF33254423F03C
:10979000FF0303FB0C5341F82230521C102AE5D37F
:1097A000F0BC704794460029B8BF7047084A126859
:1097B00002EB80035B6A1344084A52F8202002F14E
:1097C000FF0020F0FF0001FB00306146F8F7DBBE30
:1097D0007441002054465053EFBEADDEE0920100CC
:1097E00010B51F4CFFF74AFFA0B1FFF73DFF014640
:1097F000C4221C480BF040FCFFF73BFF01464FF42E
:10980000C27220680BF038FC2068406DBDE8104043
:1098100002F0E8B84FF4C27120680BF032FC00216E
:109820000420FAF78DFFFEF79DFFDBE758B10E4AE3
:109830000168914207D1406820F00F00B0F5087F21
:1098400004BF012070470020704730B1006820F04D
:109850000F00502804BF012070470020704700000F
:1098600078410020747F00204150535210B572B6E9
:109870000120F8F7C5FCF9F7C3FBF9F7F1FB4FF04E
:10988000FF30F9F7F3F9554880234FF400520021D7
:1098900052F821C040F821C0491CB1EB930FF7D317
:1098A000F9F7F6F9F9F70CFEF9F736FE0120F9F7AA
:1098B00008FEF8F767FD1E20F9F7F6FDF9F7FCFB47
:1098C000F8F7EAFEF9F7ACFDF9F750FCF9F7F6F90D
:1098D000F8F755FFF7F7FFFCF9F772F9F9F72CF9EC
:1098E000FEF72EF8FCF738FBFEF7D3FE62B6FFF763
:1098F00077FF3B4809F040FB3A4C2068B0F90C0177
:1099000009F022FCFFF710FCF9F73CFEFBF77FF9AA
:109910002068418A008AFEF7D5F92068806EC0F37E
:109920004E0161F35F0001F06BFDFFF74DF8FFF7AB
:10993000DBFBFAF7B9FF206890F8640000F00F0035
:10994000F8F76AFB2848006800690C2100F07002F3
:10995000012001F062FDFFF704FE002010BD224847
:109960000068006910F0200F04BF0021032003D01D
:1099700002F081F801460220FAF7E2FE01251B4CB5
:10998000FAF7CCFE062825D2DFE800F02414031EE7
:109990002111207840B9FCF730F928B900221E21A6
:1099A000022001F03AFD257002F049FBE8E7FEF7DE
:1099B0000AFFE5E7FCF759F8FAF7B0FE012804BF03
:1099C0000220FAF7BAFEDBE701F0F1FDD8E7FEF777
:1099D000C9FED5E7FAF742FFD2E700000082002077
:1099E000747F002078410020849201007C41002097
:1099F000FE490870704710B44FF42C30FC4A0168DF
:109A000091421CD14168B1F5007F18D383680022D0
:109A10008446B3F5066F88BF4FF406630021B1EBAF
:109A2000930F24BF10BC70475CF82140491C2244AE
:109A3000B1EB930FF8D3002A04BF10BC704700208D
:109A400010BC70472DE9F0414FF42C350446E84E28
:109A50002868B04217D16868B0F5007F13D3A968B1
:109A600000222B46B1F5066F88BF4FF40661002037
:109A7000B0EB910F08D253F820C0401C6244B0EB09
:109A8000910FF8D302B1002500274FF40668B5B155
:109A9000AA68B2F5066F88BF4FF4066229462046D1
:109AA0000BF0EAFAA868B0F5066F22D2C4F8507835
:109AB000C4F85478C4F80880C4F8587819E0FF2234
:109AC0004FF4066120460BF0E6FA4FF40070C4E94B
:109AD0000060C4E9028784F8207084F8217084F85B
:109AE000227084F8237040F2FF70C4E90407A76174
:109AF000E7610120BDE8F08110B590F8221049001F
:109B000004BF4FF40561816000210B46C16081688C
:109B10008446B1F5066F88BF4FF406610022B2EBB0
:109B2000910F06D25CF82240521C2344B2EB910FF5
:109B3000F8D35942C1604FF42C304FF406626146AD
:109B4000F8F721FD012818BF002010BD4FF4007167
:109B500070B402685160016801F1500291F821C0AF
:109B600091F820300CFB03F102EB41010022BCF123
:109B7000000F08D900EB4204521CB4F88A4021F8C7
:109B8000024B9445F6D80022002B08D900EB420482
:109B9000521CB4F8CA4021F8024B9342F6D804682C
:109BA000002294F82240002C0BD900EB4204521CF6
:109BB000B4F88A4221F8024B046894F82240944297
:109BC000F3D80468002294F82340002C0BD900EB52
:109BD0004204521CB4F8CA4221F8024B046894F8BB
:109BE00023409442F3D80022BCF1000F07D900EBC8
:109BF0004204521CA48821F8024B9445F7D8002255
:109C0000002B08D900EB4204521CB4F8444021F860
:109C1000024B9342F6D8B0F8862021F8022BB0F818
:109C2000882021F8022BB0F8842021F8022B002490
:109C30000022BCF1000F88BF00EB841508D905EBAA
:109C40004206521CB6F80A6121F8026B9445F6D818
:109C50000022002B88BF00EB841508D905EB4206D3
:109C6000521CB6F8CA6121F8026B9342F6D8641C04
:109C7000032CDDD30023D0F800C000229CF822C0C2
:109C8000BCF1000F88BF00EB831C0BD90CEB420426
:109C9000521CB4F80A4321F8024B046894F822409D
:109CA0009442F3D8D0F800C000229CF823C0BCF145
:109CB000000F88BF00EB831C0BD90CEB4204521C35
:109CC000B4F88A4321F8024B046894F82340944284
:109CD000F3D85B1C022BCED370BC70472DE9F74F35
:109CE00088B000250A992C462E460968049101F196
:109CF00050030999002984BF3E49D1F800801CD93E
:109D00000022002888BFB8F9CE700DD933F9021BA4
:109D10000029B4BFC1F1000C8C46BC45BCBF0D444A
:109D2000641C521C8242F1D30999761C8E42E7D3FF
:109D3000002CC8BF95FBF4FA08DC4908414301EB4D
:109D40005002049901EB4201B1F950A000210291A7
:109D50000191049950310091002103910999002942
:109D600075D92449009E069609684FF0000B4FF004
:109D70000109B1F9C0E0D1F8B4105F46C1F3074161
:109D8000D846CDF814B0079100282AD9B6F900209A
:109D90004FF0000C06999344634600280ED9B1F9A0
:109DA0000040A51A002DB8BF151B7545B8BF0CF1B2
:109DB000010C01EB49015B1C8342F0D307998C45F0
:109DC00003D305997F1C1144059108F1010806EBA6
:109DD00049068045DAD3002FC4BF059991FBF7F1FE
:109DE00001DC9BFBF0F109B2039B05E07D41002003
:109DF00053454C46784100200A9A02EB4302918079
:109E0000FE4A1268B2F9BA30AAEB030399420ADD9E
:109E1000B2F9B82052448A4205DD019A11440191F9
:109E20000299491C02910099099A01EB40010091A5
:109E30000399491C0391914293D30299002906DDAD
:109E4000DDE9011291FBF2F1019103E0FFE75146D8
:109E5000CDF804A00A9AA2F886100021029103917D
:109E600004995031009100210491002869D9E349F7
:109E7000009F069709684FF0000B099EB1F9BCE0FE
:109E8000D1F8B410D846090ED946CDF814B00791D0
:109E9000002E2CD9B7F900204FF0000C06999344FE
:109EA0006346002E0ED9B1F90040A51A002DB8BFA7
:109EB000151B7545B8BF0CF1010C01EB40015B1C93
:109EC000B342F0D307998C4504D3059908F10108F2
:109ED0001144059109F1010907EB4007B145D9D3B8
:109EE000B8F1000FC4BF059991FBF8F101DC9BFBB1
:109EF000F6F1049B0A9A09B202EB4302A2F844105D
:109F0000BE4A1268B2F9BA30AAEB030399420ADDDD
:109F1000B2F9B82052448A4205DD039A11440391F4
:109F20000299491C02910099891C00910499491CCD
:109F3000049181429BD302980028C4BF039991FBEE
:109F4000F0FA0A98A0F888A001980A99504400B243
:109F500000EBD0704010A1F884000BB0BDE8F08F8A
:109F60002DE9F74F84B0A5490698DDE9044302685E
:109F70000546002000935063009B0968002B88BFB2
:109F800001262AD905EB4003B3F90430002BB4BFF6
:109F9000C3F1000C9C460FFA8CFCB1F9CC706745FC
:109FA00010DCB5F986C0BCF1000FB8BFCCF1000CD5
:109FB000002BB8BF5B42ACEB0303B1F9C6C01BB2C8
:109FC0009C4506DA536B06FA00FC43EA0C0CC2F817
:109FD00034C0009B401C9842D4D391F8CA30002B67
:109FE0007CD091F8CB00834288BF18460023DDF86F
:109FF00000C0BCF1000F84BF401C019074D94FF029
:10A00000010EDDF804C04FF000090120CA46BCF182
:10A01000010F4BD903FB0445B1F9CEC003950EFBEC
:10A020000445029503FB040602EB4605B5F9508092
:10A03000B8F1000FB4BFC8F100054546AC4535DBAB
:10A040000EFB040602EB4605B5F95060002EB4BFC6
:10A0500075423546AC4529DB039D2F1A02EB4705B7
:10A06000B5F94E50002DB4BF6F422F46BC451DDBE5
:10A07000029F3F1A02EB4707B7F94E70002FB4BF9B
:10A08000C7F1000BBB46E34510DCA6EB0808B1F9AD
:10A09000C8604645B8BF09F101097D1BB542C8BF7C
:10A0A0000AF1010A401C019DA842BBD3AAEB09009A
:10A0B0000028B8BFA9EB0A0091F8CAC0604507DBC9
:10A0C0000120D2F834C098404CEA000CC2F834C0E9
:10A0D00000985B1C834207D2002B00E004E018BF0D
:10A0E000A3F1010E8DD18AE7069C049D4FF0000C70
:10A0F00020686346002DC0F830C088BF012714D9FE
:10A1000004EB4306B6F94460002EB8BF764236B27F
:10A11000B1F9CC80B04505DD066B07FA03F846EAD5
:10A12000080606635B1CAB42EAD300236E1E002EBA
:10A1300084BFB1464FF0010A2DD904EB4305B5F9B0
:10A140004670B5F94460BD1B002DB8BFF51B2DB29C
:10A15000B1F9C480A8451ADAB4F98850A6EB05080D
:10A16000B8F1000FB8BFA5EB06080FFA88F87E1B00
:10A17000002EB8BFEE1B35B2A845056BAEBF0AFA7C
:10A1800003F65E1C0AFA06F645EA0605056303F1C6
:10A1900001034B45D1D3DDE9056500202B68002E76
:10A1A000C3F83CC088BF012714D905EB4004B1F9BE
:10A1B000D880B4F90A41A04503DCB1F9DA80A045A2
:10A1C00005DADC6B07FA00F844EA0804DC63401C9B
:10A1D000B042EAD3069D049E00202B68002EC3F8EF
:10A1E00038C088BF012718D905EB4004B1F9D880E1
:10A1F000B4F9CA41A04507DC02E000007841002024
:10A20000B1F9DA80A04505DA9C6B07FA00F844EA58
:10A2100008049C63401CB042E6D3DDE905650020DC
:10A220002B68002EC3F844C088BF012714D905EB62
:10A230004004B1F9DC80B4F94A41A04503DCB1F92E
:10A24000DE80A04505DA5C6C07FA00F844EA0804F1
:10A250005C64401CB042EAD3069D049E00202B683B
:10A26000002EC3F840C088BF012714D905EB400475
:10A27000B1F9DC80B4F90A42A04503DCB1F9DE8013
:10A28000A04505DA1C6C07FA00F844EA08041C64CF
:10A29000401CB042EAD3DDE90574049E2068002327
:10A2A000002FC0F84CC0C0F848C088BF4FF001086C
:10A2B00014D904EB4305B1F9E090B5F98A51A945E9
:10A2C00003DCB1F9E290A94505DAC56C08FA03F997
:10A2D00045EA0905C5645B1CBB42EAD30023002E96
:10A2E00088BF012714D904EB4305B1F9E080B5F923
:10A2F0004A52A84503DCB1F9E280A84505DA856C2D
:10A3000007FA03F845EA080585645B1CB342EAD303
:10A31000D2F83880106C30EA08031364916C43EA79
:10A32000080021EA00049464116B44EA000021EA69
:10A330000005156316D00021049E0846002E88BF34
:10A3400001260FD906FA00F73B4218BF491C401CF2
:10A35000049FB842F6D3012904D148EA0300C2F8A9
:10A3600040C0906324B1D06C002808BFC2F848C038
:10A37000D2F83C80506C30EA08035364D16C43EA55
:10A38000080021EA0004D464516B44EA000021EA89
:10A390000009C2F8349016D00021059E0846002E10
:10A3A00088BF01260FD906FA00F73B4218BF491CA7
:10A3B000401C059FB842F6D3012904D148EA0300A6
:10A3C000C2F844C0D06324B1906C002808BFC2F822
:10A3D0004CC01DB1106940F010001061B9F1000FC0
:10A3E00003D0106940F020001061906B18B1106923
:10A3F00040F040001061D06B18B1106940F080004F
:10A400001061106C18B1106940F480701061506CCC
:10A4100018B1106940F400701061906C18B11069A7
:10A4200040F480601061D06C18B1106940F4806015
:10A43000106107B00120BDE8F08F2DE9F04FB1B0F9
:10A4400016460D460446F6F733FFF6F738FA0100D4
:10A450004FF011001DBF029001200390012108BFA1
:10A46000CDE90210CDE91A54F7F77DF900220DF17C
:10A47000100B002D09D98356082BB4BF1433083BA9
:10A480000BF80230521CAA42F5D3F7F76EF90021FF
:10A49000002C07D9425C0BEB0103491C83F82020F8
:10A4A0008C42F7D8F7F7D0F82D900120F6F7DCFFB3
:10A4B000FE48007810F0200F4AD0F6F700FAFC4969
:10A4C00044F2A87244F23873096800280A44194417
:10A4D0000CBFCDE90012CDE9002106F18A001C90E5
:10A4E00040301D90FF210F20FAF799FBF6F7E0FEB0
:10A4F0000025E9460DF1700A1AA850F8257002A847
:10A5000050F82500F7F7ABFC0024002F88BF0BEBB9
:10A5100045181AD918F904001C2828BF00200DD2AC
:10A5200059F8251000EBD072521051F82210C007D4
:10A53000C00E21FA00F080B2F7F797FC5AF8251008
:10A5400021F81400641CBC42E4D36D1C022DD3D34B
:10A55000D648007810F0010F00F0A181F6F7AFF9AE
:10A56000D3490028096801F5C46201F584610CBF74
:10A57000CDE91C12CDE91C210120F6F76BFB3090D0
:10A580000120F6F7FFFD2E900298F6F7B1FB289018
:10A590000398F6F7ADFB279024A8009022AB20AAE1
:10A5A0001EA90298F6F748FD25A8009023AB21AA22
:10A5B0001FA90398F6F740FD0298F6F7B4FD269020
:10A5C0000298F6F7B0FDBB4D01902868B0F8E41092
:10A5D0000120F6F74EFB00210120F6F7BEFD2868AA
:10A5E00090F8E6100298F6F792FB286890F8E610CB
:10A5F0000398F6F78CFB2868B0F8E8100298F6F795
:10A6000048FD2868B0F8E8100398F6F742FD0020EE
:10A61000F6F7CAFD2F902868B0F8EC10009190F87A
:10A62000EB3090F8EA2001210298F6F7D2FC286876
:10A63000B0F8EC10009190F8EB3090F8EA2001218E
:10A640000398F6F7C6FC0020F6F7AEFD14ACF7F75A
:10A650001CF8FDF7A6F9012805D02046F7F790F978
:10A66000002800F02981F6F723FE179900221AAC82
:10A67000002054F822C0BCF1000F84BF02EB42035B
:10A6800006EB831308D931F8027B03EB4008401C2A
:10A69000A8F80A718445F6D8521C022AE8D3029819
:10A6A000F5F740FE2A900398F5F73CFE29900298B2
:10A6B000F6F79EFB2C900398F6F79AFB7D4D2B90B6
:10A6C0002868B0F8EE10009190F8EB3090F8EA208E
:10A6D00001210298F6F77DFC2868B0F8EE10009191
:10A6E00090F8EB3090F8EA2001210398F6F771FC1E
:10A6F00000250020F6F758FD00210298F5F7FDFD32
:10A7000000210398F5F7F9FD0DF10808012158F82B
:10A710002500F5F7F2FD1AA8002450F825701CA8B2
:10A72000002F50F825A032D904A800EB451905EBFD
:10A73000450006EB8018002119F804B00846F6F72A
:10A740004CFD012000FA0BF102A88B4650F82500C1
:10A75000F6F741FB6FEA0B010920F6F73EFD0DF11C
:10A76000500BF6F792FFFDF71CF9012804D058466C
:10A77000F7F706F900287CD0F6F79AFDBAF8000042
:10A7800008EB4401641CA1F84A01BC42D3D3002168
:10A790000846F6F722FD6D1C022DAAD32A990298CD
:10A7A000F5F7ABFD29990398F5F7A7FD2C990298C9
:10A7B000F6F711FB2B990398F6F70DFB3D4C20683B
:10A7C000B0F8F010009190F8EB3090F8EA200121F9
:10A7D0000298F6F7FEFB2068B0F8F010009190F8B0
:10A7E000EB3090F8EA2001210398F6F7F2FB012004
:10A7F000F6F7DAFC14ACF6F748FFFDF7D2F80128BB
:10A8000004D02046F7F7BCF800285BD0F6F750FDDF
:10A81000179900221AAC002054F822C0BCF1000F96
:10A8200084BF02EB420306EB831308D931F8025BC5
:10A8300003EB4007401CA7F88A518445F6D8521C08
:10A84000022AE8D301203099F6F713FA01202E9955
:10A85000F6F783FC28990298F6F759FA2799039896
:10A86000F6F755FA24980090229B209A1E99029898
:10A8700000E024E0F6F7ADFB25980090239B219A99
:10A880001F990398F6F7A5FB26990298F6F701FCA5
:10A8900001990398F6F7FDFB2F98F6F785FC2D98A4
:10A8A000F6F7E2FD31B0BDE8F08F00007D410020F9
:10A8B000A092010078410020F9F769FFC9E6F9F795
:10A8C00066FF50E7F9F763FF97E72DE9F04FADF624
:10A8D000844DFF224FF4066102A80AF0DCFBFF2240
:10A8E00040F20C410DF668000AF0D5FB02A8CDF845
:10A8F0006808FFF7A7F8FD4D4FF0000495F800A099
:10A900001AF0800F00F0C680DDF868080DF66802C6
:10A9100090F820C090F82110503001FB0CF300EBB0
:10A9200043000023002908D902EB430730F8026BEB
:10A930005B1CA7F88A609942F6D80023BCF1000F8F
:10A9400008D902EB430730F8026B5B1CA7F8CA601A
:10A950009C45F6D81668002396F82260002E0BD985
:10A9600002EB430730F8026BA7F88A6216685B1C9B
:10A9700096F822609E42F3D81668002396F823606A
:10A98000002E0BD902EB430730F8026BA7F8CA621E
:10A9900016685B1C96F823609E42F3D800230029BA
:10A9A00007D902EB430730F8026B5B1CBE8099426B
:10A9B000F7D80023BCF1000F08D902EB430730F8A9
:10A9C000026B5B1CA7F844609C45F6D830F8023B4C
:10A9D000A2F8863030F8023BA2F8883030F8023B0B
:10A9E000A2F8843000260023002988BF02EB8617D6
:10A9F00008D907EB430930F8028B5B1CA9F80A81E0
:10AA00009942F6D80023BCF1000F88BF02EB8617ED
:10AA100008D907EB430930F8028B5B1CA9F8CA81FF
:10AA20009C45F6D8761C032EDDD30026176800233C
:10AA300097F82270002F88BF02EB86170CD907EB1E
:10AA4000430930F8028BA9F80A83D2F800805B1C16
:10AA500098F822809845F2D81768002397F8237059
:10AA6000002F88BF02EB86170CD907EB430930F89B
:10AA7000028BA9F88A83D2F800805B1C98F82380A7
:10AA80009845F2D8761C022ED0D36046FFF726F9FF
:10AA9000012693E096480DF668080026006890F8B5
:10AAA000B40000F00F0700F07FFD012809D00F214E
:10AAB0003846F9F703FF012808D0002000F071FDA7
:10AAC0007CE000210846F6F7E2FC02E0012000F0FD
:10AAD00068FD884890F8009087480778002F18BFD5
:10AAE000B9F1000F68D0DDF868684FF4006106F135
:10AAF000500086F8209086F8217086F8224086F86B
:10AB000023400AF0BEFAF7F7E0F91AF0180F09D05F
:10AB10007A494246087886F82200497886F8231058
:10AB200000F09CFA1AF0210F04D0424639464846FC
:10AB3000FFF783FC1AF0030F3DD0BA46CDF804802E
:10AB4000F6F782FD06460220F6F78EFCFF210F2065
:10AB5000FAF765F8F6F7ACFB3046F6F785FCDDF85A
:10AB60006888002108F15000009053464A46084684
:10AB7000F7F7B2F80020F7F772F900260AFB09FB95
:10AB8000BBF1000F0AD908EB4607B7F85000F7F7FA
:10AB90006CF9761CA7F85000B345F4D858480078F3
:10ABA0001D2804BF08F15000FDF766F951464846DC
:10ABB000019AFFF793F80126F6F711FD9DF828009A
:10ABC0009DF82910CDF8740C002E12BF00280DF648
:10ABD000844DBDE8F08F002904BF0DF6844DBDE81B
:10ABE000F08F0020069041480078CDF87C0C10F0E2
:10ABF000020F00F0E9800020DDF8686847F6FF7A70
:10AC0000DDF8742C06F150086FEA0A090090054639
:10AC1000019000294AD936480068CDF8780C05FB28
:10AC200002F0012438F910304FF0000B1F46BC46EB
:10AC3000012A19D905FB024038F910006045C8BF48
:10AC400084469842B8BF0346A0EB070EBEF1000F42
:10AC5000B8BFA7EB000E0FFA8EF75F45C8BFBB4623
:10AC60000746641C9442E5D3CC45C8BFE146534532
:10AC7000B8BF9A46ACEB03000028B8BFA3EB0C00AA
:10AC800000B2DDF8783CB3F9C030834205DBDDF873
:10AC9000780CB0F9C200834505DD012000FA05F308
:10ACA0000198184301906D1C8D42B8D30025002AED
:10ACB00056D90F480068CDF8780C38F915300124C2
:10ACC0001F46BC464FF0000B012927D904FB025058
:10ACD00038F910006045C8BF84469842B8BF0346A3
:10ACE000A0EB070EBEF1000F0CE000007D4100203C
:10ACF000784100207E4000207F40002086400020D8
:10AD0000F9400020B8BFA7EB000E0FFA8EF75F45A1
:10AD1000C8BFBB460746641C8C42D7D3CC45C8BFCE
:10AD2000E1465345B8BF9A46ACEB03000028B8BFD4
:10AD3000A3EB0C0000B2DDF8783CB3F9BC308342E1
:10AD400005DBDDF8780CB0F9BE00834505DD012098
:10AD500000FA05F30098184300906D1C9542ACD39F
:10AD60000198F06218B1306940F008003061009835
:10AD7000B06218B1306940F004003061A6F824A038
:10AD8000A6F82690BDF9EC28A9EB02000028B8BF70
:10AD9000A2EB0900FE4A1368B3F9B820904203DD24
:10ADA000306940F002003061BDF9EC28A2EB0A00E6
:10ADB0000028B8BFAAEB0200B3F9BA20904203DD25
:10ADC000306940F001003061DDF87C0CF14C10F08E
:10ADD000010F05D00DF66802DDF8740CFFF7C0F81E
:10ADE0002078CDF8740C10F0080F7BD0DDF86838AF
:10ADF00000209DF82AA09DF82B90C3F85008024629
:10AE00008446E348CDE900A900680DF6680E1E46A9
:10AE100003F5056B5DF82C800021B8F1000F88BFA9
:10AE20000EEB8C1717D907EB4104B0F9D650B4F9E3
:10AE30008A42A54209D04FF00104D6F8505804FACE
:10AE400002F445EA0404CBF8004001F1010102F1EB
:10AE500001028845E7D80CF1010CBCF1020FD9D3EF
:10AE6000DEF80060002106F6540BC6F85418CDE950
:10AE700000A90A460C4600215DF82480B8F1000FB5
:10AE800088BF0EEBC41719D907EB410CB0F9D850A5
:10AE9000BCF90AC3654503DCB0F9DA50654509DA47
:10AEA0004FF0010CD6F854580CFA02FC45EA0C0C91
:10AEB000CBF800C0491C521C8845E5D8641C022C04
:10AEC000D9D3DEF80060002106F6580BC6F85818F2
:10AED000CDE900A90A460C4600215DF82480B8F1AE
:10AEE000000F00E062E088BF0EEBC41719D907EB32
:10AEF000410CB0F9DC50BCF94AC3654503DCB0F93C
:10AF0000DE50654509DA4FF0010CD6F858580CFAB6
:10AF100002FC45EA0C0CCBF800C0491C521C8845C9
:10AF2000E5D8641C022CD7D303F65407D3F8545841
:10AF3000D3F858083E1D30EA0502C3F85828D3F864
:10AF4000504842EA050124EA01080AEB090CC3F85B
:10AF5000508816D000210846BCF1000F88BF01249C
:10AF60000FD904FA00F912EA090F18BF491C401C56
:10AF70006045F6D3012904D145EA0200386000207B
:10AF80003060B8F1000F03D0186940F480301861C8
:10AF9000D3F8540818B1186940F400301861D3F898
:10AFA000580818B1186940F480201861DDF8740C55
:10AFB00010F0400F36D10798401C079006980028E3
:10AFC00014BF0998089800F1010014BF0990089077
:10AFD0000DF66800FEF7BAFD9DF82A0002A94000B0
:10AFE00004BF4FF4056004900020024605900498C9
:10AFF0008C46B0F5066F94BF03464FF406630020FD
:10B00000B0EB930F06D25CF82040401C2244B0EB1A
:10B01000930FF8D35042C8604FF42C304FF40662BF
:10B02000F7F7B1FA0A208DF800009DF818008DF8A6
:10B0300001009DF819008DF802009DF81A008DF8A6
:10B0400003009DF81B008DF80400052269460120CD
:10B0500000F00AFA0DF6844DBDE8F08F2DE9F04FAF
:10B06000A1B017460D460446F6F722F902221C92BB
:10B0700012221D92CDE90245F6F7E6FA199020203A
:10B08000F6F7F2F943480DF1380A4FF0010B00785A
:10B0900010F0180F44D0404844F6180201681144DB
:10B0A0000091006844F68801084401901C98F5F767
:10B0B0009FFE0E901D98F5F79BFE0F90FF210F202D
:10B0C000F9F7ADFDF6F7F4F8002502A850F8259041
:10B0D0001CA850F82500F6F7C2FE0024264607EB10
:10B0E000851816E05AF825000BFA04F108420FD033
:10B0F0005DF82500610850F82100E107C90EC8403D
:10B1000080B2F6F7B2FE08EB4601761CA1F88A027F
:10B11000641C4E4538BF1C2CE4D36D1C022DD4D3C7
:10B120001C48007810F0080F00F05E811A48016892
:10B1300001F51A610C91006800F52E600D90022057
:10B14000F5F788FD20900220F6F71CF81B901C985C
:10B15000F5F7CEFD16901D98F5F7CAFD17900AA8D1
:10B16000009006AB04AA08A91C98F5F765FF0BA888
:10B17000009007AB05AA09A91D98F5F75DFF1C987B
:10B18000F5F7D1FF1E901C98F5F7CDFF019005E073
:10B19000784100207D410020A09201000020F6F7B8
:10B1A00003F8964C1F902068B0F8E4100220F5F7E1
:10B1B00060FD00210220F5F7D0FF206890F8E6102E
:10B1C0001C98F5F7A4FD206890F8E6101D98F5F797
:10B1D0009EFD2068B0F8E8101C98F5F75AFF20682B
:10B1E000B0F8E8101D98F5F754FF2068B0F8EC109F
:10B1F000009190F8EB3090F8EA2001211C98F5F7C7
:10B20000E8FE2068B0F8EC10009190F8EB3090F870
:10B21000EA2001211D98F5F7DCFE0020F5F7C4FFB8
:10B2200010ADF6F732FAFCF7BCFB012804D0284633
:10B23000F6F7A6FB00285FD0F6F73AF8159900223A
:10B2400002AD002055F822C0BCF1000F88BF07EB0B
:10B25000C21308D931F8026B03EB4008401CA8F870
:10B260000A638445F6D8521C022AEAD31C98F5F7E3
:10B2700059F81A901D98F5F755F818901C98F5F79D
:10B28000B7FD0E901D98F5F7B3FD0F902068B0F84C
:10B29000EE10009190F8EB3090F8EA2001211C9814
:10B2A000F5F797FE2068B0F8EE10009190F8EB30BB
:10B2B00090F8EA2001211D98F5F78BFE0020F5F7A4
:10B2C00073FF002400211C98F5F717F800211D9842
:10B2D000F5F713F80DF17008012158F82400F5F77F
:10B2E0000CF802A8002550F824900CA82E4650F81F
:10B2F00024A007EBC41831E0F9F749FA93E70EA848
:10B3000050F82410012000FA05FB11EA0B0F24D09D
:10B3100000210846F5F761FF1CA8594650F82400A3
:10B32000F5F759FD6FEA0B010920F5F756FF0DF10E
:10B33000400BF6F7AAF9FCF734FB012804D0584675
:10B34000F6F71EFB002855D0F5F7B2FFBAF800005B
:10B3500008EB4601761CA1F84A036D1C4E4538BF28
:10B360001C2DCCD300210846F5F737FF641C022CB6
:10B37000A8D31A991C98F4F7C0FF18991D98F4F7F0
:10B38000BCFF0E991C98F5F726FD0F991D98F5F74F
:10B3900022FD02202099F5F76CFC02201B99F5F79D
:10B3A000DCFE16991C98F5F7B2FC17991D98F5F775
:10B3B000AEFC0A980090069B049A08991C98F5F731
:10B3C00008FE0B980090079B059A09991D98F5F7C0
:10B3D00000FE1E991C98F5F75CFE01991D98F5F783
:10B3E00058FE1F98F5F7E0FE1998F6F73DF821B0E2
:10B3F000BDE8F08FF9F7CBF99DE700007841002018
:10B400006549C2B2C0F307200A804880704762488D
:10B410004188008861F31F207047DFF87CC1012359
:10B420008340BCF800C013EA0C0F08BF704700B59A
:10B4300083B000F03F008DF800008DF801108DF80A
:10B440000220100A8DF80300100C8DF80400100E75
:10B450008DF8050000208DF806008DF8070068467D
:10B460000AF06AF803B000BDDFF82CC10123834065
:10B47000BCF800C013EA0C0F08BF704710B582B0CB
:10B4800000F03F008DF80000072A88BF0722002047
:10B490006B46002A09D911F800C01C18401C84F81A
:10B4A00001C09042F7D3072805D200211A18401C8A
:10B4B00051700728FAD318460AF03EF802B010BDC2
:10B4C000DFF8D4C001238340BCF802C013EA0C0F9C
:10B4D00008BF704710B582B000F03F0040F0800018
:10B4E0008DF80000072A88BF072200206B46002A3B
:10B4F00009D911F800C01C18401C84F801C0904202
:10B50000F7D3072805D200211A18401C51700728CC
:10B51000FAD318460AF010F802B010BD70B51E4DEF
:10B5200082B040EA0122AC880228234602D00528D6
:10B5300005D009E0002918BF022905D103E0002940
:10B5400018BF022900D11446A34204BF02B070BD47
:10B550000126F7F797FC297844EA004011F0080F1C
:10B5600017D003218DF800108DF801608DF80200CE
:10B57000010A8DF80310010C8DF80410000E8DF8EF
:10B58000050000208DF806008DF80700684609F0D8
:10B59000D3FFAC8002B070BD7E410020FE49087030
:10B5A0007047FD4948707047FB48407870472DE967
:10B5B000F04FF94991B000204870FCF7F2F90128EA
:10B5C00006D1F9F7ABF803281CBF11B0BDE8F08F26
:10B5D000F14C207810F0010F07D0FFF776F92078B2
:10B5E00020F001002070FCF7D8F9207810F0020F4D
:10B5F00000F0E281E948E84900684978B0F858006D
:10B600000229C0F303200DD0E34CA17801F00F0113
:10B61000F9F754F901280CBF02200020607005D012
:10B6200000F0B2B900210846F5F731FFF6F70CF843
:10B63000DFF864A30E909AF8020010F0100F18BF04
:10B64000F6F73EFCFF210F20F9F7E9FAD44800781D
:10B650000490D44800780590D34890F800B0D348BF
:10B6600000780D90059800281CBF0498002813D07E
:10B67000FDF73FFDFDF733FD0020F8F7D9FA002074
:10B68000F8F737FB9AF8020010F0100F0CD00120E9
:10B69000F8F77BFB01200BE00D98002818BFBBF1E9
:10B6A000000FE5D100F070B90020F8F76EFB002024
:10B6B000F8F76BFB0120F5F7B0FAF5F7CEFF1E2087
:10B6C000FCF730FB00210846FCF7C0FA8146012157
:10B6D0000020FCF7BBFADDE904128046002001FBE4
:10B6E00002F7002F84BFB24A510C06D929F8102066
:10B6F00028F81010401C8742F8D81E20FCF7B8FC30
:10B7000000210120FCF7A2FA054601210846FCF7BA
:10B710009DFA0D99044600200BEB0106002E84BF14
:10B72000A3494A0C06D925F8101024F81020401C13
:10B730008642F8D800200C909748808800287DD950
:10B74000701C40080F90FCF72CF9012876D006A851
:10B75000F6F716F9002872D00798002847D08E48CF
:10B76000807810F0100F0CD0DDF81CA0F8F726FA46
:10B77000059A0092524601461046049B0BF02CFCA1
:10B7800021E00020002300900190029003901A46CF
:10B79000194607980AF0C8FA82467F48807810F068
:10B7A000200F03D0FDF7A4FB824609E0F8F706FA64
:10B7B000059A0092524601461046049B0BF00CFC81
:10B7C000BAF1000F13D00020002F10D93AF9101051
:10B7D00039F910208A42B8BF29F8101038F9102022
:10B7E0008A42C8BF28F81010401C8742EED80E9835
:10B7F00010F0010F1CBF0A98002832D066488078EC
:10B8000010F0200F0AD0002211460A980AF049FDD4
:10B81000FDF771FB5FEA000A23D00BE0DDF828A0FA
:10B82000F8F747FA022200925246014610460F9B53
:10B830000BF0D2FB0020002E13D901E01FE016E030
:10B840003AF9101035F910208A42B8BF25F81010C7
:10B8500034F910208A42C8BF24F81010401C8642D8
:10B86000EBD8F6F7C3F80C98401C0C9002E0F8F700
:10B870008EFF0C98484989888842FFF464AFF5F739
:10B8800017FDFDF72CFCFDF735FC43490C98898822
:10B89000884273D30E9810F0020F26D000224FF684
:10B8A000FF731046002F0ED939F9101038F910C067
:10B8B000A1EB0C019142C8BF0A469942B8BF0B46A2
:10B8C000401C8742F0D80B208DF80000100A8DF83C
:10B8D00001008DF80220180A8DF803008DF804305D
:10B8E000052269460120FFF7BFFD0E9810F0010FF9
:10B8F00044D000224FF6FF731046002E0ED935F9C2
:10B90000101034F910C0A1EB0C019142C8BF0A46D7
:10B910009942B8BF0B46401C8642F0D80020BBF1CC
:10B92000000F84BF0D9901EB0B0615D9311A05EBF9
:10B93000410C04EB41013CF8027CABEB000C05EB45
:10B940004C0804EB4C0CA8F8667031F8021C401C43
:10B95000ACF866108345E9D80D208DF80000100A78
:10B960008DF801008DF80220180A8DF803008DF87B
:10B970000430052269460120FFF776FD3020FCF7F0
:10B98000D1F93020FCF774FBF5F729FE0248017865
:10B9900021F0020101700DE0844100207841002077
:10B9A0007E4000207F400020834000208440002013
:10B9B0000080FFFFFBF7F1FFF8F7B0FE03281CBF84
:10B9C00011B0BDE8F08FF8F7E2FEF6E504498870A3
:10B9D00070470348807870470149888070470000AD
:10B9E00084410020FE4982B26FF30F00C1E90602D4
:10B9F0007047FB4A0028D16914BF41F0020021F0D2
:10BA00000200D0617047F648007FC0F340007047E5
:10BA1000F34AF02303EA0010D16921F0F001084352
:10BA2000D0617047EE48007FC0F303107047EC4AC6
:10BA30000028D16914BF41F0010021F00100D0615C
:10BA40007047E748007F00F001007047E44B9969B8
:10BA5000C1F30362120721F07F4142EA006008430C
:10BA600098617047DE488069C0F303607047DC4826
:10BA70008069000F7047DB480068406DC0F30360C9
:10BA80007047012101FA00F04FF47F0101EA004103
:10BA9000D3488269114381617047012101FA00F0A6
:10BAA0004FF47F0101EA0041CD48826922EA010199
:10BAB00081617047CA488069C0F307407047C84831
:10BAC000008BC0F303307047C54910B50246886942
:10BAD0004FF47043C0F3033420F4704003EA0233A0
:10BAE0001843886103210846FFF797FC204610BDE4
:10BAF000BB48808BC0F38020704770B5B84E0446B9
:10BB0000C0F38000F569C5F30021884218BFF8F73B
:10BB10000AF814F0010F14BF45F0400025F0400072
:10BB200014F0040F14BF40F4807020F4807014F0FF
:10BB3000080F14BF40F4007020F4007014F0100FD0
:10BB400014BF40F4806020F4806014F0200F14BF14
:10BB500040F4006020F4006014F0800F14BF40F443
:10BB6000005020F40050F061BDE87040FDF70DBDBD
:10BB70009B48C169002011F0400F18BF012011F04F
:10BB8000200F18BF40F0020011F4807F18BF40F072
:10BB9000040011F4007F18BF40F0080011F4806F1A
:10BBA00018BF40F0100011F4006F18BF40F02000E3
:10BBB00011F4005F18BF40F0800070478848007F94
:10BBC000C0F3801070478648007FC0F34010704774
:10BBD0008348808BC0F3002070478148808BC0F37E
:10BBE00040207047FDF7EABA7D48808BC0F3C02043
:10BBF00070477B48808BC0F3003070477848C0693D
:10BC0000C0F3003129B1C0F34010002804BF012067
:10BC10007047002070477248808BC0F340307047F7
:10BC20006F490A6A1043086270476D49486270475D
:10BC30006B4890F8240000F001007047F0B587B021
:10BC40000446F8F76BFD0646F8F76BFD0746052E30
:10BC50000CBF654D654D6248007FC0F3031218BFED
:10BC6000052F05D1FFF7CAFF002818BF42F00202D6
:10BC700011462046F8F722FE002804BF07B0F0BDA9
:10BC8000FDF737FAF7F7EBFE0446F7F7FEF800206A
:10BC9000F4F7C3FFF5F7F9FCFBF783FE012809D0A1
:10BCA000F8F73CFDB04205D1F8F73BFDB84208BFBC
:10BCB000002C09D0F5F7FCFAFDF71CFAF8F76FFF36
:10BCC000F7F71FF907B0F0BD6846F5F759FE48B120
:10BCD0006846FCF7E8FB6846A847040008BFF5F78C
:10BCE000D4FCD9E7F8F748FDD6E7414870473C4A0D
:10BCF0005082918270472DE9F14F94B00024029454
:10BD00000394049405943B4806940794089409947A
:10BD10000A940B940C940D940E940F940778364863
:10BD2000DFF8D890DFF8C880067899F8000025463B
:10BD3000032804BF4046FCF79FF83B460096149A40
:10BD4000414610460BF048F92C480078062804BFFD
:10BD50001498FCF791F82248DFF88880808BC0F3B4
:10BD60000020002808BFCDE900070BD0D8F800005C
:10BD700090F83C11009190F83D0102282CBF801EE4
:10BD80000020019014984FF000090146002E88BF52
:10BD9000A24614D930F902CB0122012F09D930F97A
:10BDA000023B521CA3EB0C0C21F802CB9C469742A1
:10BDB000F5D809F1010921F802ABB145EAD34FF0FA
:10BDC000000A149BD1469C46CDF840A0002E84BFAB
:10BDD000781E119065D933F9028B002010E0000025
:10BDE0008C410020784100201D7A0100E984010087
:10BDF000808200207E4000207F400020F94000200B
:10BE000060F31F4460F30F041199012001293DD90B
:10BE100033F9027BA7EB08010AB22CF8022B002AA7
:10BE2000B8BF524211B222140FFA84F8129242445F
:10BE30000DF108080A4438F910808A459044B8BFCB
:10BE40008A46C145B8BFC146DFF844B4DBF800B04C
:10BE5000BBF93CE08E45C4BFBBF83EB0C34508DC2F
:10BE6000DDF80080404524BFDDF80480804545F1C1
:10BE70000005B846129F67F30F0461F31F4402A93F
:10BE800021F810201199401C8842C1D300202CF8C1
:10BE9000020B9B1C2CF8020B1098401C1090B04217
:10BEA00099D3FC48B0F90A105145B8BFA0F80AA0D0
:10BEB000B0F90C104945B8BFA0F80C90F6480078CE
:10BEC000012804BF1498FBF7D7FF284615B0BDE83A
:10BED000F08F2DE9F05F0446F048F1490026007824
:10BEE00009783746B3464518F7F7CCFB8146F7F794
:10BEF000E0FEDFF8A0A39AF8031000EB4108E94840
:10BF00000078032804BF4046FCF7CCF8B9F1000FD5
:10BF10007ED09AF8030009EB4009E2480078022835
:10BF200004BF4846FCF7BEF80020002D0CD939F8B4
:10BF3000101038F81020114434F81020511A24F849
:10BF40001010401C8542F2D8DFF8588398F80000A2
:10BF5000062804BF2046FCF7A5F80020691E00292A
:10BF600084BFBAF914C00B4613D904EB400134F86E
:10BF700010204988891A09B224F810100029B4BF8A
:10BF80004A420A466245BCBF0E447F1C401C984290
:10BF9000EBD3002FC8BF96FBF7F636B204EB45078C
:10BFA00027F8026C98F80000072804BF2046FCF729
:10BFB00079F800216A1E0846002A88BF13460FD967
:10BFC00034F81020921B12B224F81020002AB8BFB7
:10BFD000524212B29142B8BF1146401C9842EFD370
:10BFE00027F8021CBAF90E008142C8BFAAF80E1049
:10BFF000BAF91200814208DD98F800004FF0010BF9
:10C00000142804BF2046FCF74DF898F8000000E023
:10C0100007E0012804BF2046FCF744F85846BDE875
:10C02000F09F0020002D8FD934F8101038F8102020
:10C03000891A24F81010401C8542F5D884E72DE9B0
:10C04000F04F944E87B04FF0000A86F802A0FDF73B
:10C0500071F8DFF83CB2DBF80000B0F93610B0F947
:10C060003400FCF7F7FE042000F002F978B1307FCD
:10C07000C0F3401010B9FFF7C1FD40B9DBF8000074
:10C08000806DC0F303400F2818BFF7F730FD05207F
:10C0900000F0EEF858B1FFF7B1FD40B1DBF8000059
:10C0A000806DC0F303500F2818BFF7F720FDF8F795
:10C0B00035FB022808BFDFF8F08171D1B069C0F309
:10C0C0000364DBF80000A100806DC6F828A0C8401A
:10C0D000C6F82CA000F00F09C6F830A021460220B7
:10C0E000C6F834A0FFF71AFA062C40D2DFE804F0B5
:10C0F0005C0303036060B069C0F30364307F022C0B
:10C10000C0F303120ED011464846F8F7D7FB0028BB
:10C110002DD0FCF7EEFFFCF7E2FFF7F7A0FC0500DF
:10C1200009D022E0FFF76AFD002814BF42F00202A6
:10C1300022F00202E7E7F5F790FA86F800A0DFF8B0
:10C140006C915B4FFBF72DFC01280AD0F8F7E6FA5B
:10C15000022806D1B069C0F30360A04208BF002DD9
:10C1600006D0FCF7BCFFFCF7C5FFF8F718FD5DE053
:10C170006846F5F705FCA0B16846FCF794F96846F7
:10C180000AF0DAF9054699F8000030B1386880689D
:10C19000C8F800003868C0F800A0F5F727FCD1E720
:10C1A0004DE0F8F7F4FACDE748460AF05EFC3DE0D2
:10C1B000F8F7B4FA0546F8F7B4FA0746052D0CBFB0
:10C1C0003C4C3D4C307FC0F3031218BF052F05D106
:10C1D000FFF714FD002818BF42F00202114648463E
:10C1E000F8F76CFB10B3FCF784FFF7F738FC8146D7
:10C1F000F6F74BFE0020F4F710FDF5F746FAFBF7D3
:10C20000D0FB01280AD0F8F789FAA84206D1F8F73E
:10C2100088FAB84208BFB9F1000F17D0F5F748F80F
:10C22000FCF768FFF8F7BBFCF6F76BFEFBF7B9FB12
:10C23000012804D0F8F772FA02283FF43FAFF7F76D
:10C2400071FC07B0BDE8F04FFCF774BF6846F5F726
:10C2500097FB50B16846FCF726F96846A0475FEAAD
:10C26000000908BFF5F711FAC9E7F8F785FAC6E73C
:10C27000084A0228117F9269C1F30311C2F30742F1
:10C280001CD0012808BF11F0020F21D019E00000D6
:10C29000784100208C410020F9400020844000209B
:10C2A00083400020FE4000205C400020054000202C
:10C2B000689201001D7A0100E984010011F0040F69
:10C2C00006D0012101FA00F0104018BF012070478C
:10C2D00000207047334A30B4146894F86CC01CF0E6
:10C2E000040F1ABF012222EA0C050CF00105B0F977
:10C2F0000030B1F900201DB1E58AAA1A521E12B20F
:10C300001CF0020F03D0A48AE31A5B1E1BB21CF0C0
:10C31000040F19BF02800B8003800A8030BC704775
:10C320004FF6FF71A0F89C10A0F89E10A0F8A01086
:10C33000A0F8A21070472DE9F0470E46824603F0A0
:10C3400079FA074603F06CFA002500F13709002E50
:10C350008CBF4FF6FF78BDE8F08705EB051000EBCA
:10C36000451007EB800494F8BC0001280CD1A4F818
:10C370009C80A4F89E80A4F8A080A4F8A280224605
:10C380004946504601F052FA94F8C100022812BF03
:10C390000328204600F05CFD681CC5B2B542DCD322
:10C3A000BDE8F08718420020FE48DFF8FCC30268B1
:10C3B00092F87C00518A00FB01F3508BB3FBF0F341
:10C3C000CCF8043092F87D304B43B3FBF0F3CCF85B
:10C3D00008300B01B3FBF0F35B43CCF80C30C1EB3E
:10C3E000C103B3FBF0F301EB4101B1FBF0F05B43A0
:10C3F0004043CCE90430B2F87400C0F3033120208C
:10C40000062907D2DFE801F006030605090B102014
:10C4100000E04020ACF8000070478020FAE74FF4BD
:10C420008070F7E72DE9F04F85B09846DDE90E956D
:10C430000F46044603F0F4F9DB48AE464FF0000A1D
:10C440000688CDF80890C16801910069DFF85C9317
:10C45000009094F8C110A9F11502A9F10B0CA2F1FA
:10C460000A0002291CBF94F8A71002292BD094F8C7
:10C470008530CF4901EBC30151E90231B7F800B073
:10C48000CDF810B0B7F802B0CDF80CB0DDF804B0BC
:10C49000D8452DD394F8B8B0BBF1020F28D094F84A
:10C4A000858008F802A094F8858008F80CA094F81C
:10C4B000858018F800A0BAF1640F3CBF0AF1010AA8
:10C4C00008F800A034E094F885B03B8879880BF830
:10C4D00000A094F885B00BF802A094F885B00BF892
:10C4E0000CA094F885B009EB4B0B2BF8025CC5E768
:10C4F000DDF800B0D84594F8B88016D2B8F1020F34
:10C500002ED094F8858008F800A094F8858008F86B
:10C510000CA094F885A01AF80280B8F1640F3CBF13
:10C5200008F101080AF8028002E0B8F1020F17D002
:10C5300094F8858018F80220012A25D909EB4800D3
:10C5400030F8022CAA4288BF20F8025C94F88500DB
:10C5500009EB400232F8020CA8422CD33ED92FE05E
:10C5600094F8858008F800A094F8858008F802A067
:10C5700094F885A01AF80C80B8F1640F3CBF08F15C
:10C5800001080AF80C80D3D394F88520105C0128A8
:10C5900019D909EB420030F8022CAA4288BF20F8D2
:10C5A000025C94F88500DDF808C009EB400232F81F
:10C5B000020C604503D2304422F8020C0EE00DD983
:10C5C000A0EB0600F8E712F80C00012806D909EBE9
:10C5D000420232F8020C7045EDD3F1D894F885C0D0
:10C5E000049A09EB4C0030F8020CA0F5807505FBAD
:10C5F00003F303EB0222B2FBF0F205FB01F3039914
:10C6000003EB0121B1FBF0F0694901EBCC0343F8E6
:10C61000082C94F8853001EBC30141F8040CBA8072
:10C62000F88005B0BDE8F08F2DE9F84F6149624B05
:10C6300001444FF0000E01F801EC0344012103F81E
:10C64000011C5E49744601EB401100915C49724641
:10C6500001EB401B01F5A07101EB4019009800218E
:10C660000BEB041809EB041700EB0416002008EB91
:10C67000C10307EBC10C06EBC10503EB800A4AF8C6
:10C68000202C0CEB800A4AF8202C05EB800A401C79
:10C6900000B24AF8202C0228EFDB481C01B2022924
:10C6A000E4DB601C04B2022CD8DB3E48454E00217E
:10C6B000D0F800C0A6F110070BEB0E1809EB0E1A0C
:10C6C000002006EBC10908EBC1050AEBC10407EB2A
:10C6D000C103814207D1BCF87A2043F82020BCF87E
:10C6E000782049F8202053F8202005EB800B02EB3E
:10C6F000820252004BF8202C04EB800B401C00B24D
:10C700004BF8202C0228E4DB481C01B20229D7DBBD
:10C71000BDE8F88F10B490F885C02B4C00230CF8BE
:10C72000043090F885C00A340CF804301D4B90F8A2
:10C7300085C01B6893F87430C3F303131B021534D0
:10C7400004EB4C0C2CF8023C90F885C0A4F16E036D
:10C7500003EBCC0C4CF8081C90F8851003EBC101DE
:10C7600041F8042C90F8850010BC5DE770B50446D4
:10C7700003F075F802460C4894F8C110406802298D
:10C7800000FB00FC114828D00649096891F8701098
:10C7900011F0100F2AD094F88520A0F1AB0101EB25
:10C7A000820115E018420020C8410020E2840020E8
:10C7B00074840020C0880020CA8800208087002060
:10C7C00000850020F0410020C3840020F584002073
:10C7D00031F8042C31F8021C14E094F88550B4F8B8
:10C7E000A020B4F8A210C8232B540BE094F88610B4
:10C7F00001EB011303EB411102EB8101B1F8A02021
:10C80000B1F8A210B4F8A030B4F8A2509B1A03FB00
:10C8100003F66B1A03FB0363634510DA94F8853063
:10C8200013F800C0BCF10F0F84BFA4F8A020A4F837
:10C83000A210195CC8293CBF491C195470BD0021C5
:10C8400094F88520115470BD2DE9F041044603F0A1
:10C8500006F80146FD48DFF8F8C380680CF10B07C5
:10C8600000FB00F694F8C100022844D094F886003A
:10C8700000EB001202EB401001EB8000B0F8A010BA
:10C88000B0F8A200B4F8A030B4F8A2205D1A05FBFD
:10C8900005F8151A05FB0585B5420ADA94F88550A6
:10C8A00015F80C50012D04BFA4F8A010A4F8A200A4
:10C8B00013D094F8855007EB850636F8048CA3EB6B
:10C8C00008084144A4F8A01036F8021C511A084484
:10C8D000A4F8A200002005F80C0094F8850007EBEE
:10C8E000800020F8043C94F8850007EB800020F8D5
:10C8F000022CBDE8F08194F88520B4F8A01007EB75
:10C900008202B4F8A20022F8041C94F8852007EBF8
:10C91000820222F8020C94F88530012203F80C20E0
:10C92000B0E72DE9F04F90F885C08FB04FF48063E9
:10C9300000290CBFC74CC84C04EB4C14C74D0292E5
:10C9400005EB4C1705F5A5756544A4F1200415F811
:10C95000016C07EB061505EBC10858F8205CA2EB4B
:10C960000502039290F8C120022A1CBF90F8A7008C
:10C97000022800F00A8158F81C8C04EB061205EB23
:10C980000809CDF83090D2F80490D6689568106800
:10C9900009EB0602DFF8C89228441044D9F800A039
:10C9A00035445044D9F804A0DFF8B8B25244D9F85D
:10C9B00008A0D9F80C9055444E44DDF808A0DDF8E5
:10C9C0003090AAEB0909CDF82090DDF80C90A9EB86
:10C9D0000809CDF82C90DBF8009009EB000ACDF89F
:10C9E00028A0DBF8049009EB020ADBF80890DBF8DA
:10C9F0000CB0A9440BEB060EDDF828B00BFB0EFBC8
:10CA00000AFB19BB9BFBF3FB4FEA8E2E9EFBFBFE42
:10CA10004FEA8A2A9AFBFBFACDF838E0CAF1000EF9
:10CA2000DDF828A04FEA892999FBFBF94FEA8A2A09
:10CA30009AFBFBFACDF834E0DDF838E0C9F10009E3
:10CA400000FB0EFB02FB09BB9BFBF3FBDDF834E0B4
:10CA5000CDF828B000FB0EFB02FB0ABB9BFBF3FBEF
:10CA6000CDF824B0DDF838E005FB0EFB06FB09B974
:10CA700099FBF3FBDDF834E0CDF838B005FB0EF997
:10CA800006FB0A9999FBF3FADDF828B0DDF820904F
:10CA90000BFB09FEDDF824B0DDF82C900BFB09EE52
:10CAA000DDF838B0DDF820909EFBF3FE0BFB09FBB0
:10CAB000DDF82C900AFB09BBDDF83090CAF5806ADE
:10CAC000F144CDF800909BFBF3F9C844DDF828B0A1
:10CAD000CDF80480CBF58068DDF824B0CBF10009F7
:10CAE000DDF838B0CBF1000E08FB00FB09FB05BBFD
:10CAF00008FB02F80EFB00F009FB06880AFB0500A4
:10CB00009BFBF3FB98FBF3F890FBF3F0CDF810B030
:10CB1000CDE905800EFB02F00AFB060090FBF3F066
:10CB2000079051480022E84604AE00EB0C0358F889
:10CB3000220013F8015C07EB051505EBC10505EBB9
:10CB4000820545F8200C002006EBC20513F801AC65
:10CB500055F8209004EB0A1A0AEBC20A4AF8209012
:10CB6000401C00B20228F1DB501C02B2022ADEDBBC
:10CB70003D48604410F8010C07EB001000EBC100C9
:10CB800050F8200C0FB0BDE8F08F374A0020624407
:10CB9000039012F8012C02AB07EB021202EBC10268
:10CBA00053F8204002EB8005401C00B245F8204CB1
:10CBB0000228F5DBDCE70288438862F30F018088F6
:10CBC00063F31F419A4284BF63F30F0162F31F4175
:10CBD0000A0C824288BF60F31F4188B20A0C90425F
:10CBE00084BF62F30F0160F31F41080C704770B5FA
:10CBF0000146154691F8C1601C4B91F8851090F8DC
:10CC000085202C88688801EB4101A3F1780C0CEB9E
:10CC1000810C022E2CD03CF80A1C2CF8081C3CF885
:10CC20000C1C2CF80A1C2CF80C4C3CF8041C2CF89E
:10CC3000021C3CF8061C2CF8041C99182CF8060C55
:10CC400011F8011C012924D02CE00000C84100206B
:10CC50003F8400200085002040860020808700203F
:10CC6000E0410020F0410020C08800204C890020D5
:10CC70002CF8084C2CF80A4C2CF80C4C2CF8020C14
:10CC80002CF8040C1A442CF8060C012102F8011CA3
:10CC900008E0ACF10C00FFF78EFF0446ACF1060093
:10CCA000FFF789FFAC80E88070BD30B44FF0000C16
:10CCB00088B0634601EB001101EB430030F8100C23
:10CCC0008444581C83B2082BF6D300234FEADC05BA
:10CCD00018466C4601EB400C3CF810CCACEB050C54
:10CCE0000CFB0CFC44F820C0401C80B263440828B4
:10CCF000F0D3D80831F80A3C31F8101C591A4943CE
:10CD0000116008B030BC70472DE9F041044690F83E
:10CD1000855090F8C1C0DB4882B04FF00008BCF1EC
:10CD2000020F07D100EB050C0CF8018C81F8B880DC
:10CD300084F8B8802844D44F10F801CC07EB0516CE
:10CD400006EB4C0626F8102C0CF10102D2B2A6F824
:10CD5000903000F8012C082A09D300F8018C91F8D2
:10CD6000B800002804BF012081F8B80008E091F85D
:10CD7000B800002802BF84F8B88002B0BDE8F08196
:10CD80006A46C1492846FFF790FF064601AA07F107
:10CD9000A0012846FFF789FF0146BC48406986424A
:10CDA00096BF81420320022084F8B80002B0BDE89B
:10CDB000F081B0F89C30B1F89CC0A3EB0C02002AC3
:10CDC000B8BFACEB0302B0F89E30B1F89E10581A11
:10CDD0000028B8BFC81A02FB02F100FB0010704720
:10CDE00070B50D46044602F01BFD94F8C100A84E34
:10CDF00002281DBF94F8A7000228012DB4F8A00056
:10CE00000FBFB4F8A22094F8850006EBC00151E9E9
:10CE1000020232213125B4F8A0C0B4F8A23005FBDB
:10CE200000C0B0FBF1F005FB0232B2FBF1F194F867
:10CE3000852006EBC20242F8080C94F8852006EB28
:10CE4000C20242F8041CA4F8A000A4F8A21070BD0D
:10CE50002DE9F04F85B0044600F028F9054602F0B0
:10CE6000FEFC834602F0DCFC8A4A0646007B116821
:10CE700080B1086FC0F34043C0F3C04AC0F38040A4
:10CE800004930090486FC0F303414FEA0129C0F3B7
:10CE9000035013E091F87000C0F34003C0F3C00AE0
:10CEA000C0F3800004930090307D012809D091F8F0
:10CEB000740001074FEA1159C0F303104FEA00282C
:10CEC00006E0B1F87400C0F303204FEA0029C84619
:10CED0007048006890F8700010F0010F00F0C680F4
:10CEE00094F8857094F88600B4F89C10ADF808109A
:10CEF000B4F89E10ADF80A1000EB001101EB4010E1
:10CF00000BEB800B02AA59462046FFF770FEBAF1E0
:10CF1000010F70D060490020394401F8010C94F8E9
:10CF2000C100022819BF94F8A70002283846FFF76D
:10CF30007BFBBDF8082000212046FFF7F2FC82466B
:10CF4000BDF80A2001212046FFF7EBFCAA45B8BF37
:10CF5000AA46A842B8BF28464E4B1968B1F910201E
:10CF6000521BA2F1010CD445B8BFE246B1F9121030
:10CF7000491B4A1E8242B8BF10461FFA8AF283B28A
:10CF80004648ADF80C20C1190A30ADF80E303844CF
:10CF900011F801CC10F8015C01F8015C00F801CC3B
:10CFA0000098012804BFADF80820ADF80A305946B2
:10CFB0002046FFF7A9FEB4F89C00BBF89C20811A1C
:10CFC0000029B8BF111AB4F89E30BBF89E20981AF9
:10CFD0000028B8BFD01A494300FB0013CDE90098E0
:10CFE00096F82A2002A92046FFF71CFA0498012887
:10CFF00012D109E0FFE7BDF80C00ADF80800BDF85C
:10D000000E00ADF80A008AE7BDF80C00ADF8080084
:10D01000BDF80E00ADF80A00BDF80800A4F8A000A5
:10D020001C4DBDF80A00A4F8A200286890F8700012
:10D0300010F0200F09D01A48384410F8010C20B91C
:10D0400096F82A102046FFF791FB286890F87000A8
:10D0500010F0100F04BF05B0BDE8F08F96F82A104D
:10D060002046FFF7F1FB05B0BDE8F08FB4F89C0057
:10D07000A4F8A000B4F89E00A4F8A20005B0BDE892
:10D08000F08F0000968A002056890020C8410020B9
:10D09000A08A0020184200204C890020C08800206F
:10D0A00040840020FE487047FE487047FE480078E4
:10D0B00070470346002002460029D8BF704753F846
:10D0C00022C0521C60449142F9DC70472DE9F047C0
:10D0D0000D46074602F0D2FB044602F0CBFBF249B4
:10D0E000DFF8C0834E78290291FBF0FC390291FBF6
:10D0F000F4F35D1200214FEA6C27002CC8BFDFF863
:10D10000AC930BDD01FB03F205EB222248F8212052
:10D1100049F82120491C09B28C42F3DC0021E04D82
:10D120000028C8BFDFF888930BDD01FB0CF207EB8A
:10D13000222245F8212049F82120491C09B28842C1
:10D14000F3DC03FB06F2D8F8003012139B1AC8F880
:10D15000003008EB84030CFB06F153F804CC0913F0
:10D16000624443F8042C2A6805EB8000521A2A60B6
:10D1700050F8042C114440F8041CBDE8F087CD4958
:10D1800030B40B68C84A1428B3F812C0198A28BFF3
:10D19000082411D2A0F10F050924052D0CD36D1D13
:10D1A000052D38BF0A2407D3451F052D38BF0B2492
:10D1B00002D3052838BF0C2454705B8B0CFB00F0A5
:10D1C000B0FBF3F0107030BC60467FE7B94810B593
:10D1D000026892F86C30508A118ADB08528B434304
:10D1E000B3FBF2F2B04B1A7009225A70FFF76EFFD0
:10D1F000B14900204FF6FF7221F8202001EB800397
:10D20000401C80B25A800A28F6D310BD2DE9F04F99
:10D21000B3B00D460446CC22A849684607F02CFF5F
:10D22000A448B5F902200068012A90F807C090F8D8
:10D230000680478A068A687800FB0CF109B2D8BFDD
:10D2400001222B78DFF878E2EB4683B1ACF10109DB
:10D250004B45194417D104EB410131F9021C012956
:10D26000D8BF0121C902494291FBF2F140E004EB31
:10D270004101B1F902100129D8BF0121C90291FB76
:10D28000F2F109B235E004EB410939F9021C012938
:10D29000D8BF0121B9F90290B9F1010FD8BF4FF001
:10D2A00001094FF0640A01FB0AF109FB0AF901EBDD
:10D2B000620109EB620991FBF2F199FBF2F93BF98A
:10D2C00011103BF91990494508BF002111D001EB1D
:10D2D000090A1AF5004FB8BFF24604DBBAF5004F51
:10D2E000A8BF47F6FF7AA1EB0901C90291FBFAF149
:10D2F00009B2A0B1A8F101094845A0F1010909FB53
:10D300000CF90FFA89F9994415D134F91940012C17
:10D31000D8BF0124E402644294FBF2F246E003EB3E
:10D320000C0934F91940012CD8BF0124E40294FB04
:10D33000F2F212B23BE034F91990B9F1010FD8BF03
:10D340004FF0010900F1010A0AFB0CFA0FFA8AFA00
:10D350009A4434F91AA0BAF1010FD8BF4FF0010A6C
:10D36000642409FB04F404EB620494FBF2F44FF030
:10D3700064090AFB09F909EB620999FBF2F23BF92E
:10D3800014403BF91220944208BF00220FD004EB56
:10D39000020919F5004F05DBB9F5004FB4BFCE46C1
:10D3A00047F6FF7EA21AD20292FBFEF212B21B04D3
:10D3B000000403EB011100EB021201F5004002F53D
:10D3C000004190FBFCF091FBF8F1704379430014AD
:10D3D00009140028B4BF00220246B242C8BF30463A
:10D3E00002DC0028B8BF00200029B4BF00220A4692
:10D3F000BA42C8BF394602DC0029B8BF0021A5F8EF
:10D400009C00A5F89E1033B0BDE8F08F2DE9F74FD2
:10D41000ADF5007D0F4614467021684607F031FED9
:10D4200070211CA807F02DFE702138A807F029FEF6
:10D43000702154A807F025FE02F011FA05461A489B
:10D4400090F8008002F0ECF97D9002F0FCF9709009
:10D450003730739002F016FA789016480068418AC7
:10D460007B91008A7C9002F005FA064602F006FAEB
:10D4700082460C487A90703879902078617894F8D8
:10D48000853001FB060094F88610385C01EB011230
:10D4900002EB411105EB810200F03F00064911E06B
:10D4A000F08A0020608B002000420020408C002089
:10D4B000D08B002018420020B08C002088950100FD
:10D4C0000080FFFF01EB830C3CF8045CA5F57F4175
:10D4D000FF3907D03CF8023CA3F57F41FF3918BF64
:10D4E000294601D19188D388B4F804B0CDF8C8B1E9
:10D4F000DFF83C930BF1050BA9FB0BEBCBF3CF0B48
:10D50000CDF8DCB1B4F806B0CDF8C4B10BF1050B21
:10D51000A9FB0BEBCBF3CF0BCDF8F8B101F1050B69
:10D52000A9FB0BEBCBF3CF0E03F1050BA9FB0BB95A
:10D53000CDF8D4E1DDF8C8B14CF6CD4E0BFB0EFBB7
:10D540004FEADB4BCDF8D8B1DDF8C4B1C9F3CF0950
:10D550000BFB0EFB4FEADB4BCDF8D0B101FB0EFB12
:10D560004FEADB4BCDF8C8B103FB0EFB4FEADB4BB8
:10D57000CDF8C4B1DDF8D4E1DDF8DCB1F34504BF8A
:10D58000DDF8F8B1CB450BD0DDF8C8B1DDF8D891A6
:10D59000D94518D1DDF8C4B1DDF8D091D94512D103
:10D5A000DDF8F49199F82A90B9F1020F0BD3DDF868
:10D5B000C0B19BF82AB0CB4504BF94F88490B9F170
:10D5C000020F00F0D3804FF6FF712CF8041C994A2B
:10D5D00094F8853002EB830222F8021CA17A719143
:10D5E000E17A7091257B617B709B0DF1700B8B4212
:10D5F0002AD803FB06F292B27292719AAA421FD8FD
:10D60000DDF8C8C10CEB0209DDF800C23CF919C015
:10D6100017F8099009F03F0981450DD1DDF8E09137
:10D62000CC4509DB5DF822E0E6444DF822E05BF8EA
:10D630002390CC444BF823C0521C92B2AA42DFD9AB
:10D640005A1C93B28B42D4D900216A460846002E58
:10D6500040F3E78052F82030401C1944B042F9DB17
:10D66000002940F3DE8000215A460846BAF1000F37
:10D6700040F3D78052F82030401C19448245F9DC31
:10D68000002940F3CE800020002E84BF694638AACE
:10D690000CD9799B51F820C053F820300CFB03F3D0
:10D6A00042F82030401C80B28642F2D80020BAF105
:10D6B000000F88BF54A90BD97A9A5BF8203052F832
:10D6C00020205A4341F82020401C80B28245F3D8E4
:10D6D000002138AA0846002E05DD52F82030401CF3
:10D6E00019448642F9DC00226B461046002E05DD07
:10D6F00053F820C0401C62448642F9DC91FBF2FCE6
:10D70000002154AA0846BAF1000F05DD52F8203076
:10D71000401C19448245F9DC00225B461046BAF1F0
:10D72000000F05DD53F82050401C2A448245F9DCE7
:10D7300091FBF2F0C445B8BFC4464045B8BF40466F
:10D740007C99A1EB08014A1E6245B8BF94467B99BB
:10D75000A1EB08014A1E8242B8BF1046A4F89CC043
:10D76000A4F89E000DF5037DBDE8F08FDFF8C490AE
:10D770004FF6FF7B5D4504BF3CF8025C5D4507D179
:10D780002CF8041C94F8851009EB810121F8023C67
:10D79000917AA37A994238BFA172D17AE37A9942F9
:10D7A00038BFE172117B237B994288BF2173517B83
:10D7B000637B994288BF6173A17A719194F80B9051
:10D7C000CDF8C09113785278617B02FB0633739ACF
:10D7D000257B8945D25C02F03F0B3FF605AF09FB84
:10D7E00006F292B27292719AAA4213D8729BDDF835
:10D7F000CCC113441CF803C00CF03F0EDE4505D12C
:10D800002CF03F0C4CEA000C07F803C0521C92B2FB
:10D81000AA42EBD909F101021FFA82F98945DED942
:10D82000E2E60020A4F89C009AE7EFE5EEE50000B0
:10D83000CDCCCCCCB08C002070B514460D4606463D
:10D8400002F018F88446D5E9040101EB8101430098
:10D850008900AA69B1FBF3F102EB82008000B0FB02
:10D86000F3F202FB0C102180628036F81000A080D9
:10D8700070BD2DE9F0410446DDE90606089F0D461E
:10D8800000281CBF002081F8210002D00020BDE844
:10D89000F081286820606868C4F80A001068606039
:10D8A000908820817022194604F1140007F0E4FBEF
:10D8B000A868C4F80E002869A061A889A082A88B76
:10D8C000A4F8700095F8200084F8BD0095F82200B7
:10D8D00084F8BE00012084F8BC0084F8BF70307862
:10D8E000401CC0B230700D2828BF0120CED3BDE847
:10D8F000F0812DE9FF5F1F461646054601F090FFB7
:10D90000B0F902004FEAE00A01F0C1FF504502DD24
:10D9100001F0BDFF82460022934690469146304674
:10D92000BE4221DCB0420CBF0146411ECBB2B84220
:10D930000CBF0146411C01F0FF0C08F101011FFA68
:10D9400081F835F9101051450ADD49B135F9133028
:10D950009942A4BF35F91C30994201DB82B203E041
:10D96000401C00B28742DDDA3C46B74220DB0CBFE8
:10D970002046601EC1B2BC420CBF2046601CC3B230
:10D9800009F101001FFA80F935F9140050450BDD4B
:10D9900050B135F911108842A4BF35F913108842EF
:10D9A00002DB1FFA84FB03E0601E04B2B442DEDA3D
:10D9B00093450DD04FEA48022946019807F066FBCF
:10D9C00001984FEA490205EB4B0100EB480004E0E7
:10D9D000B81B4000821C2946019807F057FB08EB52
:10D9E000090004B080B2BDE8F09F2DE9F0479CB07B
:10D9F000844624988A464FF00008017840784446CF
:10DA0000CDF80080CDF80480CDF80880CDF80C80EA
:10DA1000CDF81080CDF81480CDF81880CDF81C809A
:10DA2000CDF82080CDF82480CDF82880CDF82C804A
:10DA3000CDF830804FEA8109CDF83480CDF83880B8
:10DA40001094119414941F46860012941394159404
:10DA500016941994179418941A944B4622466946C2
:10DA60006046CDF83C801B94FFF743FF05463346E4
:10DA700022460EA95046FFF73CFF0446002109F15B
:10DA80000200854215DC0020002DC8BFE94610DDEC
:10DA900009EB400239F91030B2F902C0ACEB0302D5
:10DAA000002AB8BFA3EB0C021144401C00B2A842EC
:10DAB000EEDBA6EB08000022801CA042A4BF0020E1
:10DAC000002CC8BF0DF1380810DD08EB400338F911
:10DAD00010C0B3F90260A6EB0C03002BB8BFACEB8F
:10DAE00006031A44401C00B2A042EEDB88009100FD
:10DAF000B0FBF5F0B1FBF4F10844C0F34F003884FB
:10DB00001CB0BDE8F0877047704770470028DCBF45
:10DB1000002070474FF480714FEA002C00200B1258
:10DB20009CFBF3F30A46991801EBD1714910531A83
:10DB3000002BB8BF8B1A802B02DB401C6428EED36D
:10DB4000081270472DE9FF4F85B01F4616460D4657
:10DB5000002401F08FFE0190B6F900E0B6F9020052
:10DB60000290287903906A79E87995F806A0A4468E
:10DB7000654666460090824229DC0398504521DCC8
:10DB8000029902EB8203C1EB430303FB03FB019900
:10DB900002FB0108059931F918100A290EDD00EB86
:10DBA0008008CEEB480808FB08F903FB08F809FBDE
:10DBB00001CC0BFB015508FB01660C44401C00B274
:10DBC0005045E4DD501C02B200988242D5DDDFF8FA
:10DBD000308B88FB0C104111A1EBE07188FB052014
:10DBE0004211A2EBE07288FB06304311A3EBE07018
:10DBF0000902120291FBF4F192FBF4F2000290FB95
:10DC0000F4F001FB02F300FB103004128818C0F19D
:10DC1000000CA0000CFB0CF1C0EB21200012410015
:10DC20000029D8BF002015DD0D024FF480700021BF
:10DC3000031295FBF3F30246981800EBD0704010E6
:10DC4000131A002BB8BF831A802B02DB491C6429EE
:10DC5000EED30012000200EBD071CCEB61000CEBB4
:10DC6000610149427C610028B8BF4042F860002948
:10DC7000B8BF494200EB8002520088FB0232D31049
:10DC8000A3EBE2733961FF2BC8BFFF234211481198
:10DC9000FF2A88BFFF22FF2888BFFF2087F86C304B
:10DCA00087F86D2087F86E0009B0BDE8F08F2DE988
:10DCB000F04117460C46064601F0DCFD054601F032
:10DCC000DDFD844623786078002BCCBF591E0021EF
:10DCD0000AB2691E8B42B8BF591C0CB20028CCBFD7
:10DCE000411E00210BB2ACF101018842B4BF401CBF
:10DCF000084600B24FF0000C83420FDC1146A242EE
:10DD000008DC03FB0518491C36F9188009B2C44425
:10DD1000A142F6DD591C0BB28342EFDDC7F81CC0EF
:10DD2000BDE8F081CA69002A12DBB0F902204B6914
:10DD300093FBF2F00028B8BF404240F2DC5383422C
:10DD400006DB886990FBF2F00528DCBF00207047F5
:10DD5000012070472DE9F007A0F1020ADDE90A541D
:10DD6000DDE90896079F4FF0000804EB400C8A4558
:10DD7000B2BFA3F800803CF804ACA3F800A0431E97
:10DD80008B42B2BFA7F800803CF8021C398034F8FF
:10DD90001010A9F80010411C91428EBFA6F8008017
:10DDA000BCF802103180801C90428EBFA5F8008024
:10DDB000BCF804002880BDE8F00770472DE9F001A9
:10DDC0008A1ADDE90847DDE90565DDF81CC09942DE
:10DDD00002BF20F832C0BDE8F0017047AB1BACEBCE
:10DDE0000501A4EB0C05CB1A2EB2711A01EB41010F
:10DDF0003C1B49000FB203EB4303A11B5B0001EB8B
:10DE000041011DB249000BB2794205EB8101C3EB20
:10DE1000031421448C00002CC8BF41F38F1104DC93
:10DE2000890049420912494209B24C4203EB84037A
:10DE30001DB24B1B002B03DD2B2463431B1205E09B
:10DE40006FF02A0463431B125B421BB26C1001EBA0
:10DE500045012B256943A6EB21210DB29E0000212F
:10DE60005F0106EB041607EB84174FF06C0803FB09
:10DE700008F304EBC40403EB041305EB450406EBC1
:10DE8000851607EBC51703EB841306EB0C2607EB8F
:10DE90000C2703EB0C2346F30F2647F30F2743F31E
:10DEA0000F2400EBC20320F832C05E80491C9F8023
:10DEB00089B2DC800429F4D3BDE8F00170472DE974
:10DEC000FF4F03F1010885B01E46154681461146F5
:10DED000424532BF002709B0BDE8F08FB246881E28
:10DEE000A842B2BF3B4609EB410030F9043C4A1E50
:10DEF000AA42B2BF3A4609EB410030F9022C39F987
:10DF000011C04C1C54458EBF384609EB4100B0F996
:10DF1000020001F1020BB3458EBFBA4609EB410A7C
:10DF2000BAF904A00FFA8AFA00B2CDF808C0CDE918
:10DF3000030A18B212B2CDE9000233462A46069807
:10DF4000FFF73CFFA1B24145C8D309B0BDE8F08F4F
:10DF500030B48278037890F803C04478D21AACEBDE
:10DF6000040C0B70D2B20CF0FF0483784FF0000C5D
:10DF70008B70052A26D209E023B38D7883F0010344
:10DF80006D1E8D70521ED2B2052AF5D242784A70AB
:10DF9000C078C870052C3CBF30BC7047BCF1000F86
:10DFA00001BF4878401C48704FF0010C1FBFC87873
:10DFB000401EC8708CF0010C601EC4B2052CEDD25E
:10DFC00030BC70470B785B1C0B700123DAE72DE93E
:10DFD000FF4FF5B01C46DDE98295074601F04EFC87
:10DFE000064601F047FC804670A909F10400FFF7DE
:10DFF000AFFF9DF8C001002818BF401EC0B28DF8C9
:10E00000C0019DF8C211A8F1010291420CBF114656
:10E01000491CCAB28DF8C2219DF8C111002918BF50
:10E02000491E8DF8C1119DF8C311731E99420CBF92
:10E030001946491C8DF8C311101A20709DF8C301B0
:10E040009DF8C111E946401A607028789DF8C0110A
:10E050009DF8C141401AC6B2A878B5F90450001B1A
:10E0600000F0FF089DF8C301A04224BF4FF0000A52
:10E07000DFF890B639D3CDF888A1CDF88CA1CDF8D2
:10E0800090A1CDF894A1CDF898A1CDF89CA1CDF8A0
:10E09000A0A1CDF8A4A1CDF8A8A1CDF8ACA1CDF850
:10E0A000B0A1CDF8B4A1CDF8B8A1CDF8BCA1DBF8F2
:10E0B00000009DF8C2319DF8C021C07962A960437B
:10E0C00007EB4000FFF7FBFE9DF8C1013822201A44
:10E0D000C0EBC00009EBC00062A906F0D7FF601CCE
:10E0E000C4B29DF8C301A042C5D2B700C8EBC808AE
:10E0F000FCB209EBC8013822769806F0C7FF6FF032
:10E10000020000EB86003A1D824218DD9DF8C01126
:10E110009DF8C231591A00EB880339F913309D423A
:10E1200009DA002807DBB0EB810F04DCC4B204EB92
:10E13000880339F91350401C00B28242EBDC9DF891
:10E14000C3119DF8C1210020891A0029A8BF71AA16
:10E150000BDBC0EBC00304EB830339F8133022F868
:10E160001030401CC0B28142F3DACBB2002271A859
:10E170007799FFF7A4FE79B0BDE8F08F2DE9F05F45
:10E1800014460E46054601F04BFBDFF878A500F17A
:10E1900037072078DAF80020617894F805C0D27942
:10E1A00001FB0200385C00F03F08E079401C60454C
:10E1B0008CBF4FF00009BDE8F09F2379A079401C87
:10E1C000984221D9DAF8001007EB030BC87900FB5D
:10E1D0000CF20CFB003012F80B2002F03F0242451B
:10E1E00018BF25F8109009D136F91020B1F90C109C
:10E1F0008A42CCBF25F8102025F81090581CC3B2D5
:10E20000A079401C9842DDD80CF1010000F0FF0C11
:10E21000E079401C6045D0D8BDE8F09F2DE9FF4F64
:10E2200087B00E461598446801F024FB059001F074
:10E2300025FB00210291079A00910191039104911D
:10E24000116031800746220E4FF00009C4F3072009
:10E250000599C846EA460692824224BF04F0FF0EA2
:10E26000C4F3074B3DD3F446E34535D3059A00FB91
:10E2700002C3149A32F913400A2C0EDB3288521C66
:10E280003280B84238BF0746404588BF80468C453B
:10E2900038BF6146CC4588BFE14600233AF91320D8
:10E2A000A2420FDA0822082B09D20AEB420535F800
:10E2B000025C2AF81250521ED2B29342F5D32AF8C9
:10E2C000124003E05A1CD3B2092BE7D30CF1010230
:10E2D00002F0FF0CDC45C9D9401C069AC0B290423E
:10E2E000C1D9A9EB01000999401C08700A99A8EB53
:10E2F0000700401C0870002007993AF91020401CC4
:10E300000968C0B20A44079909280A60F4D30BB01F
:10E31000BDE8F08F2DE9FF4F0746FB4815468FB04B
:10E32000D0E900121C9CCDE90212D0E90212CDE91D
:10E330000412D0E90412CDE90612D0E90610CDE9A5
:10E34000081001F06DFA37300A9001F093FA00904E
:10E3500001F094FA064610980021A6F1010EB0F9DA
:10E3600002200D9200780C901098009E4FEA022A2D
:10E3700040780B90761E8946884608468C460B46A8
:10E38000CDF838A00196002624F8116002AE36F8C8
:10E3900013A00C9E56440DF1100A36B23AF813B091
:10E3A000DDF82CA0DA440FFA8AFBDDF800A0BBF1FF
:10E3B000000F0BFB0A6A0FFA8AFAA8BFDE4529DBB9
:10E3C000002EA4BFDDF804B0B34523DB37F91A6093
:10E3D00024F81160002EDCBF012624F8116034F906
:10E3E0001160DDF838B008F10108BBFBF6FBD94439
:10E3F00008F0FF088642C8BF3046DDF828B01BF899
:10E400000AA0BAF1000F1CBF0CF1010C0CF0FF0CBC
:10E41000324412B2491C5B1CDBB2C9B2042BB2D32A
:10E420000023002624F8116006AE36F813A00C9ED7
:10E4300056440DF1200A36B23AF813B0DDF82CA09C
:10E44000DA440FFA8AFADDF800B0BAF1000F0AFBDD
:10E450000B6B0FFA8BFBA8BFD64517DB002EA4BFB2
:10E46000DDF804A0B24511DB37F91B6024F8116018
:10E47000002EDCBF012624F811600A9E16F80B60FE
:10E48000002E1CBF0CF1010C0CF0FF0C491C5B1C96
:10E49000DBB2C9B2042BC4D31299130281F800C0B5
:10E4A0000D99084400B2B3FBF0F3B9FBF8F11B027D
:10E4B000B3FBF1F3090AA5F84A002965A5F848203D
:10E4C0006B65109805F16B03CDE900705A1E911E23
:10E4D000081FFFF7A3FE13B0BDE8F08F2DE9F0038E
:10E4E000DFF820C2B0F902400025DCF800C0BCF91A
:10E4F0002C60BCF92E809CF8BF90A64227DDB2F9B3
:10E500000060002EC4BFB2F902C0BCF1000F04DDF0
:10E51000B444A4440FFA8CFC12E0B2F904C0BCF17C
:10E52000000FC1BFB2F90670002FBC44A44405DC43
:10E530005788A4443E44B444D688B4440FFA8CFCB3
:10E54000C44504DAB0F81CC0CC4538BF01254FF0F3
:10E55000000C32F81C600CF1010C34440FFA8CFCF6
:10E5600024B2BCF1040FF4DB002D14BF581C8089C9
:10E5700094FBF0F0A1F858002846BDE8F00370477E
:10E580002DE9FF4F85B00C4606460025DDF8489082
:10E5900001F070F9039001F071F9029096F8008093
:10E5A0007778B68901F073F9B4F90020B4F9021054
:10E5B00001911144B4F90430B4F9062000924010DE
:10E5C0001A449142CCBF11B209B2B4F908C0B4F9EF
:10E5D0000EA0B4F90A30B4F90C200CEB0A0B03EBD3
:10E5E000020EF345CCBF0FFA8BFB0FFA8EFB3FB93F
:10E5F000DDF804E08645C4BF00F1010EA4F800E098
:10E60000DDF808E0AEF1010E774505D1B4F90070F0
:10E610008742C4BF471C6780B8F1000F04D1009F38
:10E620008742C4BF471CA780039F7F1EB84505D102
:10E63000B4F904708742C4BF471CE780B4F9047082
:10E640008742C4BFB4F9068080451CDD8445BEBF47
:10E650008342B4F90030834206DB8245BEBF82426A
:10E66000B4F90220824200DA0125052E20D2079853
:10E67000401CB0421CD1594523DCB9F1010F20D90F
:10E680000898F0B921E0B4F900808045C4BFB4F91E
:10E6900002808045E9DD8445BCBF82428742E3DBDE
:10E6A0008342BEBF8245B4F906208242DCDBDCE750
:10E6B000594501DD012D04D1B9F1010F01D90898A7
:10E6C00018B109B00020BDE8F08F09B00120BDE805
:10E6D000F08F70B5044601F0CDF8054601F0CEF894
:10E6E0002178024600291CBF681E814206D060784E
:10E6F00000281FBF511E8842002070BD012070BD40
:10E700001F85EB5118420020549601002DE9F0417D
:10E7100086B014460D468046002601F081F8074673
:10E7200002A8009001AB224629464046FFF7F2FDC1
:10E73000387D002804BF97F82E00002807D19DF8E7
:10E74000043002AA21462846FFF7C8FE064601F01B
:10E7500091F8074601F092F82978024600291CBF7B
:10E76000781E814206D0687800281EBF511E88425C
:10E77000002000D10120002184F85A6084F85F1045
:10E7800084F8610006B0BDE8F08170B514460D460E
:10E7900001F046F802460020127D002A18BF70BD25
:10E7A000A9891E2987BF94F86D104B2994F86D1024
:10E7B000642988BF012070BD2DE9F74FA6B08046BF
:10E7C00001F038F8044601F02BF800218146289822
:10E7D0008DF804100F460E46002840F3C480279899
:10E7E00006EBC60100EB810595F82100012840F0F9
:10E7F000B480702102A806F044FC00201E901F90F7
:10E8000002A84FF0000B249001F00AF8824620A8DD
:10E81000009025AB29464046249AFFF77BFD9AF8E5
:10E820001400002804BF9AF82E00002807D19DF894
:10E83000943020AA28462499FFF750FE834601F021
:10E8400019F8824601F01AF80146287800281CBF02
:10E85000AAF10102904206D0687800281EBF491E26
:10E860008842002000D1012000218DF862B08DF88F
:10E8700067108DF8690000F0FDFF0346D5E905102B
:10E880002A6901EB81015200890000EB8000B1FB95
:10E89000F2F18000B0FBF2F0ADF87810ADF87A003C
:10E8A00000FB031002AB38F81000ADF87C001EAA84
:10E8B00029464046FFF746F900F0B2FF007D4FF0D1
:10E8C000000B00285AD0BBF1010F04BF012089F8CA
:10E8D00030009DF80400702200EB001101EB4010A5
:10E8E00004EB800A2868CAF800006868CAF80A00C1
:10E8F0001E98CAF80400BDF87C00AAF8080002A916
:10E900000AF1140006F0B8FBA868CAF80E002869DE
:10E91000CAF81800A889AAF81400A88BAAF87000F1
:10E9200095F820008AF8BD0095F822008AF8BE000C
:10E9300001208AF8BC008AF8BFB09DF80400401C92
:10E94000C0B28DF804000D282CBF01200020012842
:10E9500009D0A889B84288BF0746701C06B228981B
:10E960008642FFF63CAFA9F804709DF80400002829
:10E970007DD099F8301001290DD0A9E0A8891E2872
:10E9800087BF9DF875004B289DF87500642888BFE7
:10E990004FF0010B97E7032869D8C0F10400C6B215
:10E9A0000025002E88BF012761D99DF80400702240
:10E9B00000EB001101EB4010216844F820109DF895
:10E9C000040000EB001101EB401004EB8000D4F8D0
:10E9D0000A10C0F80A109DF8040000EB001101EBCA
:10E9E000401004EB800061684160218901819DF83D
:10E9F000040000EB001101EB401004EB8000143028
:10EA000004F1140106F038FB9DF8040000EB00113E
:10EA100001EB401004EB8000D4F80E10C0F80E108B
:10EA20009DF80400A16900EB001202EB401004EB1A
:10EA3000800081619DF80400A18A00EB001202EBC6
:10EA4000401004EB800081829DF80400B4F870103F
:10EA500000EB001202EB401004EB8000A0F87010F5
:10EA60009DF8040094F8BD1000EB001200E02FE0C8
:10EA700002EB401004EB800080F8BD109DF804000C
:10EA800094F8BE1000EB001202EB401004EB800083
:10EA900080F8BE109DF8040000EB001101EB40105F
:10EAA00004EB800080F8BC709DF8040000EB0011BE
:10EAB00001EB401004EB800080F8BF709DF804006B
:10EAC000401C8DF80400681CC5B2AE423FF66DAF25
:10EAD0009DF8040029B0BDE8F08FF0B5ADF23C4DD3
:10EAE0000F46064600F09CFE044600F0ACFE0546CC
:10EAF0004FF48761684606F0C4FA207D012805D1ED
:10EB000095F82A203146384605F04CFE6A463946CB
:10EB1000304603F0A7F884F82800024669463046DC
:10EB2000FFF74AFE0546207D012803D129463046DD
:10EB300006F08CFA84F829500DF23C4DF0BD00002F
:10EB40002DE9F007B0F90060B0F902500446012049
:10EB50000E804D808446012ADCBFBDE8F007704777
:10EB600034F92CA004EB8C07A6EB0A09B7F9028054
:10EB700009FB09F9A5EB080808FB0898984510DD82
:10EB800021F820A001EB8006401C7D8800B2758032
:10EB90009042D9BF34F92C60B7F90250BDE8F007B4
:10EBA00070470CF1010C0FFA8CFC6245D8DCBDE813
:10EBB000F007704730B400230028B4BF4242024639
:10EBC0000029B4BFC1F1000C8C4652B9FE4CB4EB25
:10EBD0000C4F06D80029B4BF5A204FF4877030BCC0
:10EBE00070474FEA0C4CBCFBF2FCF84C002254F886
:10EBF0002250654506D804EB82056D68AC4501D20C
:10EC0000134603E0521C12B2592AF0DB00FB01F25A
:10EC1000002ABCBF5A4213B20028B8BFC3F1B400E7
:10EC200008DB0029B1BF5842C3F5B47000B230BC54
:10EC3000A8BF704700B230BC70472DE9F04F0024E8
:10EC4000A3F1010BBBF1000FC4BFDFF87CE3DFF8D9
:10EC50007CA364DD00EB840C30F92460BCF9045023
:10EC6000AF1BBCF90650BCF902C00026A5EB0C0591
:10EC700007FB07FC05FB05CC42F824C0002FB4BFFE
:10EC8000C7F10008B846002DB4BFC5F1000CAC4672
:10EC9000B8F1000F09D1BEEB0C4F06D8002DB4BF60
:10ECA0004FF05A0C4FF4877C31E04FEA0C4CBCFB20
:10ECB000F8F84FF0000C5AF82C90C14507D80AEB31
:10ECC0008C09D9F80490C84501D2664606E00CF1DB
:10ECD000010C0FFA8CFCBCF1590FECDB07FB05FCB7
:10ECE000BCF1000FBCBFC6F1000C0FFA8CF6002F70
:10ECF000B8BFC6F1B40C08DB002DB2BFC6F1000CE2
:10ED0000C6F5B47C0FFA8CFC01DA0FFA8CFC21F802
:10ED100024C004F1010C0FFA8CF45C459ADB00224C
:10ED2000A3F1020CBCF1000F17DD01EB820331F8F7
:10ED300022409888001B00B2B428C8BFA0F5B47068
:10ED400005DC10F1B40FB8BF00F5B47000DA00B202
:10ED50005880501C02B26245E7DB0FFA8BF0BDE829
:10ED6000F08F70B406460020844604460029DCBFBC
:10ED700070BC704706EB84056D88AC440FFA8CFCC0
:10ED8000BCF1000FB4BFCCF100056546954207DD2C
:10ED900004F1010C23F810C0401C80B24FF0000CAD
:10EDA000641C24B28C42E5DB70BC7047F0B4B0F850
:10EDB00000C0049DA2F800C0B0F802C0A2F802C0D2
:10EDC00000244FF0010C002D15DD33F8146002EB28
:10EDD0008C0730F8266022F82C6033F81460641C2D
:10EDE00000EB86060CF1010C768824B27E800FFAC7
:10EDF0008CFCA542E9DC00EB810030F8041C22F811
:10EE00002C1002EB8C0130F8020C4880F0BC0CF1A5
:10EE1000010000B270472DE9FF4F4FF0000B5D4637
:10EE2000DC4658465B465F46D8465E460029C8BF6A
:10EE3000A1F1010A57DD009C04EB8604B4F90240FD
:10EE400004F19609B9F5967F08D835B304FB05FEA1
:10EE5000BEF1000FC6BF23441BB2012704F1320EDE
:10EE6000BEF1640F11D9BCF1000F1CD004FB0CF4EF
:10EE7000002C0ADA08F1010404F0FF08BCF1010FCC
:10EE80000CBF4FF0FF3C4FF0010CB9F5967F11D845
:10EE9000564518BF012F1DD10CE0002CACBF012539
:10EEA0004FF0FF35D2E7002CACBF4FF0010C4FF014
:10EEB000FF3CDBE770B903F17804F02C07D9002B95
:10EEC000BABF02205B4201201BB29B4602E0002336
:10EED0001F461D46741C26B28E42ACDB002818BFAC
:10EEE000A2F800B001D100211180039981F80080BF
:10EEF00004B0BDE8F08FF0B51D1E059C16464FF01E
:10EF0000000C10DD04EB8C0351F82C20DA6004EBCC
:10EF10004C0336F82C20A3F8C4210CF101020FFA9F
:10EF200082FC6545EEDC84F8A052B0F900C0B0F96F
:10EF3000021030F9253000EB8500B0F90220ACEB6F
:10EF40000300891A00FB00F201FB0127FFF732FEE4
:10EF5000A760A08006EB8500B6F9001030F9042CFC
:10EF6000881A0028B8BF501A00B2B428C4BFC0F530
:10EF7000B47000B2A4F8A402F0BD2DE9F74F85B03B
:10EF80000020019082460090114A012000FA0AF008
:10EF90001268B2F8B420024240F0048105980022C1
:10EFA00000EBCA13187830B103285BD091F800C089
:10EFB000844500D00122B3F90200002804BFB3F851
:10EFC00004C0BCF1000F05E03B4A39007496010013
:10EFD000184200201CBF91F800C0BCF1000F08D0FF
:10EFE000B1F902C0844503DBB3F90400844500DDB8
:10EFF000521CD3F808C0BCF1000F04BFD868002829
:10F0000007D08868604503DBD3F80CC0604500DD9D
:10F01000521CB3F91000002804BFB3F812C0BCF1B1
:10F02000000F08D0B1F904C0844503DBB3F9120026
:10F03000844500DD521C988A002802BFD88A002827
:10F040004FF0010970D04FF0000993F834E091F8C7
:10F05000A0B2CC46C8464E46CDF80C90DE4507D946
:10F06000521C61E00878012818BF0228A2D1A2E74B
:10F070000020BBF1000F50D9ABF101040494AEF1B4
:10F080000104029403EB8C04B4F91450B4F9164053
:10F0900055EA040704BF01270397A54211DD01EBE0
:10F0A0004007B7F9C471B7F5B47FDEBFBD4204F5C0
:10F0B000B47424B205DD002FA2BFBC42A5F5B4751F
:10F0C0002DB201EB4007B7F9C471BD4201DCBC426F
:10F0D0000ADA039C012C07D050EA0C040AD0F4454C
:10F0E00048D2012E09D005E009F1010404F0FF091E
:10F0F00001260EE04FF001080FE00CF1010C0CF0BE
:10F10000FF0C00281CBF401EC0B20026029CA44574
:10F11000F0DC401CC0B25845B4D3AEF101008445C8
:10F120009EDBB8F1010F9BD093F87800002804BF54
:10F1300093F879C0BCF1000F08D091F8A1C26045E6
:10F1400003D893F87900604500D2521C93F87A00F6
:10F1500000281CBF91F8A2C2844538BF521CB3F8E6
:10F160007C0000281CBFB1F8A432834288BF521C27
:10F17000C2B908E0049C8442BCDC002E1CBF029C87
:10F18000A445B7DAC2E7B9F1000F0BD0009A07988F
:10F1900000F802A00098401CC0B200900198401CEA
:10F1A000C0B201900AF101000FFA80FABAF10D0F16
:10F1B000FFF6EAAE019808B0BDE8F08F2DE9F04FF8
:10F1C000ADF6F45D17460DF52C79FE4EB0F900C092
:10F1D000B0F90250326801242346B2F8B8A0ADF865
:10F1E000B0C2ADF8B252012926DD00EB830230F93E
:10F1F00023B0B2F90280ACEB0B0EA5EB08080EFBB6
:10F200000EFE08FB08E8C24512DA29F824B009EB23
:10F210008405B2F802C0A5F802C004F1010C0FFA8F
:10F220008CF4A142A4BF30F923C0B2F9025003DB31
:10F230005A1C13B28B42D8DB23460DF628420DF53B
:10F24000FB614846FFF7F9FC401E0FFA80FC30686E
:10F2500000220DF5FB6590F8BB600DF648381046AE
:10F260001146BCF1000F14DD05EB81035B881844E7
:10F2700000B20028B4BF43420346B34205DD481C38
:10F2800028F81200501C82B20020491C09B26145C6
:10F29000EADBBDF8B002ADF86804BDF8B202ADF823
:10F2A0006A04012000210DF52C7C0DF58D63454687
:10F2B000002A14DD35F8116003EB80083CF8266065
:10F2C00023F8206035F81160401C0CEB8606491CC1
:10F2D000768809B2A8F8026000B28A42EADC0CEB38
:10F2E000840131F8042C23F8202003EB800231F84C
:10F2F000021C5180401C03B20DF519620DF5C4616A
:10F300000DF58D60FFF799FC0446401E01B201AB7C
:10F310000DF624420DF5C460FFF77DFD8DF8080061
:10F32000BDF8240CADF80A009DF804008DF8A90280
:10F330008DF8AA7202A8009023460DF5C4620DF55F
:10F3400019610DF58D60FFF7D6FD0DF55E6202A91E
:10F350009D48FFF712FE01281EBF00200DF6F45D48
:10F36000BDE8F08F9DF8E00D974901EBC01090F8D3
:10F370007F000DF6F45DBDE8F08F94480021017028
:10F380008170C1700171704700220029D8BF704799
:10F390002DE9F003DFF82C8282B04FF0010930F93B
:10F3A00022C000EB8207ADF800C0B7F90230ADF81B
:10F3B0000430D8F8005095F86C4014F0040F14BFD6
:10F3C00029EA040604F001061EB1AE79F31A5B1EA9
:10F3D0001BB214F0020F06D0ED79A5EB0C0CACF1CA
:10F3E000010C0FFA8CFC14F0040F19BFADF80030BB
:10F3F000ADF804C0ADF800C0ADF80430BDF8003081
:10F4000003EB031C0CEB4313193320F82230BDF837
:10F410000430521C03EB031C0CEB4313193312B2E0
:10F420007B808A42BBDB02B0BDE8F00370472DE968
:10F43000F043DFF8909100263746D9F800300029D4
:10F4400093F807809D79334615DD30F923C0C44514
:10F45000B8BFE046B445C8BF664600EB830CBCF9B4
:10F460000240AC42B8BF2546BC42C8BF27465B1C21
:10F470001BB28B42E9DBA6EB080303F101031CB2CC
:10F48000A7EB050303F101031BB29C42CCBF274647
:10F490001F46B4BFA4469C4682F800C04C4A002BCD
:10F4A0001570D9F800C09CF807C0ACEB060CACF1A5
:10F4B000010C82F801C0B8BF5B42464A002C1370B1
:10F4C000B8BF64425470032FBCBF0020BDE8F08376
:10F4D000FFF75AFF0120BDE8F0832DE9F34F3949CA
:10F4E0009DB04FF0000909681C914A4691F806B09A
:10F4F000C979CDF80090CDF80490CDF80890CDF8FA
:10F500000C90CDF81090CDF81490CDF81890CDF85F
:10F510001C90CDF82090CDF82490CDF82890CDF80F
:10F520002C90CDF83090CDF83490CDF838901092E2
:10F53000119214924FF0000A1292139215921692A1
:10F540001992C846179218921A924FF0FF345546F6
:10F55000D4460DF1380E6E46CDF83C901B92BBF1AF
:10F56000000F28DD002200291FDD0CFB012330F9EC
:10F570001330322B10DD36F812706D1C1F4426F844
:10F5800012703EF81C70A3421F442EF81C7008DD58
:10F590001C469146E04604E013F1280FB8BF4FF037
:10F5A000010A521C12B28A42DFDB0CF101020FFA8F
:10F5B00082FCDC45D6DB00220120ABF1010BBBF164
:10F5C000010F09E018420020DC97010002420020F0
:10F5D000074200200942002014DD0EEB400C3EF9EA
:10F5E00010303CF9027CBB42A2BFBCF902C09C4572
:10F5F000322B03DD801C521C00B2D2B2401C00B280
:10F600005845EADB00230120A1F1010E7C4FBEF139
:10F61000010F16DD06EB400C36F910103CF902BC68
:10F620005945A2BFBCF902C08C45322903DD801CBC
:10F63000591C00B2CBB2401C00B27045EADB012B72
:10F6400006D8012A04D8BAF1010F01D0502D02D9F1
:10F650000220B87020E06A48002C0178B87813DDE9
:10F66000002804BF0120B870664820F8219000EB04
:10F670008100A0F802801C9890F8B600884224BF50
:10F68000481C387016D307E0012809D0022813D08F
:10F69000032801D00020B870B8781FB0BDE8F08F03
:10F6A0000329F7D957481E9AFFF7C1FE002818BF53
:10F6B0000320F0D10220EEE70329EDD8EAE72DE997
:10F6C000F00707460020012F84BF4FF0000CDFF841
:10F6D000388108BF08789CBFBDE8F0077047CCEBC5
:10F6E000CC0618F80640BC4218D100231A46002C5C
:10F6F000C8BF06EB08050EDD05EB020911F802A0F4
:10F7000099F80190D1451CBF5B1CDBB2521C12B2B0
:10F710009442F1DC13B906EB080080790CF1010288
:10F720000FFA82FCBCF1030FD9DBBDE8F00770478C
:10F7300070B584B000258DF808502E46406802A9A7
:10F74000FFF7CBFE2E4C40B1012808BF65700FD0EB
:10F75000022809D003280DD01DE0207901281AD1F4
:10F760006078401C607016E065702570A570E570CB
:10F77000257110E09DF8082021782248FFF71EFD32
:10F780000146224AE0781154401CE07065702570F3
:10F79000A570012020711E486278006890F8BA10A8
:10F7A000914204D990F8B700E178884224D81749EB
:10F7B000E078FFF784FF02001AD01648DFF858C03F
:10F7C00001789CF8003040789CF801C08DF800204A
:10F7D0008DF801100B4484448DF802008DF803303D
:10F7E0008DF804C0052269460120FBF769FE012659
:10F7F0002570A570E570257104B0304670BD00001D
:10F8000002420020D88C00205C9E01000B420020A8
:10F810001842002007420020094200205E4870473D
:10F820005E485F490078C0EB001000EBC00001EBC0
:10F83000C0007047594840F27D21407848435949FB
:10F8400001EB8000704755485549007880F0010071
:10F85000C0EB001000EBC00001EBC00070474F4848
:10F8600040F27D21407880F0010048434D4901EB92
:10F870008000704749488068C07970474748806871
:10F880008079704745488068B0F90C00704743485C
:10F890008068B0F90E0070474048017881F001019E
:10F8A000017070473D48417881F001014170704717
:10F8B00040F6F41105F0E5BB4FF4876105F0E1BBBC
:10F8C0002A2105F0EDBB354910B58860FDF77EFCB7
:10F8D000BDE81040FCF768BD3048017881F00101B7
:10F8E0000170417881F00101417070472B494860F7
:10F8F00070472A484068704728488168497A11F063
:10F90000010F12BF00200079C0F300107047234898
:10F910000079C0F38000704720484068C0F38060E1
:10F9200070471E480079C0F3C00070471B4800793B
:10F93000C0F3C010704770B50D4618490646184A06
:10F940000878C0EB001000EBC00002EBC004487860
:10F9500040F27D21484302F5076101EB800040F64B
:10F96000F41105F08EFB29463046FFF7B6F804F097
:10F9700075FA304603F0D3FA2946304602F04EFFBE
:10F9800020B994F829103046FCF7D5FC02F050FF5E
:10F9900094F82A0070BD0000908E002010420020D4
:10F9A000BC8E00202C970020FE48704790F805C0C0
:10F9B0009C4588BF437190F804C0944588BF02718C
:10F9C00090F807C09C4538BFC37190F806C09445B5
:10F9D00038BF8271B0F902C08C4502DA41800270F2
:10F9E0004370B0F80CC00CF1010CA0F80CC0D0F8BA
:10F9F00010C08C44C0F810C0D0F814C001FB02C283
:10FA00004261826901FB0321816170472DE9FF4F4B
:10FA100081B00F4680460E9EFFF72CFF0546FFF78C
:10FA20002DFF82460498039968433144425CBA42F0
:10FA300008BF00F80180012104984FF0000C401A23
:10FA400003B20498084400908342C4BF05B0BDE8E7
:10FA5000F08F0398401A0FFA80FB039800EB01091E
:10FA60005A469145A8BF03FB05F416DB002BA8BF3F
:10FA70009A450EDD002AA8BF95420ADDB01814F899
:10FA800000E0BE4505D104F800800CF101000FFA3A
:10FA900080FC501C02B29145E8DA581C03B2009871
:10FAA0009842DDDABCF1000F04BF05B0BDE8F08F6D
:10FAB000481C01B20529BFDD05B0BDE8F08F2DE976
:10FAC000F34F85B00746FFF7ABFE0446FFF7D2FEC3
:10FAD0008246069804F137054FF0000900289CBFC4
:10FAE00007B0BDE8F08F0026A0EB0900401E039090
:10FAF000002854DD06EBC60807EB8804B4F90200C1
:10FB0000B4F92610884245DA616A20682160606293
:10FB1000A16A60686160A06204F10C000FC80093E4
:10FB2000E369019304F1300393E80858C4E9033B07
:10FB3000C4E905CE236CE36104F1300B009BABE814
:10FB40000F00019B236417F8280061784FF0FF0B2A
:10FB500001FB0A00285C019094F8242094F82530D9
:10FB600003FB0A20285C0290014600955846FFF7E7
:10FB70004DFF0095DDE90110637817F82820FFF7A5
:10FB800045FF009594F8253094F8242059460198B3
:10FB9000FFF73CFF701C86B20398B042AADC09F163
:10FBA00001001FFA80F9069881459CD307B0BDE893
:10FBB000F08F2DE9FF4F8046002097B015460E4686
:10FBC0008346824604461190FFF72AFE8146FFF7DE
:10FBD0003AFE1290FFF722FE1090FFF74FFE074605
:10FBE000FFF748FE159099F80000149099F801006D
:10FBF0001390B9F902C01322B8F1000F13BF1A987D
:10FC00000120119000287DD00020002F0CD9012167
:10FC10006C46002338F910E09645CCBF215423549C
:10FC2000401CC0B2B842F5D3159938467C1808ABD1
:10FC3000A7420FD2C11B38F910E0C9B29645CCBF1C
:10FC40004FF0010E4FF0000E03F801E0401CC0B26F
:10FC50008442EFD81498185C20B910994FF0010B2A
:10FC600081F829B01398E8461DF8000020B91099D2
:10FC70004FF0010A81F829A000242146002D88BFF9
:10FC8000022722D901EBC10206EB820090F821E0A5
:10FC9000BEF1010F15D1B0F902E0E64511DABBF172
:10FCA000000F03D116F822209A5C32B1BAF1000F8E
:10FCB00007D1427818F802201AB980F82170601C28
:10FCC000C4B2481CC1B2A942DCD312981A9990F868
:10FCD0002A00091B884218DD022816D90024204674
:10FCE000002D88BF012223D900EBC00106EB810162
:10FCF00091F82130022B08BF81F82120401CC0B2AE
:10FD0000A84200E014E0EFD312E00020002D88BFED
:10FD100000220DD900EBC00106EB810191F82130E2
:10FD2000022B08BF81F82120401CC0B2A842F1D3A9
:10FD300099F82D00204489F82D0011981BB0BDE8DA
:10FD4000F08F2DE9F00300228FB0944600920192CB
:10FD500002920392049205920692079208920992E7
:10FD60000A920B920C920D920E92002884BF6F465D
:10FD70000C4D43D9002200283AD9CCEB0C1301EBEF
:10FD800043060CF10104B35C012B2DD135F81C3076
:10FD9000CBB335F81280B8F1000F0CBF25F8123044
:10FDA000434501E014AB00201ED00023002807D9F2
:10FDB00035F8138027F813805B1CDBB29842F7D824
:10FDC0000023002810D935F81380944530D837F82F
:10FDD0001C90C84508BF37F8128001D125F8138060
:10FDE0005B1CDBB28342EED3521CD2B28242CAD336
:10FDF0000CF1010202F0FF0C8445BBD30FB00020D0
:10FE0000BDE8F0037047FFE735F81230002B18BF4C
:10FE100025F81C30E8D1944599BF25F81C4025F8F9
:10FE20001240531C25F81C3088BF25F81230DBE740
:10FE300037F81290C84508BF37F81C80D0D1CDE7FD
:10FE40002DE9F04F0546501EC0B2DDE9094BDDE952
:10FE50000C9800EBC00A03EB8A061F4686F8019057
:10FE600035F814007080085D1044085503F82A80A6
:10FE7000012086F8210086F8048086F8068086F83E
:10FE8000059086F8079035F914104B4642463046E7
:10FE9000FFF78CFD707850B904EB0B0135F9142095
:10FEA00035F911108A4208BF09F101000ED00B99F3
:10FEB000491E88420BD1A4EB0B0035F9141035F91B
:10FEC0001000814208BFA9F1010000D1707017F83D
:10FED0002A1005EB440041B935F91420B0F902307D
:10FEE0009A4208BF08F101000CD0ABF10102914227
:10FEF0000AD135F9141030F9020C814208BFA8F17B
:10FF0000010001D107F82A0017F82A10204661F3F2
:10FF10000700717861F30F20718861F31F40BDE81D
:10FF2000F08F2DE9F34FAFB00646002028908021D6
:10FF300006A805F0A6F8FFF773FC80464FF4806131
:10FF4000373005F0ADF808F13704FFF7A0FC279033
:10FF5000FFF794FC2990FFF78DFC0746B8F90200E3
:10FF6000269098F8069098F8082048460DF1180A4F
:10FF70008242A4BFFA214FF0FF3309DB2AF8201098
:10FF80000AEB800C401C00B2ACF802308242F5DA79
:10FF900098F8072098F8090090426CDB04EB090000
:10FFA0000AEB890B009002FB0791002036F9113013
:10FFB00027998B4211DD009902FB07F30A20585460
:10FFC0003AF929009042C8BF2AF82920BBF902005B
:10FFD0009042B8BFABF80220012098F808104D46B7
:10FFE000A94242DD02FB075109B206EB410C36F98A
:10FFF0001130BCF902C06345DCBFDDF89CE0E6458A
:020000021000EC
:100000002BDA002818BF012829D16345BCBF002086
:1000100060540CDB3AF925008242B8BF2AF825204B
:100020000AEB8500B0F902309342B8BF428098F8DD
:100030000800401EA8420BD10AEB8500B0F904303D
:100040009342C8BF8280B0F906309342B8BFC280E5
:100050000A2021444870012001E001282DD0691CAC
:100060000DB298F80810A942BCDC501C02B298F8F6
:100070000900904297DA0020059098F8080048455A
:10008000C0F2EA802998401E2D90781E2C9006A878
:1000900030F929A000EB89002B90B0F902005045FF
:1000A000A4BF09F0FF002A90C0F2CD800AFB0790A0
:1000B00005B2605D0A2813D0BBE03AF92510002094
:1000C0009142C8BF2AF825200AEB8501B1F902C088
:1000D0009445B8BF4A8026998B42C8BF2693BEE795
:1000E00000208446421E00904FF0FF300AEB0201D0
:1000F0000029A4BF2D9B8B4221DB09EB0003002BC1
:10010000A4BFDDF8B0B09B4519DB52EA000B16D056
:1001100001FB07331BB236F915E036F913B0F3458E
:1001200004DD002363550123009308E0E35C13F032
:10013000800F04D003F03F034FF0010C2893401CC4
:1001400000B20128D4DD501C02B2012ACCDD009897
:10015000002818BFBCF1010F6BD136F91530279874
:10016000834266DDBCF1010F08D00598401CC0B287
:1001700005901E2841D91E20059064E0289809F0BA
:10018000FF0200EBC001309800EB810024380AF038
:10019000FF0190F805C08C4588BF417190F804C0FC
:1001A000944588BF027190F807C08C4538BFC17173
:1001B00090F806C0944538BF8271B0F902C09C45E2
:1001C00002DA438002704170B0F80CC00CF1010CEF
:1001D000A0F80CC0D0F810C09C44C0F810C0D0F8F3
:1001E00014C003FB02C24261826903FB01218161E9
:1001F000289840F0800060551BE0DDE929020AF0F4
:10020000FF01CDE90201CDE90057049221463046B5
:10021000309B059AFFF714FE0599021441F0800106
:10022000615526998A4204D188F80000000A88F8AE
:1002300001000AF101000FFA80FA2B98B0F90200D0
:100240005045BFF633AF09F101000FFA80F998F875
:1002500008004845BFF61BAF059831B0BDE8F08FE8
:100260002DE9F0470024884681462546FFF70FFB1D
:100270000746FFF7D5FA0646FFF749FB0028B6F90F
:10028000020014BF411081100022B8F1000F88BF96
:100290004FF0000C1FD902EBC20009EB8003B3F949
:1002A00002008842C8BFB8420BDC93F821A0BAF123
:1002B000010F0CD183F821C0B842C4BF601CC4B286
:1002C00005E093F82100012804BF681CC5B2501C4A
:1002D00082B24245DFD396F82D00204486F82D00E7
:1002E0002846BDE8F08770B515460E460446FFF770
:1002F000AAFAFFF795FA002180F82D10294630461A
:10030000FFF7AEFF002C08BF70BD03462A463146FA
:100310002046BDE870404CE42DE9F00F8246DDE94F
:1003200008690120DDF828809B464B451EDC00272C
:100330001446DC46B442D8BF63450DDC0CFB0845CF
:1003400031F91550002DC8BF2F44641CACF1010CCD
:1003500024B20FFA8CFCEDE74AF82070401C0BF138
:10036000010C0FFA8CFBC0B2CB45E0DD521C17B27A
:10037000B742C4BFBDE8F00F704700243A464D466F
:10038000B242D8BFAB420EDC05FB082C31F91CC0D1
:10039000BCF1000FC8BF6444521CA5F1010C12B29D
:1003A0000FFA8CF5ECE74AF82040401C7A1C17B293
:1003B000C0B2B742E1DDBDE8F00F70472DE9F00FA4
:1003C0008246DDE909980120DDF820B01D464B4545
:1003D0001EDC00265C46AC469442A8BF9C450DDB63
:1003E0000CFB084731F91770002FC8BF3E44641E4C
:1003F000ACF1010C24B20FFA8CFCEDE74AF8206056
:10040000401C05F1010C0FFA8CF5C0B2A945E0DAE9
:10041000ABF1010C0FFA8CF7BA42C4BFBDE8F00F84
:10042000704700263C464D469442A8BF9D4210DBD3
:1004300005FB084C31F91CC0BCF1000FC8BF664475
:10044000A4F1010C0FFA8CF4A5F1010C0FFA8CF554
:10045000EAE74AF82060401CA7F1010C0FFA8CF77C
:10046000C0B29742DDDABDE8F00F70472DE9F00722
:100470004FF000084746464645464FF0010C01291B
:1004800024D900EB8C0950F82C4059F804AC5445A1
:10049000C4BFD9F804A054450BDDB44204DD354691
:1004A00047462646E0460BE0A542BCBF25466746C8
:1004B00006E0D9F804904C4504BF641E40F82C4077
:1004C0000CF1010C0CF0FF0C8C45DAD3C2E900658D
:1004D00083F800805F70BDE8F007704730B41C6897
:1004E000029D8C42C4BFD3F804C0944507DC9442FB
:1004F000C7BF5A688A42642030BCD8BF704795F89D
:1005000000C06A7894453ABF614694461146224637
:10051000614508D850F821309342B8BF1A46491CAB
:10052000C9B26145F6D96420504390FBF4F030BC69
:1005300070472DE9FF4FC9B000240F468046A346FF
:100540004FF4807104A8039404F09BFD44944594F7
:10055000FFF779F94690FE480068008C04B2FFF777
:1005600089F94790FFF78AF900268146DDF81CA13A
:100570003546304618F8001001EBC10107EB810148
:100580000A795245B8BF92464A794A45B8BF914662
:100590008A79B242C8BF1646C979A942C8BF0D467A
:1005A000401CC0B20228E5D347980096CDE901501F
:1005B0004B46524604A84B99FFF7AEFE014603ABEB
:1005C00044AA04A8FFF752FF03A8009098F801007E
:1005D00044AB00EBC00007EB8000B0F9022098F8B4
:1005E000000000EBC00007EB8000B0F9021004A887
:1005F000FFF774FF48904FF4807104A804F041FDA8
:1006000047980096CDE901504B46524604A84B99B5
:10061000FFF7D4FE014603AB44AA04A8FFF726FF68
:1006200003A8009098F8010044AB00EBC00007EB72
:100630008000B0F9022098F8000000EBC00007EB42
:100640008000B0F9021004A8FFF748FF4899A142C2
:1006500003DA642808BF084606D0A04201DA6429FC
:1006600002D04FF0010B2AE0642828DA469991F86D
:100670002A1081B1469991F83210022904BFA4F1E1
:1006800014010CB2469991F83110052912BF0329C3
:1006900004F114010CB2A042E3DA46994FF0020BC8
:1006A00091F83210022901D0192803DA4C9802215E
:1006B000817004E02D2802DD4C98012181704C9856
:1006C00080F801B04DB0BDE8F08F2DE9F04782B061
:1006D0000024994692468846074600940194FFF705
:1006E0009FF80546FFF7AFF8B5F902008610FFF74F
:1006F000CEF8B04202DDFFF7CAF806464FF0000C14
:10070000002F21DD93496A4601AB0CEBCC0008EBCE
:10071000800090F82150012D10D1B0F90200B042B4
:100720000CDD31F81C50002D18BF022C3CBF1555B4
:1007300003F804C0601CC4B2022C05D80CF10100FF
:100740000FFA80FCBC45E0DB89F80040022C1CBF9E
:1007500002B0BDE8F0879DF800009DF801108842C6
:100760001CBF02B0BDE8F0874B465246414601A887
:10077000FFF7DFFE02B0BDE8F0872DE9FF4F04462A
:10078000ADF5097D0020DDF85CA283908590409056
:1007900041904290439044904590469047904890B5
:1007A00049904A904B904C904D904E904F90509065
:1007B0005190529053905490559056905790589015
:1007C00059905A905B905C905D905E905F906090C5
:1007D0006190629063906490659066906790689075
:1007E00069906A906B906C906D906E906F90709025
:1007F00071907290739074907590769077907890D5
:1008000079907A90064680467B907C907D907E9091
:100810007F90FFF705F88346FFF715F80BF13700D7
:1008200087904B48006890F8279090F824108091AA
:1008300090F826008690FFF71DF88290FFF71EF8CB
:10084000829D0746819584909BF82E00012808BF61
:100850004FEA69099BF80C0002281ABF03280528F3
:10086000A9F1140900218B9800282ED98A9830F814
:10087000110000EBC00304EB83000279AA4238BFE9
:1008800015464279BA4238BF17468279B24288BFCC
:100890001646C279424588BF904614F82320819BB2
:1008A0009A4238BF81924078849B984238BF8490A6
:1008B000839B9A4288BF8392859A904288BF859095
:1008C000481CC1B28B988142D0D33A46474598BF65
:1008D0000DF5A07E33D82C46B54298BFD01B2AD840
:1008E0008299879B02FB014189B25B5CFBB1DDF819
:1008F00058C23EF810303CF911100B442EF810305D
:1009000070AB33F910C08C45B8BF23F81010631BCF
:100910000DF5807C3CF813B08B442CF813B00DF52A
:10092000C07C3CF913B08B45B8BF2CF81310611C88
:10093000CCB2B442D4D9501CC2B24245CBD900216A
:100940004FF47A74BDF800310A46084604E000000E
:100950001842002014AB0020A6EB050BBBF1000FE2
:1009600030DD6426EC462DF820600CEB800C002670
:10097000CDF808C2ACF802600DF5807C3CF910603F
:100980000CEB400CBCF902E07645C8BF022115DA39
:1009900000290CBF012101290CD060A931F812E017
:1009A0008299A1F802E06421714391FBF3F12DF8E3
:1009B00020100121BCF80230421CD2B2401CC0B24F
:1009C0005845CEDB40A9002031F81B300BF0FF0268
:1009D0001BF0FF064DD040A931F916C001EB4601CE
:1009E00031F902ECF445C8BF02203EDAC0B3012859
:1009F00037D0B1F902E03046F4450BD1401CC0B20B
:100A00000DF5807C3CF910E00CEB400CBCF902C009
:100A1000E645F3D0EC460CEB800CCDF808C2BCF8F0
:100A200002E00DF5C07C3CF81220DDF808C27244EB
:100A300092B2ACF80220DDF808C25208ACF80220ED
:100A400040AA4FF0640C32F9102002FB0CF292FB2A
:100A5000F3F23DF8203092B2934288BF2DF8202067
:100A6000012031F8023C711ECAB2711E11F0FF065E
:100A7000B1D1BBF1000F3CDD8098000288903DF8B9
:100A800026006A46642830D2A919829102EB8601B9
:100A900087914A8880998A423CBF8699814210D2C8
:100AA000FEF727FF10F0040F0BD1879A8898528821
:100AB000B0FBF2F03DF826205043C0F30F202DF894
:100AC00026003DF8260048450FDADDE981128A420A
:100AD000A4BF8399914208DBA04206D204460120BC
:100AE000AAF800008298AAF80200701CC6B2B345AA
:100AF000C5DC0021BDF84031A8EB07050A460846D1
:100B0000002DC8BF0DF1800E2EDD4FF0640C2EF8C5
:100B100020C00EEB80084FF0000CA8F802C00DF5C5
:100B2000A07C3CF910600CEB400CBCF902B05E45B7
:100B3000C8BF022114DA00290CBF012101290BD002
:100B400070A931F81210A8F802106421714391FBCA
:100B5000F3F12EF820100121BCF80230421CD2B271
:100B6000401CC0B2A842D0DB50A9002031F815309B
:100B7000EAB215F0FF0618BF0DF5E07845D00DF587
:100B8000A07B0BEB46013BF916C031F902ECF445B2
:100B9000C8BF022035DA78B301282ED0B1F902B0EF
:100BA0003046DC4508BF0DF5A07C09D1401CC0B221
:100BB0000CEB400E3CF910B0BEF902E0F345F5D065
:100BC0000DF1800E0EEB800C38F81220BCF802B04C
:100BD0005A4492B25208ACF8022050AA4FF0640C6A
:100BE00032F9102002FB0CF292FBF3F23EF82030B7
:100BF0009342C8BF2EF82020012031F8023C711E1C
:100C0000CAB2711E11F0FF06B9D1002D3CDD8098EB
:100C10000002819020A931F82600642830D201EB2F
:100C2000860B8099BBF8022007EB06088A423CBF7E
:100C30008699814211D2FEF75CFE10F0040F0CD1B0
:100C4000BBF80220819820A9B0FBF2F031F82620F1
:100C50005043C0F30F2021F8260020A830F82600CA
:100C600048450DDA84998845A4BF8599414507DB3D
:100C7000A04205D204460220AAF80000AAF8028089
:100C8000701CC6B2B542C5DCB4F57A7F0CBF00203B
:100C900001200DF50D7DBDE8F08F2DE9F001002755
:100CA000059E5F704FF01E0C83F800C0BC46002804
:100CB0009CBFBDE8F001704731F81C40651E1D2D3A
:100CC0000AD20CEBCC0506EB850595F82150012DD9
:100CD00018BF21F81C7008D00CF1010C0CF0FF0CAF
:100CE0008445E9D3BDE8F00170475D784DB193F8D4
:100CF0000080A045F0D122F815C05C78641C5C70BF
:100D0000EAE71C70A2F800C05C78641C5C70E3E742
:100D10002DE9F04F93B081460020DDF870A00090DF
:100D2000019002900390049005900690079008901F
:100D300009900A900B900C901F46164688460D901D
:100D40000E900F90109000251190FEF797FD04462D
:100D5000FEF790FD0146388801281EBF022813B017
:100D6000BDE8F08FBA78521C8DF80420012808BF26
:100D70008DF8051003D0022808BF8DF80540002427
:100D80009AF80100EE460DF1080B03A9002838D9A6
:100D90003888012802D0022807D00DE036F8140068
:100DA00000EBC00018F8205006E036F8140000EB05
:100DB000C00008EB800045787888A8422CBF4FF02F
:100DC000000C4FF0010C16F814201BF80C00CCEBB3
:100DD0000C1301EB4303C254401C0BF80C0001A898
:100DE00010F80C20AA4206D900F80C5016F814008E
:100DF000401C0EF80C00601CC4B29AF80100A0421E
:100E0000C6D89DF8080000281BBF9DF809000028DF
:100E10001E250025002200201BF80240002C0ED9C0
:100E2000C2EB021301EB430C1EF802302B441CF8FA
:100E30000060401CC0B229F816308442F7D8501C1C
:100E4000C2B2022AE7D313B0BDE8F08F2DE9F04F0C
:100E500093B000260296039604960596069607968A
:100E6000089609960A960B960C960D961C46904687
:100E70000F4605460E960F96109611960DF10C0B27
:100E80000DF1100A129607960C9611960296089686
:100E90008DF809601E200496059606960D968DF82D
:100EA000080009960A960B96129600200E960F9649
:100EB000109604A90DF1080C0396002D5AD934F8A8
:100EC00010305A1E1D2A0AD200EBC00207EB820224
:100ED00092F82120012A18BF24F810601FD0401C6E
:100EE000C0B2A842EBD39DF80920002A42D0012AC3
:100EF00004BFBDF8100024F81060C4D0CDE9008B09
:100F00009DF808303846FFF738FC00B302A800907F
:100F100003AB04AA39462046FFF7FAFEB3E79CF874
:100F200001205AB19CF800909945D8D121F81200BF
:100F30009CF80120521C8CF80120D0E78CF800307E
:100F400008809CF80120521C8CF80120C7E79DF80E
:100F500009100020002996D93AF81010401CC0B2A0
:100F600034F811201E3224F811209DF80910814216
:100F7000F2D888E70020002D9CBF13B0BDE8F08FA9
:100F800034F810101E2984BF1E3924F81010401C9C
:100F9000C0B2A842F4D313B0BDE8F08F00EBC00399
:100FA00002EB830301EBC10C02EB8C02243B243ADD
:100FB000884208BF704718791179884238BF10718C
:100FC00098799179884288BF90715879517988428F
:100FD00038BF5071D879D179884288BFD071908953
:100FE0009989084490811069196908441061506911
:100FF0005969084450619069996908449061B3F94E
:101000000200B2F90210884204DD50801878107096
:1010100058785070012082F82000002083F82100C9
:1010200070472DE9F0471C46904689460746FEF773
:1010300021FC6379E1799942B8BFBDE8F08794F863
:1010400004C0A179614513DB03FB00C18DB27E5D55
:1010500006F03F01494504D106F0800141EA08014C
:1010600079550CF101010FFA81FCA1796145EBDAA8
:10107000591C0BB2E1799942E1DABDE8F087F0B58D
:101080008FB00024134600940194029403940494B6
:101090000D460646059406940794089409940A940C
:1010A0000B940C940D943C22194668460E9403F060
:1010B000EDFFA446634661466A46002D09D932F821
:1010C000110000281CBF581CC3B2481CC1B2A94261
:1010D000F5D3F01A0021C6B2002D18D932F811301C
:1010E0008BB10CF1010000F0FF0C481CC0B2A8420B
:1010F00009D232F810709F4208BF22F81040401CFD
:10110000C0B2A842F5D3481CC1B2A942E6D306EB4F
:101110000C000FB0C0B2F0BD70B50546FEF780FB05
:101120000446FEF790FB697800220126022908D0C8
:10113000012912D084F8312084F8322084F8332039
:1011400070BD2878022814BF0320052084F83100E0
:1011500084F8326084F8332070BD90F83110022397
:101160004FF0040C022907D004290FD0052904BF31
:101170002978022922D02AE090F82A0038B384F88E
:1011800031C084F8323084F8336070BD90F832108A
:1011900002291CD190F82A10C9B184F831C090F806
:1011A0003300401CC0B284F8330084F83230052884
:1011B00004BF84F8322084F8332070BD90F82A00F0
:1011C00000281CBF84F8313084F83230C2D184F852
:1011D00031C084F8322084F8332070BD2DE9F74FF8
:1011E0004FF0000AB8B00D46CDF8B8A0CDF83CA03D
:1011F000CDF840A0CDF844A0CDF848A0CDF84CA043
:10120000CDF850A0CDF854A0CDF858A0CDF85CA0F2
:10121000CDF860A0CDF864A0CDF868A0CDF86CA0A2
:10122000CDF870A0CDF874A0CDF800A0CDF804A042
:10123000CDF808A0CDF80CA0CDF810A0CDF814A0E2
:10124000CDF818A0CDF81CA0CDF820A0CDF824A092
:10125000CDF828A0CDF82CA0CDF830A0CDF834A042
:10126000CDF838A0CDF878A0CDF87CA0CDF880A03E
:10127000CDF884A0CDF888A0CDF88CA0CDF890A0B2
:10128000CDF894A0CDF898A0CDF89CA00446D04607
:10129000D146CDF8A0A0CDF8A4A0CDF8A8A0CDF857
:1012A000ACA0CDF8B0A0FEF7BBFA0746FEF7CBFA2C
:1012B0002D90FEF7D4FA309007F1370034902D9836
:1012C00037303290FEF7D6FA319056460020FF4B69
:1012D0006AF30706002C0BD900EBC00105EB810176
:1012E00091F82120012A16D0401CC0B2A042F3D3AD
:1012F00087F834A087F835A0012187F836A0B9F126
:10130000010F08BF87F83410387B02281CBF032860
:10131000052813D10EE0721CD2B262F30706012A2F
:1013200008BF13F8108091F82010012908BF4FF072
:101330000109D9E73A98817001202E902D984FF03D
:10134000000990F82900002884BF601E2F9040F209
:10135000D68009EB091000EB4913309800EB8302AB
:1013600092F8BC0001287DD10021039108910091E1
:101370000191029104910D910591069107910991B6
:1013800030980A910B910C910E9110F8233092F83D
:1013900001C031980CFB00333298C05C00F03F0074
:1013A00036902E9801282CD0907B339092F80FA085
:1013B00092F8108092F811C00020002C52D900EB56
:1013C000C002DDF8C4B015F8223005EB8202359278
:1013D000527802FB0B3EDDF8C8B01BF80EB0DDF80A
:1013E000CCE00BF03F0B734528BF98451DD39245C9
:1013F00098BF624519D8359A92F82120012A14D154
:1014000008E0907A339092F80BA092F80C8092F852
:101410000DC0D1E7AD4A32F8102032B1369B5B45A2
:1014200003D1491C2DF81020C9B2401CC0B2A04203
:10143000C5D3012959D94FF0000ECDF878E0CDF889
:101440007CE0CDF880E0CDF884E0CDF888E0CDF800
:101450008CE0CDF890E0CDF894E0CDF898E0CDF8B0
:101460009CE000E041E0CDF8A8E02F99CDF8A0E0A5
:10147000CDF8A4E0CDF8ACE07046CDF8B0E000299E
:10148000C4BFE8460DF1780C2FDD38F8101039B3E1
:10149000421C0023D1B22CF81020A14220D238F8EF
:1014A00010A038F811B0DA4505D12CF811205B1CDA
:1014B00028F811E0DBB2491CC9B28C42EFD8002BEE
:1014C0001CBF0021002C88BF0FAB09D93CF81120AC
:1014D000002A18BF23F81120491CC9B2A142F5D334
:1014E000401C2F99C0B28842CFDB09F1010000F007
:1014F000FF092D9890F8290048453FF62AAFF6B22B
:101500000FAA21463046FFF7BAFD2D992E900020F4
:1015100091F82A10A1B1B14212D82D9991F8341046
:1015200001290CD02D9991F8351001291CBF97F88D
:101530003410012903D03A998978012900D101207A
:1015400087F835003A994E702E998E4228BF0128AF
:1015500042D14FF00008002C3BD90FAE36F81810DE
:1015600089B32A4608F10100FFF718FD08F10100D0
:1015700000F0FF0A16F8189008EBC80005EB80068B
:10158000349FFEF777F984467179F07988421ADB47
:101590003079B279904211DC01FB0C0292B2BB5C53
:1015A00003F03F0BD34504D103F0800343EA090362
:1015B000BB54401CB27900B28242EDDA481C01B241
:1015C000F0798842E4DA08F1010000F0FF08A04554
:1015D000C3D33A992E9848703A98FFF79DFD3BB0D7
:1015E000BDE8F08F10B44FF0000C634600280ED910
:1015F00031F8134014B10CF1010C03E05B1CDBB2B9
:101600008342F5D3BCF1000F18BF012000D10220A6
:10161000507010BC704730B44FF0000C6446634605
:1016200000289CBF30BC704703EBC30501EB850568
:1016300095F82150012D06D1BCF1000F0FD0641C8C
:1016400022F813C0E4B25B1CDBB28342ECD3012C62
:1016500084BF02EB4C0020F802CC30BC704703F191
:10166000010C0CF0FF0C0124EDE72DE9F043C1B0B3
:101670000E4607469846154614688021684603F0D2
:1016800000FD98F804C028780022E946604515D985
:1016900007EB8C0157F82C004968401A49F82C00D8
:1016A0000028BFBF41428A420A466CF307040CF18E
:1016B000010000F0FF0C28786045E9D880214846F9
:1016C00003F0DFFC002298F806C001E014AB002014
:1016D0006878844516D907EB8C0157F82C0051F82F
:1016E000041C401A49F82C000028BFBF41428A421E
:1016F0000A466CF30F24ACF1010000F0FF0C68788F
:101700006045E8D3802120A803F0BBFC98F80500D1
:10171000A978002320AF884213D206EB800256F846
:1017200020105268891A47F820100029BFBF4A428A
:101730009342134660F31744401CA978C0B281421B
:10174000EBD88021384603F09CFC98F80700E97834
:101750000023884214D906EB800256F8201052F874
:10176000042C891A47F820100029BFBF4A4293422F
:10177000134660F31F64401EE978C0B28142EAD389
:101780002C6041B0BDE8F0832DE9FF4FC5B016468F
:101790000546FEF758F8FEF762F8FEF76BF8429040
:1017A00000204190489800289CBF49B0BDE8F08FC8
:1017B00000214198469A00EBC00002EB8004A1830F
:1017C00094F82110012940F0FD804699627811F8C3
:1017D0002010429802FB00108021305C00F03F098D
:1017E000684603F04EFC802120A803F04AFCB4F9BF
:1017F000020045F256514143C0104390A0798DF844
:10180000000120798DF80101E0798DF802016079FD
:101810008DF80301A07920722079A0720A14E07972
:1018200000276072A2EBE17163790FFA81FCB84680
:101830003A46E3729842C0F0C5802179A07981428E
:1018400058D8429803FB001080B216F800A00AF0A6
:101850003F0ACA4549D135F910B0DDF80CA1D3458E
:1018600019DD9DF800A18A4588BF8DF800119DF80B
:1018700001A18A4538BF8DF801119DF802A19A4552
:1018800088BF8DF802319DF803A19A4538BF8DF8C5
:101890000331521C92B235F910A0E24515DD94F8DF
:1018A00008A08A4588BF217294F80AA08A4538BFEB
:1018B000A17294F809A09A4588BF637294F80BA0AE
:1018C0009A4538BFE3727F1CBFB20DF1800B35F92A
:1018D00010E05BF823A0F2444BF823A05DF821A0B0
:1018E00035F9100050444DF82100481CC1B2A079D0
:1018F0008842A6D2581CC3B2E07998429DD2002AF1
:101900005DD0234640AA20A96846FFF7AEFE4FF0FF
:10191000000A6179E079D4465346884224BF49F0F1
:10192000C00043904BD32079A279904230D8429A9C
:1019300001FB020292B216F802B00BF03F0ECE4548
:1019400021D19DF800E186459CBF9DF801E17045DD
:1019500013D89DF802E18E459CBF9DF803E17145C7
:101960000BD835F91220904402FB00AA02FB01CCEF
:101970005A1C0FFA88F893B205E0DDF80CE12BEA67
:101980000E0B06F802B0401CA279C0B28242CED241
:10199000481CC1B2E0798842C5D283B19DF80001EC
:1019A00020719DF8020160719DF80101A0719DF800
:1019B0000301E071C4F81080A381C4E905AC002FD5
:1019C00018BFA78341984899401CC0B241908842F3
:1019D000FFF4EEAE49B0BDE8F08F2DE9FF4F91B0B6
:1019E00000201090019002900390049005900690C2
:1019F0000790089009900A909A46914606460B90E7
:101A00000C900D900E900F90FDF70AFF0446FDF725
:101A10001AFF0746207B04F1370502281ABF032866
:101A200005280126207D012819D010AB51464846D3
:101A3000119AFEF74AFE9DF8400001280AD93C227F
:101A4000944901A803F022FB01AB51464846119A84
:101A5000FFF7FCF99DF84030022B33D06AE0607D3F
:101A600001280BD03C228B4901A803F00FFB01ABEE
:101A700051464846119AFFF7E9F97BE00021D44628
:101A800001AB0A460846B9F1000F73D900EBC00458
:101A90000CEB840494F82140012C04D171B1521C48
:101AA00023F81010D2B2401CC0B24845EED3012A30
:101AB00084BF03EB410020F8021C5BE0411CC9B26B
:101AC0000122F0E79DF84100012819D1002101AA67
:101AD0000846B9F1000F0ED932F810C0BCF1000F62
:101AE00001D0491C03E0401CC0B24845F4D3002992
:101AF00018BF012000D102208DF84100022B19D11E
:101B0000C0B2022816D100200190029003900490E8
:101B1000059006900790089009900A900B900C9001
:101B20000D900E900F909DF84200002804BF0120F8
:101B30008DF84200002E04BF207D00281AD197F8AE
:101B40003100052818BF032814D1022B12D9002018
:101B500001900290039004900590069007900890E1
:101B600009900A900B900C900D900E900F90012010
:101B70008DF842000026B9F1000F3BD901AF37F8CC
:101B8000161099B306EBC6000AEB800494F8210006
:101B900001282BD15246701CFFF700FA701C00F090
:101BA000FF0817F81670FDF765FE84466179E07945
:101BB00088421BDB2079A279904212DC01FB0C02E7
:101BC00092B2AB5C03F03F0BC34505D103F0800339
:101BD00043EA070B05F802B0401CA27900B282422A
:101BE000ECDA481C01B2E0798842E3DA701CC6B234
:101BF0004E45C3D3129CFDF726FEFDF711FE0021D2
:101C000080F82D1049465046FEF72AFB2CB10346BA
